:020000040800F2
:100000000000022019E70B089DE70B08E1AF060886
:100010009DE70B089DE70B089DE70B08000000001B
:100020000000000000000000000000009DE70B0839
:100030009DE70B08000000009DE70B08D944050868
:100040009DE70B089DE70B089DE70B089DE70B0854
:100050009DE70B089DE70B083126050835260508A6
:10006000392605083D26050841260508E53F040810
:10007000F93F04080D4004082140040835400408F5
:10008000494004085D4004089DE70B089DE70B0804
:100090009DE70B089DE70B089DE70B084526050823
:1000A0009DE70B089DE70B089DE70B08614A0408D4
:1000B000754A0408894A04089D4A0408093304085B
:1000C000FD3204083D330408313304089DE70B0872
:1000D0009DE70B0825550408315504083D550408D3
:1000E000492605089DE70B0800000000D94A0408CE
:1000F000294B0408514B0408C54A04087140040800
:100100009DE70B0899650408B14A04089DE70B08B0
:10011000495504089DE70B089DE70B08F197040873
:100120008540040899400408AD400408C140040813
:10013000D54004089DE70B089DE70B089DE70B08D9
:1001400000000000000000000000000000000000AF
:10015000E9400408FD40040811410408555504080D
:1001600071330408653304089DE70B089DE70B080D
:100170009DE70B089DE70B089DE70B0800000000BA
:100180009DE70B089DE70B08615504086D550408B1
:100190009DE70B089DE70B089DE70B089DE70B0803
:1001A0009DE70B089DE70B089DE70B089DE70B08F3
:1001B0009DE70B089DE70B089DE70B089DE70B08E3
:1001C0009DE70B089DE70B089DE70B089DE70B08D3
:1001D0009DE70B08018404089DE70B089DE70B08C9
:1001E0009DE70B089DE70B089DE70B089DE70B08B3
:1001F0009DE70B089DE70B089DE70B089DE70B08A3
:100200009DE70B089DE70B089DE70B089DE70B0892
:10021000ED4A0408014B0408154B04089DE70B0840
:100220009DE70B089DE70B089DE70B080000000009
:100230009D6504089DE70B08000000009DE70B0882
:100240009DE70B089DE70B089DE70B089DE70B0852
:100250009DE70B089DE70B089DE70B089DE70B0842
:100260009DE70B089DE70B089DE70B089DE70B0832
:100270009DE70B089DE70B089DE70B0800000000B9
:100280009DE70B08000000009DE70B080000000040
:08029000000000009DE70B08CF
:08029800C4D60B0001000000B8
:1002A00078A50124020100000200140098A5012491
:1002B0000202000002001400B8A50124020A000096
:1002C00002001400D8A50124020300000400140059
:1002D000F8A50124020800000400140018A6012457
:1002E000010B00000001770038A60124010C00007A
:1002F0000001760058A601240110000000017600DC
:1003000078A60124010D01000001770098A60124C0
:100310000112000000017600B8A6012401140000BB
:1003200000001E00D8A60124011A000000000D00E4
:10033000F8A60124011B000000002C0018A70124CE
:100340000115000000000C0038A701240116000070
:1003500000000C0058A70124011C000000000E0042
:1003600078A70124011D000000001E0098A70124A9
:100370000117000000000C00B8A7012401180000BC
:1003800000000E00D8A701240119000000000C0095
:10039000F8A70124011F000000000C0018A8012488
:1003A0000120000000000C0038A8012401290100F0
:1003B0000001180058A80124012100000001480094
:1003C00078A80124012200000001490098A8012416
:1003D0000123000000014A00B8A801240124000004
:1003E00000014B00D8A801240125000000014C00A9
:1003F000F8A801240126000000014D0018A90124DD
:100400000127000000014E0038A901240128000046
:1004100000014F0058A90124012C00000000290010
:1004200078A90124012D01000000290098A90124C8
:10043000012E010000007000B8A901240130000065
:1004400000003100D8A90124012F01000000520052
:10045000F8A90124013101000001280018AA012493
:10046000013201000001280038AA012401350000F2
:1004700000003C0058AA01240138000000002000C0
:020000040804EE
:10000000836B5A6D12F0500F5A6D1AD1196842F471
:1000100000725A650A6812F0080FCA6816D012F406
:10002000406F15D1CA68920412D45A6D22F48072BE
:100030005A655A6DD1040BD45A6D42F001025A65CB
:100040007047D20604D4DB6CDB6C18479007ECD009
:10005000704700BF704700BF836B5A6D42F040028B
:100060005A659A6D42F004029A65704702685549D4
:1000700038B5554B554D564CAA4218BF9A420CBF45
:10008000012300238A4208BF43F001033031A2421A
:1000900008BF43F0010330348A4208BF43F0010334
:1000A0003031A24208BF43F0010330348A4208BF16
:1000B00043F0010301F55C71A24208BF43F0010364
:1000C00004F55C748A4208BF43F001033031A24258
:1000D00008BF43F0010330348A4208BF43F00103F4
:1000E0003031A24208BF43F0010330348A4208BFD6
:1000F00043F001033031A24208BF43F001038A42BA
:1001000008BF43F0010313B9324B9A4208D10423CC
:1001100080F83530136823F001031360002038BDE8
:100120002D4B2E4D1168AA4218BF9A422C4C21F03B
:100130000E0105F13C050CBF012300231160A24212
:1001400008BF43F0010311682834AA4208BF43F0F6
:10015000010321F00101A24208BF43F0010314345E
:100160001160A24208BF43F001031E498A4208BF42
:1001700043F0010313B91C4B9A4217D10123856D3B
:10018000D0E91714226801F01F0122F480728B401D
:1001900022606B60C36ED0E91921516033B11A68D7
:1001A000D0E91C1422F480721A604C6001210022F4
:1001B000036D80F8351080F83420002BAED09847BE
:1001C000ACE700BF4000024010000240280002409F
:1001D00058000240B80402401C5402580854025807
:1001E0003054025880540258945402580168002236
:1001F0000B6880F842205A0410B40ED50B6823F423
:1002000080430B6090F84130292B10D090F841309A
:100210002A2B24D05DF8044B70471B04F2D50B68E1
:1002200023F400430B6090F84130292BEED12822B3
:10023000212380F841200022036390F841300C68AC
:1002400003F02803282B14BF6FF0F2036FF0420372
:1002500023405DF8044B0B6080F840207047282253
:10026000222380F841200022036390F841300C687B
:1002700003F02803282B14BF6FF0F4036FF044033E
:1002800023405DF8044B0B6080F84020704700BFAE
:100290000023202210B4174C4363C462036380F828
:1002A000412080F842304B07026811D5526A436AF8
:1002B0001A70436A028D013343624AB1438D013A99
:1002C000013B02859BB24385436C43F004034364C6
:1002D0000368102490F84120002190F841201A680A
:1002E00022F0FE021A60DC615DF8044B80F84010D9
:1002F000704700BF0000FFFF70B5574B002590F816
:100300004120044680F84250283AC3624585436C38
:10031000022A41EA0301036841642FD890F8411092
:1003200090F84120282001F0280102F02802282915
:1003300014BFF6214621282A1A680CBFC9436FF062
:10034000F6010A4045491A6084F84100A06B226B0F
:10035000616318B1112A42D0212A40D0E06B18B154
:10036000122A51D0222A4FD094F84130602B4FF0FE
:1003700000032DD0236384F8403070BD90F84120F5
:1003800090F841201A6822F0FE021A609A699207DA
:1003900000D59D629A69D60703D49A6942F001029A
:1003A0009A6194F84120602A10D0202284F84120DC
:1003B0009A6995060AD59A69D00605D51022DA61A0
:1003C000626C42F0040262642022DA610021BDE71F
:1003D000202284F8403084F84120236370BD1A68DD
:1003E00051042CD490F83530012BBDD000221C4B89
:1003F000036584F8402090F83520022A24D080221A
:100400004265BDE8704018471A68120403D51A689F
:1004100022F400421A6090F83530012BA4D000225B
:100420000F4B036584F8402090F83520022AE6D16E
:10043000FFF71CFE0028A0D0E06B036DE1E71A680F
:1004400022F480421A60CDE7FFF710FE002894D016
:10045000A06B036DD5E700BF0000FFFFDD040408BB
:100460002D08040803689A69196810B4D40528D5C2
:100470000C0606D4416C11F00B0F1FD15DF8044B34
:100480007047416C4FF4807441F0010141645105A3
:10049000DC6120D5416C4FF48064920541F0080185
:1004A0004164DC61E6D5426C4FF4007142F0020217
:1004B0004264D961416C11F00B0FDFD05DF8044B41
:1004C0001AE7540502D50906E4D4D3E79405D1D53B
:1004D0000906E8D4CEE79205E5D4CBE7F8B590F865
:1004E00040300D46C16A012B00F008810123AE06A1
:1004F000044680F8403001D5900656D4EB0619D555
:10050000D70617D5638D9BB2002B40F0F98094F885
:100510004130B1F1007FDBB240F0D580282B40F0B4
:10052000D28029462046FFF7B3FE0023184684F800
:100530004030F8BD68071AD42F0701D516074AD4F2
:10054000A807F2D59307F0D5638D9BB2002B00F07E
:10055000FA80616A236811F8010B228D9862638D1D
:10056000013A6162013B22859BB26385DDE7530757
:10057000E2D5638D9BB26BB12268636A526A1A70CE
:10058000638D606A228D013B0130013A9BB260624B
:1005900022856385638D9BB2002BC6D111F5803F08
:1005A000C3D02046FFF722FEBFE72368202118684A
:1005B000E66A94F84120D961213A092A1ED8DFE879
:1005C00012F0C70015001D001D001D001D001D00BC
:1005D000F000C700150094F84130226803F02803AA
:1005E000282B00F0C5800823D3619EE794F84120B2
:1005F0001A6822F0FC021A60222222635A68894992
:1006000042F400425A605A680A405A609A69910757
:1006100001D500229A629A69D20703D49A6942F0FE
:1006200001029A6147047BD51A6822F480421A605D
:10063000A26B1AB111684A6892B262856A070BD53B
:100640005A6A25F00405636A1A70636A01336362AB
:10065000238D002B40F08580638D9BB21BB1636CB2
:1006600043F004036364EB061AD5C70618D5638DFF
:100670009BB2002B40F0AA8094F84130282B03D184
:10068000B6F1007F00F0C98094F8413016F5803F44
:100690002268DBB202D0292B00F0AD801023D36199
:1006A000002384F84230666C6363002E40F084803F
:1006B000E36A5D4DAB423DD194F84130202384F88C
:1006C0004130266331E794F841202368292A4FF00E
:1006D0001002DA617FF429AF11F5803F3FF425AFB6
:1006E0009A69960701D500229A629A69D5073FF563
:1006F00058AF9A6942F001029A6152E70220F8BDB0
:1007000023681022DA61636C43F00403636431F000
:1007100080737FF40AAF616C2046FFF7EDFD04E7BC
:1007200001048BD51A6822F400421A60E26B002A99
:1007300080D183E72046FFF759FD2023E56284F846
:1007400041302663F1E631F080737FF4EEAE28E7A6
:1007500094F841201A6822F0FA021A6021222263DA
:100760004CE7013B2385638D013B9BB2638573E7B7
:10077000E1689369022990699368D56836D1C3F31B
:10078000C21383EA104313F006032FD1A16C013189
:10079000A164A16C02297FF4C8AE0821A364D161D1
:1007A000C3E694F8412094F841201A6822F0FE0232
:1007B0001A600022226321E7616C2046FFF79CFD4E
:1007C00094F84130282B7FF4B0AEAAE623681022BB
:1007D000DA61636C43F00403636436F080737FF482
:1007E0005FAF616C2046FFF787FD59E7136823F080
:1007F000B803136099E61023D3619369980701D574
:10080000002393629369D90703D4936943F00103EA
:1008100093612046FFF7EAFC42E729462046FFF7AE
:1008200037FD3DE700E800FE0000FFFF836B9A6B99
:100830000AB100211165DA6B0AB10021116593F844
:100840004120602A05D000221A63002283F840204C
:1008500070470022202183F841101A63002283F898
:1008600040207047016870B4CC072DD5914A1369B8
:10087000926A03F03803102B00F0E180182B00F08F
:10088000D9804368B3F5803F00F00581002B00F06C
:100890005A81B3F5A02F874B1A6800F0678222F4C3
:1008A00080321A601A6822F480221A60824B41F268
:1008B000883C804C1D6804E01A68521B624500F2B7
:1008C0003F8122689603F7D58A0768D4CD0631D5D3
:1008D000784A1369926A03F03803082B00F0C0804D
:1008E000182B00F0B880C369724C002B00F05F81B8
:1008F0002268714B42F0800222601D6804E01A6891
:10090000521B022A00F21C812268D205F7D56B4BDC
:10091000026A1D6841F20303B3EB154FC0F0448235
:100920006368202A23F0F8430CBF43F0804343EA76
:10093000826363600D0713D543695E4C002B00F0A2
:100940001881626F5C4B42F0010262671D6804E02F
:100950001A68521B022A00F2F380626F9207F7D5E1
:100960008C0613D58369534C002B00F0118122684B
:10097000514B42F4805222601D6804E01A68521BF9
:10098000022A00F2DD8022689204F7D5490700F1BF
:100990008880436A002B40F0BC80002059E0454A23
:1009A0001369926A13F038032BD1424AC368126864
:1009B000520701D5002B4BD03E4C226822F0190281
:1009C0001A433D4B22601D6804E01A68521B022A3C
:1009D00000F2B68022685607F7D5384B02691D68C9
:1009E00041F20303B3EB154F6368C0F0028123F4B7
:1009F0007C33402A0CBF43F4003343EA0233636084
:100A000064E7182B00F0F180C3682A4C002B00F03B
:100A1000DD80226822F019021A43274B22601D68EC
:100A200004E01A68521B022A00F28A8022685207E8
:100A3000F7D5D2E702F00302022A7FF422AF1D4B62
:100A40001B689B037FF540AF4368002B7FF43CAFEE
:100A5000012070BC704702F00302012A7FF443AF0B
:100A6000144B1B68DC0502D5C369802BF0D1134CF5
:100A700041F20303026A2468B3EB144FC0F0BF8055
:100A8000202A00F09E810B4C636823F0F84343EA70
:100A9000826363604EE7074A136843F48033136050
:100AA00004E70749044B0A6842F480720A601C6834
:100AB0000CE000BF00440258002E00240010005C2F
:100AC000004802581A68121B642A39D80A68D505EA
:100AD000F8D58268012A00F06E81002A00F04E816C
:100AE000052A9F4A116F00F0748121F001011167FE
:100AF000116F21F0040111671D6841F28834984993
:100B000003E01A68521BA2421AD80A6F9207F8D55E
:100B10003FE793490A6902F03802182A00F0D580AD
:100B20000A68022B8F4B22F080720A606FD018681F
:100B30000A6892017FF531AF1A68121A022AF7D9B2
:100B4000032070BC7047864C41F28835854B226883
:100B500022F480322260226822F4802222601E6801
:100B600003E01A68921BAA42EAD822689203F8D4DA
:100B7000AAE6626F7B4B22F0010262671D6803E008
:100B80001A68521B022ADBD8626F9607F8D4E7E690
:100B90002268744B22F4805222601D6803E01A68B8
:100BA000521B022ACCD822689604F8D4EEE62268BA
:100BB0006C4B22F0800222601D6803E01A68521B11
:100BC000022ABDD82268D605F8D4B3E62268654B60
:100BD00022F0010222601D6803E01A68521B022AFB
:100BE000AED822685607F8D470E694077FF40CAFAD
:100BF000DBE623F0FE4343EA0263636066E6584C9B
:100C0000E36823F07C5343EA0263E36092E61C68E6
:100C100003E01A68121B022A92D80A689501F8D4D8
:100C20008C6A514A2240846A2243C46A42EA04120E
:100C30008A62D0E90D24013A013C5202240492B2A6
:100C400004F4FE042243046B013CC4F30804224371
:100C5000C46B013C240604F0FE4422430A63CA6AC2
:100C600022F00102CA624A6B846C6FF3CF0242EA3F
:100C7000C4024A63CA6A046C22F00C022243384C54
:100C8000CA62CA6A406C22F002020243CA62CA6A9D
:100C900042F48032CA62CA6A42F40032CA62CA6A44
:100CA00042F48022CA62CA6A42F00102CA620A6839
:100CB00042F080720A601968226890013FF56DAEBB
:100CC0001A68521A022AF7D93AE7012B8A6A0D6B81
:100CD0003FF4BEAE02F00303846AA3427FF4B8AED1
:100CE000C2F30512C36A9A427FF4B2AE036BC5F336
:100CF0000802013B9A427FF4ABAE436BC5F3462238
:100D0000013B9A427FF4A4AE836BC5F30642013BDC
:100D10009A427FF49DAEC36BC5F30665013B9D42CD
:100D20007FF496AE4B6B816CC3F3CC0399423FF4D6
:100D300034AE0B480B4BC26A22F00102C2621A6841
:100D400018688242FCD0064A536B6FF3CF0343EA24
:100D5000C1035363D36A43F00103D3621DE600BFAE
:100D600000440258002E00240CFCFFFF42F48022B5
:100D70001A601A6842F480321A6097E5194941F204
:100D800088350A6F22F001020A670A6F22F0040216
:100D90000A671C6804E01A68121BAA423FF6D0AE2C
:100DA0000A6F9607F7D4F4E5E36823F07C5343EA2F
:100DB0000263E360BEE50B490A6F42F001020A6775
:100DC0009AE6084A536823F0F84343F0804353609F
:100DD000B0E541F004011167116F41F001011167A5
:100DE0008AE600BF00440258334B30B4996A9C6ACB
:100DF000DD6A14F47C7F5A6BC4F3051036D0C2F35D
:100E0000CC0205F0010501F0030107EE900A05FB95
:100E100002F20129B8EEE77A06EE902AFAEEE96AC4
:100E200002D0022942D019B3DFED247A87EE876A17
:100E30001B6BC3F3080307EE903AF7EE005AF8EE87
:100E4000E77A77EEA67A77EEA57A67EE867A1A4B7E
:100E50001B6BC3F34623013307EE103AF8EEC76A63
:100E600087EEA67AFCEEC77A17EE900A30BC704780
:100E70001A6892061DD51968F7EE005A104A1B6BC6
:100E8000C1F3C101C3F30803CA4007EE903A06EE6E
:100E9000102AF8EEE77AB8EEC66A77EEA66AC6EED2
:100EA000077A36EEA57A67EE877AD0E7DFED057A26
:100EB000BCE7DFED057AB9E7004402580024744A24
:100EC0000090D00320BCBE4B0024744C836A1A07E8
:100ED00010B406D50168846B4A6822F400422243AC
:100EE0004A60DC0706D50168C46A4A6822F4003209
:100EF00022434A60990706D50168046B4A6822F4C8
:100F0000803222434A605A0706D50168446B4A681A
:100F100022F4802222434A60DC0606D50168C46BB5
:100F20008A6822F4805222438A60990606D50168B5
:100F3000046C8A6822F4005222438A605A060AD559
:100F40000168446C4A68B4F5801F22F4801242EABA
:100F500004024A600BD01B0606D50268C16C5368B8
:100F600023F400230B4353605DF8044B70474A6839
:100F7000846C22F4C00222434A60ECE70022836BB7
:100F8000A3F85E20704700BF124B41F2883C124A22
:100F900001461B68A2FB03235B0A0CFB03F33BB176
:100FA0004A6B12F0450F01D0920404D5013BF7D1F2
:100FB0004FF0004070474B6B5B0707D4486B10F055
:100FC000010014BF0123054B8B63704704231846AF
:100FD0008B63704700000024D34D6210C5002000D1
:100FE000036942681F2B70B430D9A3F1200520217A
:100FF0005468A940214227D08169087C022835D055
:1010000048681F2BC9681B4D4E680169C1F3032452
:10101000194951F8244015F804C0056856F80C40E9
:1010200024F0010446F80C40407901EB4001088CA3
:10103000E96800F4F05021EA0001E96010D9A3F159
:10104000200120238B40D36070BC7047202114689E
:1010500099402142F8D08169087C0228D0D105E06E
:10106000202101FA03F370BC9360704700200874DC
:10107000C6E700BFC8750C0858740C08D0E90723F0
:101080009A423CBFC1685218D01A7047D0E9092370
:1010900000699A4238BF12180138D31AC01A704733
:1010A000D0E90902101AB0FA80F04009704700BF79
:1010B000016A034640694A1C405CD9688A4228BFDD
:1010C00000221A62704700BF436A826910B4D1548B
:1010D000436A416B046901330A68A34228BF0023B5
:1010E0005DF8044B42F0800243620A60704700BF23
:1010F000436BD86910F0100002D0102201201A6250
:10110000704700BF704700BF704700BF704700BF07
:1011100001207047014B5868704700BF002E002423
:10112000074B93F8A422012A01D10020704793F8BD
:10113000A402A0F10300B0FA80F04009704700BF9C
:10114000002E0024012380F849307047EFF311820C
:10115000702383F312880849D2B2D1E9B93182F3FE
:101160001188581E8B42A0EB01008CBF0023012385
:1011700000EB0330704700BF002E002470B5D0F89C
:10118000D442D0F8C86200EB840EDEF8C05245B3FA
:1011900001F00F040A4604EB840C00EB8C0CDCF825
:1011A00018306BB9DEF8C43200211B69C5F814127F
:1011B00023B105F50471D5F808029847002070BDE9
:1011C00004EBC40406EB8406F469B3FBF4F604FBF9
:1011D0001633002BE6D11A46CCF818307AF0C6F94F
:1011E000ECE7032070BD00BFD0F8D42200EB8202F0
:1011F00010B5D2F8C042ACB101F00F03D0F8C8026C
:10120000D2F8C42204F5037103EBC303D26800EBE8
:101210008303D4F80402D3F86832C4F80C32904740
:10122000002010BD032010BDD0F8D43200EB8300A5
:1012300010B5D0F8C04284B1D0F8C4325BB194F894
:101240000002FF2807D09B68214694F801229847A6
:10125000FF2384F80032002010BD032010BD00BF22
:1012600030B52B4C86462379E5889D4242D91846F5
:10127000043419461A4602E0954246D921780C44B6
:101280000A44617892B20529F6D1A1788229F3D176
:101290009C461A461F4903E0AA4234D291F800C086
:1012A0006144624491F801C092B2BCF1050FF3D1E0
:1012B00091F802C0BCF1010FEED1164A02E0A8423B
:1012C0001DD213781A44034492F801C098B2BCF1BD
:1012D000050FF4D19378812BF1D10CB11023A371B8
:1012E00019B10020022308714B711AB100210223A9
:1012F0001171537143230748AEF8003030BD00220E
:10130000002CEBD1ECE70021D7E70024C0E700BFB9
:10131000000000240400002430B52B4C86462379BD
:10132000E5889D4242D91846043419461A4602E01F
:10133000954246D921780C440A44617892B2052935
:10134000F6D1A1788229F3D19C461A461F4903E0C1
:10135000AA4234D291F800C06144624491F801C0BD
:1013600092B2BCF1050FF3D191F802C0BCF1010FAC
:10137000EED1164A02E0A8421DD213781A44034463
:1013800092F801C098B2BCF1050FF4D19378812B8B
:10139000F1D10CB11023A37119B100204023487181
:1013A0000B711AB100214023517113714323074877
:1013B000AEF8003030BD0022002CEBD1ECE700216C
:1013C000D7E70024C0E700BF000000240400002489
:1013D000A2E700BF03460A2201481A80704700BFF7
:1013E00048000024064B4FF0120C064AA3F11400EB
:1013F000526DA1F800C0022A18BF1846704700BFFE
:101400006800002400400058042301480B80704706
:101410007C0000242DE9F047046982B0C3681C40B9
:1014200046D0814688464FF0004501F1500701F152
:101430003806B4FA84F325FA03F21B3BD243144076
:10144000C9F81020B8F1000F5FD0042B2ED8DFE8C8
:1014500003F052483D320300D8F81030D9F82CA0E0
:1014600033B19B6823B11FFA8AF108F1080098474D
:10147000D8F8283033B19B6823B11FFA8AF108F1FC
:1014800020009847D8F8403033B19B6823B11FFA49
:101490008AF108F138009847D8F8583033B19B6882
:1014A00023B11FFA8AF108F150009847002CC0D1EF
:1014B00002B0BDE8F087D8F8103008F10800D9F87C
:1014C00034105B689847002CB3D1F1E7D8F8283086
:1014D00008F12000D9F838105B689847002CA8D193
:1014E000E6E7D8F840303046D9F83C105B689847BA
:1014F000002C9ED1DCE7D8F858303846D9F8401097
:101500005B689847002C94D1D2E7042B07D8DFE81A
:1015100003F01903140F0A00D9F83C300193019B22
:10152000002C86D1C4E7D9F82C300193019BF7E752
:10153000D9F834300193019BF2E7D9F838300193A0
:10154000019BEDE7D9F840300193019BE8E700BF2C
:101550000A49D1F8EC324A685BB1002AFCD0013A62
:1015600010B513F8014B4A60C1F8EC3212B12046B5
:1015700010BDFEE779F0C2FF204610BD002E00240A
:10158000F8B50E4E96F8A432012B00D1F8BD96F8AE
:10159000A432032BFAD10D461446D6F8F07208E0B7
:1015A00008F0CCF9D6F8F032241A0544DB1B322BB4
:1015B000ECD8002C21462846F2DCF8BD002E002491
:1015C000F8B590F848305D1C0344EDB280F84850FF
:1015D00083F8341090F8493053B1132D07D9002304
:1015E00080F84830104F97F8A432012B05D1F8BD90
:1015F00080F84830002DF5D1F8BD97F8A432032BC0
:10160000F5D1D7F8F06200F134042946204608F0FD
:1016100095F9D7F8F0322D1A04449B1B322BE6D8EB
:10162000002DF2D1F8BD00BF002E0024F8B5002334
:1016300090F84850A0F8483005B9F8BD0D4F97F81C
:10164000A432012BF9D097F8A432032BF5D1D7F8A7
:10165000F06200F134042946204608F06FF9D7F80B
:10166000F0322D1A04449B1B322BE6D8002DF2D108
:10167000F8BD00BF002E00242DE9F04101210446F1
:101680004FF4077085F02EFC054600286CD0D4F886
:10169000D46204EB8606C6F8C002237CC4F8BC0200
:1016A000002B40D0402302228121204679F098FC73
:1016B0000121402302222046218779F091FC4FF03E
:1016C00001080823032282212046A4F8788179F0BA
:1016D00087FC294B0027E364D6F8C432C5F80472AE
:1016E0001B689847D5F80402C5F81472C5F818723B
:1016F00000283ED0227CD4F8C83222BBC3F88C220A
:101700004FF400749A7903F51E71C3F88402012A1C
:10171000A3F87882C3F8884223D0186879F0DEFDF8
:101720000020BDE8F08120464FF4007302228121A1
:1017300079F056FC01214FF40073022220462187E4
:1017400079F04EFCBBE79A79402403F51E71C3F88B
:101750008C72012AC3F88402A3F87882C3F8884205
:10176000DBD1C3F89402D8E7D4F8D432B03344F8CC
:1017700023000220BDE8F08101001000F8B5D0F888
:10178000C85240F20112044695F894342A87012B7E
:101790003ED00126002728683246314685F89464F9
:1017A00079F064FF27873A4631462868A5F87862C1
:1017B00085F8946479F05AFF4FF48173A4F8787136
:1017C00032460221286885F89464A5F85C3079F0E7
:1017D0004DFF85F89474D4F8D432002504EB8303CC
:1017E000E564D3F8C0228AB1D3F8C4325B68984765
:1017F000D4F8D432B03354F8230084F003FCD4F886
:10180000D432B03344F82350C4F8BC520020F8BDA1
:1018100000224FF481710287A5F87832A0F8782170
:10182000A5F85C10D7E700BFD0F8D43200EB8303F3
:10183000F0B5002683B0D3F8C0728DF80560ADF81E
:1018400006605FB191F800C004460D461CF06002CE
:101850002FD0202A05D0204679F006FD032003B0C2
:10186000F0BDCA884878002A42D01CF0800F00F0F2
:101870008380D3F8C43239469B689847EA880223AC
:101880004FF48071072AC4F8943228BF0722D4F895
:10189000C832C4E906225A629A79998203F1140186
:1018A000012A1F629E6200D11F63186879F016FD3D
:1018B00022E04B780B2BCED801A252F823F000BFC8
:1018C000FD180408F91804085718040857180408E4
:1018D000571804085718040857180408571804081C
:1018E00057180408571804083D1904083319040848
:1018F000D3F8C4329B6898470020B0E790F89C3238
:10190000032BA8D10222D0F8C8320020C4F89422B8
:1019100003F11401C4E906220DF106049862C3E93B
:1019200008424FF480729A829A79012ABDD11C63D1
:10193000BBE790F89C32032BDED08CE790F89C320A
:10194000032B88D101220221D0F8C832C0F89412AA
:1019500003F11401C0E906220DF10500C3E90802F4
:101960004FF4807200209A829A799862012A9CD161
:101970000DF10500186398E7402A4FF0030387F83C
:10198000000228BF402287F80122C4F89432D4F81C
:10199000C832C4F85821C4F85C2103F51571C3F8A6
:1019A00064229A79C3F86072012AC3F86862A3F8C6
:1019B000546208BFC3F8707277E700BF70B5124D6C
:1019C000124A2B68A2FB03239B09013BB3F1807FE2
:1019D00001D3012070BD4FF0E0220D4900240F28F3
:1019E00053614FF0F003064681F823304FF00703B0
:1019F00094611361EDD801464FF0FF3076F0F0F9B5
:101A00002046C5F8806070BD00000024D34D6210F0
:101A100000ED00E03749024603688B4233D01831AD
:101A2000591AB1FA81F1490969BB3348834240D060
:101A30001830834240D01830834236D01830834269
:101A40003DD01830834240D0183083422CD000F56E
:101A50005670834237D029498B4233D018318B429C
:101A600036D018318B4236D018318B4236D01831EF
:101A70008B4236D018318B4236D018318B4236D05B
:101A800023F0FF0013E0DBB21D491E48103B10B4E9
:101A90001D4CA4FB03435DF8044B01EB131393F8B7
:101AA0002810C2E91601704716211848D1659065C3
:101AB000704710211348F9E716211248F6E706216E
:101AC0001248F3E706211248F0E710210F48EDE72E
:101AD00010210F48EAE716210D48E7E700210D48DD
:101AE000E4E706210B48E1E710210A48DEE716216A
:101AF0000848DBE710000240400002402804024092
:101B000058740C0800000240ABAAAAAA04000240C4
:101B10000004024004040240F0B50C46114602687D
:101B20008646936913F0100C72D04FF0000C10230E
:101B300038486546D36193699E065FD445B903680A
:101B40005B1AA3423DD893699F06F8D52023D36141
:101B50004CF0040C01209369D90552D54FF48071E3
:101B60005F054CF0010CD16104D54FF480614CF05D
:101B7000080CD1619D0504D54FF400734CF0020CA4
:101B8000D3619369990701D5002393629369DB07B9
:101B900003D4936943F001039361536820241E49E1
:101BA00001200B4000215360DEF844308EF84010D5
:101BB00043EA0C03CEF844308EF841408EF84210D0
:101BC000F0BD57689EF842309669DBB2360408D5FE
:101BD0007E0406D4202B04D0536843F48043536022
:101BE000016893699F06A6D403685B1A192BF8D97C
:101BF00093694FF0200C01259E069FD5002DA5D09E
:101C0000A6E75E05B1D49C05B6D40028B9D1F0BDD5
:101C10006046A0E7002E002400E800FE2DE9F04712
:101C200007689A46089EBB6931EA03030CBF01238B
:101C30000023934220D180460C461546DFF85C9085
:101C4000324651464046FFF767FF20BBD9F80030C7
:101C5000A3EB060CD44507D9BB6934EA03030CBFD8
:101C600001230023AB420AD0BB6934EA03030CBF53
:101C700001230023AB42E3D00020BDE8F087D8F871
:101C80004430202288F840001343C8F8443088F8D4
:101C9000412088F842000120BDE8F087002E002492
:101CA0000C4A136903F03803102B0DD0182B09D000
:101CB00063B913689B060BD513680748C3F3C103C8
:101CC000D8407047FFF790B8044870470448704701
:101CD00001487047004402580090D00340787D01CD
:101CE00000093D00184A136903F03803102B10B5A2
:101CF00024D0182B09D01BBB13689B0622D5136870
:101D00001248C3F3C103D84001E0FFF76DF80E4954
:101D10000F4A8B698969C3F303230E4C01F00F014D
:101D200013440A4493F8301092F8303001F01F0247
:101D300003F01F03D0402060D84010BD0648E6E7FE
:101D40000648E4E70148E2E7004402580090D00367
:101D500058740C080000002440787D0100093D0003
:101D6000474A70B4946A956AD66A15F47C3FC5F305
:101D70000533D16B5BD0C1F3CC01C6F3001604F080
:101D8000030407EE903A06FB01F1012CB8EEE77A66
:101D900006EE901AFAEEE96A03D0022C6AD0002C03
:101DA0004AD0DFED387A87EE876A936BC3F3080376
:101DB00007EE903AF7EE005AF8EEE77A77EEA67A59
:101DC00077EEA57A67EE867A2D4AB7EE006A936BB6
:101DD000C3F3462307EE103AB8EEC77A70BC37EE6D
:101DE000067AC7EE876AFCEEE66AC0ED006A936B7E
:101DF000C3F3064307EE103AB8EEC77A37EE067A19
:101E0000C7EE876AFCEEE66AC0ED016A936BC3F326
:101E1000066306EE903AF8EEE66A76EE866A87EE9C
:101E2000A67AFCEEC77A17EE903A8360704770BCD2
:101E3000C0E900338360704713689B061DD51468A2
:101E4000F7EE005A936B1049C4F3C102C3F30803C1
:101E5000D14007EE903A06EE101AF8EEE77AB8EEA7
:101E6000C66A77EEA66AC6EE077A36EEA57A67EE00
:101E7000877AA9E7DFED057A95E7DFED057A92E746
:101E8000004402580024744A0090D00320BCBE4B8A
:101E90000024744C474A70B4946A956AD66A15F067
:101EA0007C7FC5F30553516C5BD0C1F3CC01C6F305
:101EB000002604F0030407EE903A06FB01F1012C22
:101EC000B8EEE77A06EE901AFAEEE96A03D0022C31
:101ED0006AD0002C4AD0DFED387A87EE876A136C1F
:101EE000C3F3080307EE903AF7EE005AF8EEE77AEC
:101EF00077EEA67A77EEA57A67EE867A2D4AB7EE68
:101F0000006A136CC3F3462307EE103AB8EEC77AA3
:101F100070BC37EE067AC7EE876AFCEEE66AC0ED63
:101F2000006A136CC3F3064307EE103AB8EEC77AA3
:101F300037EE067AC7EE876AFCEEE66AC0ED016A04
:101F4000136CC3F3066306EE903AF8EEE66A76EE9B
:101F5000866A87EEA67AFCEEC77A17EE903A83601F
:101F6000704770BCC0E900338360704713689B06FC
:101F70001DD51468F7EE005A136C1049C4F3C10262
:101F8000C3F30803D14007EE903A06EE101AF8EEBC
:101F9000E77AB8EEC66A77EEA66AC6EE077A36EE3C
:101FA000A57A67EE877AA9E7DFED057A95E7DFED99
:101FB000057A92E7004402580024744A0090D00346
:101FC00020BCBE4B0024744C0269836870B5044683
:101FD00005681343C069626986B029681343AC4A37
:101FE00003430A40616A1343E2682B606B6823F481
:101FF00040531343A2696B60A64B9D4200F066817B
:10200000236AAE681A43A44B33401A43AA60EB6AB2
:1020100023F00F030B43EB62A04B9D4228D0A04B53
:102020009D421AD09F4B9D4217D09F4B9D4214D08A
:102030009E4B9D4211D09E4B9D4219D09D4B9D427F
:102040000BD09D4B9D4208D0012000234FF0011280
:102050006367A266A36706B070BD984B5B6D03F023
:102060000703052BF0D8DFE803F09F7F8A925F79A2
:10207000924B5B6D03F03803282BE5D801A252F890
:1020800023F000BF31220408492004084920040835
:10209000492004084920040849200408492004086C
:1020A000492004086921040849200408492004083B
:1020B000492004084920040849200408492004084C
:1020C000492004087F210408492004084920040805
:1020D000492004084920040849200408492004082C
:1020E000492004088F2104084920040849200408D5
:1020F000492004084920040849200408492004080C
:10210000492004082921040849200408492004081A
:1021100049200408492004084920040849200408EB
:10212000492004085D210408B0F5004F644853D0ED
:10213000644B626803EB4103B3F84030B0FBF3F04B
:1021400000EB52004FF6EF73B0FBF2F0A0F110027B
:102150009A423FF679AFE860002076E7B0F5004F8D
:102160003AD04FF40040E3E7B0F5004F2DD003A87C
:10217000FFF7F6FD04980028EED0616AD8E7B0F5C5
:10218000004F71D06846FFF785FE0198F3E7B0F580
:10219000004F5ED0494B1A68920639D51B684A48F1
:1021A000C3F3C103D840C3E7B0F5004F32D0FFF707
:1021B00099FD424A434BD269C2F30212134493F889
:1021C000303003F01F03D840D5E703A8FFF7C8FD60
:1021D00004980028C0D0616A3A4B626803EB41035F
:1021E0004FF6EF71B3F84030B0FBF3F0530803EB58
:1021F0004003B3FBF2F3A3F110028A423FF624AF8F
:1022000023F00F02C3F3420392B21343EB60A3E740
:102210002D488DE7FFF766FD284A2A4BD269C2F3A5
:102220000212134493F8303003F01F03D840D0E774
:10223000B0F5004F1DD0FFF755FD204A214BD26964
:10224000C2F30222134493F8303003F01F03D84046
:1022500091E71A4B1A68900640F1A5801B681A484E
:10226000C3F3C103D840B7E76846FFF713FE0198F0
:10227000AFE7FFF737FD114A124BD269C2F30222D2
:10228000134493F8303003F01F03D840A1E700BF98
:10229000F369FFCF000C0058FFF4FF11001001405C
:1022A0000044004000480040004C00400050004006
:1022B0000014014000780040007C004000440258B7
:1022C00000093D0058740C080090D003A868374BF3
:1022D00003401343364AAB60EB6A23F00F030B4312
:1022E000EB62936D03F00703052B3FF6ADAEDFE81D
:1022F00003F0413C3303524F2D4B1A6895064CD4E2
:102300002C482D4B656803EB410305EB4501B3F801
:102310004020B0FBF2F399423FF696AEB3EB053F97
:102320003FF692AE002319467CF0DCF92A460902FA
:10233000030241EA1061680818184FF0000341F1E8
:1023400000017CF0CFF91D4BA0F540729A423FF698
:102350007BAE1B4BD860FFE66846FFF79BFD0198FC
:1023600000283FF4F9AE616ACBE703A8FFF7F8FC59
:102370000498F5E7FFF7B6FC0D4A0F4B126AC2F35B
:102380000212134493F8303003F01F03D840E7E7FC
:102390004FF40040B5E70B48B3E71B680548C3F3AB
:1023A000C103D840ADE7034816E700BFFFF4FF11B3
:1023B000004402580090D00358740C08FFFC0F0032
:1023C000000C005800093D00474A70B4946A956AB1
:1023D000D66A15F47C7FC5F30513516B5BD0C1F34E
:1023E000CC0106F0010604F0030407EE903A06FB68
:1023F00001F1012CB8EEE77A06EE901AFAEEE96ADE
:102400004ED0022C6DD0002C4DD0DFED387A87EE07
:10241000876A136BC3F3080307EE903AF7EE005A8E
:10242000F8EEE77A77EEA67A77EEA57A67EE867A07
:102430002D4AB7EE006A136BC3F3462307EE103A3A
:10244000B8EEC77A70BC37EE067AC7EE876AFCEE44
:10245000E66AC0ED006A136BC3F3064307EE103A59
:10246000B8EEC77A37EE067AC7EE876AFCEEE66A00
:10247000C0ED016A136BC3F3066306EE903AF8EE03
:10248000E66A76EE866A87EEA67AFCEEC77A17EEE3
:10249000903A8360704770BCC0E900338360704736
:1024A000DFED137AB3E713689B06AED51468F7EE39
:1024B000005A136B0F49C4F3C102C3F30803D140A0
:1024C00007EE903A06EE101AF8EEE77AB8EEC66A12
:1024D00077EEA66AC6EE077A36EEA57A67EE877AB9
:1024E000A6E7DFED057A92E7004402580024744C19
:1024F0000024744A0090D00320BCBE4B344A1368B9
:1025000030B423F08063334C1360256803E0236804
:102510005B1B022B54D813681B01F8D4936A05681F
:1025200023F47C3343EA053393628368C568013B37
:10253000013D5B022D049BB205F4FE052B4345686B
:10254000013DC5F308052B430569013D2D0605F046
:10255000FE452B439363D36A456923F0C0032B43A5
:10256000D362D36A856923F020032B43D362D36AF5
:1025700023F01003D362D36BC0696FF3CF0343EA38
:10258000C003D363D36A43F01003D362D36AD1B1DB
:1025900001290CBF43F4801343F40013D3620C4AA7
:1025A000136843F080631360216803E023685B1ABB
:1025B000022B05D813681B01F8D5002030BC7047EA
:1025C000032030BC704743F40023D362E7E700BF29
:1025D00000440258002E0024344A136830B423F01B
:1025E0008053334C1360256803E023685B1B022B88
:1025F00054D813689B00F8D4936A056823F07C7361
:1026000043EA055393628368C568013B013D5B0261
:102610002D049BB205F4FE052B434568013DC5F32F
:1026200008052B430569013D2D0605F0FE452B43AA
:102630001364D36A456923F440632B43D362D36A9E
:10264000856923F400732B43D362D36A23F4807328
:10265000D362536CC0696FF3CF0343EAC003536482
:10266000D36A43F48073D362D36AD1B101290CBF1A
:1026700043F4000343F08073D3620C4A136843F0C1
:1026800080531360216803E023685B1A022B05D88E
:1026900013689B00F8D5002030BC7047032030BC85
:1026A000704743F48003D362E7E700BF0044025859
:1026B000002E0024F0B5354AB0F1804F344DA0EB28
:1026C00002020368A0EB050E4C69B2FA82F28F6831
:1026D000BEFA8EFE0E684FEA52124FEA5E1E1FD0FF
:1026E000F2B9DFF8B8C0604537D00CF5806C6045B2
:1026F00033D00CF5806C604512D0BEF1000F0FD1C5
:10270000244D254A904218BFA8422AD002F5806283
:10271000904226D023F08003C76286621C4314E0F7
:102720004D6823F07003D1F80CC02B43C76286625A
:1027300023F4407343EA0C0323F080031C4312B9D3
:10274000BEF1000F16D00B6903630368012243F04A
:102750000403036042610460F0BD23F070034A6823
:102760001343CA6823F44073C7621343866223F09D
:1027700080031C43074A084B984218BF9042E2D09E
:1027800003F580639842DED0DFE700BF0000014020
:1027900000040140004001400044014000040040AA
:1027A000026810B452E8003F23F4907342E800310D
:1027B0000029F7D1144C02F1080353E8003F2340ED
:1027C00002F1080C4CE800310029F4D1C36E012B52
:1027D00008D0002320225DF8044BC0F88C2043670A
:1027E000C366704752E8003F23F0100342E800310F
:1027F0000029EED052E8003F23F0100342E80031F8
:102800000029EFD1E5E700BFFEFFFFEF436BDA6978
:10281000F0B5970683B0044642D5586AE36AC0B261
:10282000002B00F09580216B9847636B1A681D465A
:1028300022F480721A609A6822F001029A609A6902
:1028400042F008029A61DA69D6072DD4DA69900756
:1028500001D502221A62DA69510701D504221A62EF
:10286000DA69120701D508221A62DA69170612D549
:10287000D4F8BC20212A0ED0D4E909128A4273D0A0
:10288000A169895C0132C9B299622169B2FBF1F098
:1028900001FB1022A262DA69560608D403B0F0BD2B
:1028A000DA691D46D607D1D501221A62CEE7DA6968
:1028B00040F60F0C1E6804F1340012EA0C0F996800
:1028C00036D0B24F0F4040F0BB80DFF8CCC216EAE2
:1028D0000C0F40F06381D4F8A050012D4CD0D502EC
:1028E00002D54F0200F16781150606D501F40001FB
:1028F00006F080050D4340F043815106CED57206A7
:10290000CCD553E8002F22F0400243E8002141B12A
:10291000626B52E8003F23F0400342E80031002997
:10292000F7D120220023C4F8BC20C4F8AC30B5E7AE
:102930009506D0D506F0200501F080573D43CAD05A
:10294000D4F8A830002BA9D003B0BDE8F040184758
:10295000E3696269D054E369E2680133B3FBF2F1E1
:1029600002FB1133E36160E70022A4F88A201A68B1
:1029700022F080021A608EE7D706B0D5F506AED5F4
:102980001022B4F890501A629A68570640F11D81DF
:10299000D4F8B40001684A6892B2002A00F050816D
:1029A000AA4280F04D81C169A4F89220B1F5807FE0
:1029B00040D053E8002F22F4807243E8002141B157
:1029C000626B52E8001F21F4807142E80015002D6F
:1029D000F7D103F1080252E8002F22F0010203F1BF
:1029E000080545E800210029F3D103F1080252E867
:1029F000002F22F0400203F1080545E800210029DC
:102A0000F3D12022C4F8C020C4F8A01053E8002F4E
:102A100022F0100243E80026002EF7D15C490D6831
:102A200040B190F83530022B00F01381802380F8FC
:102A3000346043650223C4F8A430B4F892302DE723
:102A400012F0010F0CD016F4807F09D04FF0010C6A
:102A5000C3F820C0D4F8C4C04CF0010CC4F8C4C002
:102A600012F0020F7BD112F0040F0CD011F0010F05
:102A700009D04FF0040CC3F820C0D4F8C4C04CF007
:102A8000020CC4F8C4C012F0080F0CD006F0200CE1
:102A90005CEA070C07D008271F62D4F8C47047F01F
:102AA0000807C4F8C47017050AD5770108D54FF494
:102AB00000671F62D4F8C43043F02003C4F8C43068
:102AC000D4F8C430002B3FF4E9AE92060CD506F0E2
:102AD000200601F080510E4306D0D4F8A8301BB177
:102AE00001909847656B0198D4F8C420AB6802F058
:102AF000280203F04003134361D0FFF751FEAB6897
:102B00005B067FF5CBAE05F1080353E8003F23F0E9
:102B1000400305F1080141E8003262B1626B02F145
:102B2000080353E8003F23F0400302F1080040E8A7
:102B300000310029F3D1D4F8B40000283FF4AEAE40
:102B400090F83520134B022A03653BD1FDF78EFA2E
:102B500000283FF4A3AED4F8B400036DF4E611F0FE
:102B6000010F90D04FF0020C12F0040FC3F820C0F8
:102B7000D4F8C4C04CF0040CC4F8C4C083D078E7C7
:102B8000D4F8AC30002B7FF4DFAE87E601000010F4
:102B9000002E00247D0F04082001000412F0010F14
:102BA0003FF471AF16F4807F7FF450AF12F0020F44
:102BB0007FF469AF57E74FF480121A626EE6C4F8EB
:102BC000C4306BE680224265BEE6B4F89220B4F8C9
:102BD000921092B289B2AA423FF460AE00293FF44B
:102BE0005DAE53E8002F22F4907243E8002141B11A
:102BF000626B52E8001F21F4907142E80010002837
:102C0000F7D1954803F1080252E8002F024003F182
:102C1000080545E800210029F4D12022C4F8A810B5
:102C2000C4F8C020C4F8A01053E8002F22F010020E
:102C300043E800210029F7D10223C4F8A4302DE68F
:102C4000AA427FF42BAEC369B3F5807F7FF426AE32
:102C5000F2E70368814A824E824FB34218BF934223
:102C600006F118060CBF01220022B34208BF42F051
:102C700001021836B34208BF42F001021836B342CF
:102C800008BF42F001021836B34208BF42F0010209
:102C900006F55676B34208BF42F001021836B34239
:102CA00008BF42F001021836B34208BF42F00102E9
:102CB0001836B34208BF42F001021836B34208BFCB
:102CC00042F001021836B34208BF42F00102183642
:102CD000B34208BF42F00102A6F59266BB4218BF9C
:102CE000B34207F592670CBF01260026BB4208BF1E
:102CF00042F0010256EA020779D0D3F800C02CF066
:102D00001E0CC3F800C0D3F814C02CF0800CC3F81C
:102D100014C0D0F860C076BBD0F860C0DCF80060AA
:102D200026F48076CCF800601A6822F001021A605E
:102D300003E00A68521B052A24D81A68D607F8D47B
:102D4000D0E9165101F01F012FB33F238B40AB6038
:102D5000C36ED0E91921516033B11A68016F22F4B2
:102D600080721A60436F4B600122002380F8352087
:102D700080F834305EE6DCF8002022F48072CCF873
:102D80000020D1E7202103220023416580F8343060
:102D900080F835204EE6344A344EB34218BF934291
:102DA00006F114060CBF01220022B34208BF42F014
:102DB00001021436B34208BF42F001021436B34296
:102DC00008BF42F001021436B34208BF42F00102CC
:102DD000012606FA01F1696025498B4208BF42F0DD
:102DE0000102002AB4D1234A9342B1D0BCE71E4E5F
:102DF000DFF878C0634518BFB3420CF1140C0CBF68
:102E000001260026634508BF46F001060CF1140CAC
:102E1000634508BF46F001060CF1140C634508BF7A
:102E200046F001060CF1140C634508BF46F001069C
:102E3000D3F800C02CF00E0CC3F800C0DFF830C08F
:102E4000634508BF46F00106002E7FF465AF094ECA
:102E5000B3423FF461AF67E7FEFFFFEF400002407F
:102E60005800024028000240085402581C540258DE
:102E700080540258945402584B4B10B41B684B4C6E
:102E8000A4FB03435B0A03FB02F25AB18446531EC0
:102E90004748DCF83420013B024201D0920406D5B9
:102EA0005C1CF6D14FF000405DF8044B7047DCF835
:102EB00034305C0741D4DCF83430D80709D43D4BBA
:102EC000CCF83830DCF81030DBB2994205D0012064
:102ED000EAE70123CCF83830F9E7DCF8143036485B
:102EE00018400028E0D0002B2CDB5A002DD49C0089
:102EF0002DD4D9002DD41A012ED45C012FD4D901A0
:102F000030D41A0231D45C0232D499023CD4DA02B1
:102F100037D45C0332D499032DD4DA0340D41C0493
:102F20003BD4590436D49A0431D413F0080F0CBFA3
:102F30004FF480304FF40000B6E704231846CCF875
:102F40003830B1E74FF00070AEE74020ACE78020AA
:102F5000AAE74FF48070A7E74FF40070A4E74FF49E
:102F60008060A1E74FF400609EE74FF480509BE73C
:102F70004FF4005098E74FF4802095E74FF400306D
:102F800092E74FF400408FE74FF480408CE74FF416
:102F9000800089E74FF4001086E74FF4801083E744
:102FA0004FF4002080E700BF00000024D34D6210E2
:102FB00045002000C500200008E0FFFD82B000238E
:102FC000019302E00369002B09DB019B01330193AC
:102FD000019BB3F1706FF5D9032002B070478901EE
:102FE000002341F020010193016103E0036913F024
:102FF000200307D0019B01330193019BB3F1706F54
:10300000F4D9E9E7184602B0704700BF82B0002348
:10301000019302E00369002B09DB019B013301935B
:10302000019BB3F1706FF5D9032002B07047002205
:1030300010230192036103E0036913F0100307D02A
:10304000019B01330193019BB3F1706FF4D9EBE75E
:10305000184602B0704700BF82B00023019302E01F
:103060000369002B09DB019B01330193019BB3F141
:10307000706FF5D9032002B07047002301930369F4
:1030800043F00103036103E0036913F0010307D078
:10309000019B01330193019BB3F1706FF4D9E9E710
:1030A0001846E8E72DE9F843056807460C46C5F3DE
:1030B0001009B9F1000F39D18A4B4FF6FF72B3F8FE
:1030C0008030934256D0002B54D0874A02EA4328DE
:1030D00008F10068454534BF4FF001084FF0020881
:1030E000824B9D4206D903F500339D4200F2CF800A
:1030F0004FF001097E4E96F80833012B12D00123C0
:10310000B8F1010F86F808334FF00003C6F80C330E
:1031100036D0022074F010FE002800F099800023C1
:1031200086F808334FF0FF30BDE8F883704E96F80C
:103130000833012B4CD0012386F8083305F178437E
:10314000B3F5801F48D3A5F10163B3F5801F3FD2CB
:1031500000230220C6F80C3374F0EEFD002870D175
:10316000644A4FF00208D2F80C3143EA0803C2F86F
:103170000C313FE0B5F1016F67D3052011F0DCFEA3
:10318000404674F0D9FD0028C9D14046DFF864817B
:10319000D8F80C3023F4E663C8F80C30D8F80C30BB
:1031A00043EA092343F0A403C8F80C3074F0C4FDCB
:1031B000D8F80C20504B1340C8F80C300028AED182
:1031C00005F178430122B3F5801F86F8082303D365
:1031D0006FF00100BDE8F88300230120C6F80C332E
:1031E00074F0AAFD68BB434A4FF00108D36843F06E
:1031F0000203D360BFF36F8FBFF34F8F04F1200240
:1032000054F8043B944245F8043BF9D1BFF36F8F67
:10321000BFF34F8F404674F08FFDB8F1010F354A70
:1032200030D0D2F80C3123F00203C2F80C31002365
:1032300086F808330028CBD13B6820333B60BDE8DB
:10324000F883002386F80833C2E74FF0010847E708
:10325000DFF8A0800220D8F80C3123F4E663C8F828
:103260000C31D8F80C3143EA092343F0A403C8F821
:103270000C3174F061FDD8F80C211F4B1340C8F8D5
:103280000C319BE7D36823F00203D360CFE703F54B
:1032900000339D4211D903F500339D4210D903F547
:1032A00000339D4206D903F500339D420BD84FF001
:1032B00005091FE74FF004091CE74FF0020919E761
:1032C0004FF0030916E703F500339D4206D9B5F127
:1032D000016FBFF452AF4FF007090BE74FF006093B
:1032E00008E700BF00E8F11F00FE1F00FFFF010814
:1032F000002E002400200052FBF8FFFF0148FDF7DC
:10330000B1B800BF14310024084810B4D0F8143309
:10331000D0F8484399691A682CB1234600F54570E6
:103320005DF8044B18475DF8044B7047002E0024ED
:103330000148FDF797B800BF6C310024084810B46D
:10334000D0F86C33D0F8A04399691A682CB12346A1
:1033500000F55B705DF8044B18475DF8044B70474F
:10336000002E00240148FDF77DB800BFC4310024C1
:10337000084810B4D0F8C433D0F8F84399691A68F3
:103380002CB1234600F571705DF8044B18475DF8C9
:10339000044B7047002E00242DE9F04FDFF85C93BA
:1033A00000EB400583B0430009EB85050093D5F899
:1033B00084300193002B00F05E818046B5F88A00CE
:1033C00074F0B8F895F888000FF0E6F9044695F81F
:1033D00089000FF0E1F908F101030746DBB2002C88
:1033E00000F06E8140F60C12A1882372E280226800
:1033F000002800F05981037240F60C23C3809161CC
:103400003B68BA889A611121204609260FF080F99D
:10341000112138460FF07CF96525002C00F02E8133
:103420002268A38811690B4200F028811B04936174
:1034300011F0A4F805468B4611F0A0F8401B61EB93
:103440000B01052871F10001F6D314B12368A2889D
:103450009A6111F093F805468B4611F08FF8401BE6
:1034600061EB0B01052871F10001F6D3013ED3D1C8
:103470001CB1A38822681B04936111F07FF80546F4
:103480000E4611F07BF8401B61EB0601052871F137
:103490000001F6D31FB1BB883A681B04936111F099
:1034A0006DF805460E4611F069F8401B61EB060108
:1034B000052871F10001F6D314B12368A2889A613E
:1034C00011F05CF805460E4611F058F8401B61EB10
:1034D0000601052871F10001F6D317B13B68BA88DF
:1034E0009A61009B20463E21434409EB830393F8F5
:1034F0008F4022460FF02EF9224638463E210FF02B
:1035000029F9784C5823019A03FB0843C3F8142384
:10351000754B9A4200F0C380FEF7E4FB734BDA6907
:10352000C2F30212724B134493F8303003F01F03BE
:10353000D840009B434409EB830393F88C30022B63
:1035400000F0B980032B00F0B180012B14BF4FF4C1
:10355000C8714FF4487174F03DF8034658220021B9
:1035600002FB0842C2F81C13C2F81833C2E9C911A1
:10357000C2E9CC110121C2F8201392F8551301F0D1
:10358000FF00002900F0A480582123F07062242657
:103590004FF4004701FB08415648D1F8143381F835
:1035A00055631D6825F001051D601A619A6822F4B3
:1035B00000429A609F605A6822F400625A605A681A
:1035C0001043D1F82C2358601202D86820F4004030
:1035D000D860DA6000221A60186840F001001860B4
:1035E0002020C1F8582381F85503C1F8442381F8FD
:1035F000562391F855032028C5B217D191F85403EA
:10360000012813D081F85563186820F00100186074
:10361000186820F48050186018681860186840F026
:103620000100186081F8555381F85423009B022152
:103630000126314F434409EB830999F88E502846FF
:1036400074F0CEFB05F01F036A0999F88D5006FA55
:1036500003F30221284647F8223074F0C1FB5823B7
:1036600003FB084405F01F036D0906FA03F347F84E
:10367000253084F8106303B0BDE8F08F013D2AD0F7
:1036800010F07CFF83468A4610F078FFB0EB0B0009
:1036900061EB0A01052871F10001F5D3BDE6FEF7E3
:1036A00021FB124B1A6A3BE79161ACE6C82173F02B
:1036B00091FF034652E7642173F08CFF03464DE708
:1036C00000283FF4A0AE037240F60C23C38097E6B7
:1036D00082F8540358E7002C3FF4AAAEA38822686E
:1036E000A4E600BF002E0024001C0058004402582D
:1036F00058740C080080000200E100E00000002483
:103700002DE9F04F441C85B017469DF83C202DD084
:103710005824DFF8A8831E46054600FB04F408EB96
:10372000040393F81093B9F1000F1FD044444900EB
:10373000FF2F04F54574039100D0EEB9002A40F044
:10374000C680582303FB058393F85523202A04D110
:10375000B6B94FF40072C3F85823B8F818342846A5
:1037600001339BB2A8F81834FFF716FE4FF000099A
:10377000484605B0BDE8F08F93F85533202BECD1C7
:103780004FF0580A0AFB058A9AF85433012BE4D00B
:103790000122D8F800B019234FF400418AF85423CD
:1037A0002046CDF800B0FEF739FA0028D5D10E9B9F
:1037B000DAF81413CAF838332123BA4A8AF8553391
:1037C0004023CAF848038AF85633CAF858032046FB
:1037D000AAF83E634B681340039A1343B24A1A4354
:1037E0004A60594674F07AFA0246002840F0FB809D
:1037F000DAF81433802120469F620A23CDF800B006
:10380000FEF70CFA002840F0EE80BAF83E339BB287
:10381000FF2B40F21681DAF81413FF23A348AAF80D
:103820003C334B68A24A0340039803431A434A605F
:103830005826DDF80CA05F46039506FB058605E0DB
:10384000B6F83E339BB2002B00F01081394620467B
:1038500074F044FA002840F0F280D6F83813D6F815
:10386000145311F8012BB6F83C33AA62C6F838138A
:10387000013BB6F83E139BB20139A6F83C3389B23E
:10388000A6F83E13B6F83E1389B2002BD8D1002912
:10389000D6D002460A23802120460097FEF7BEF9C3
:1038A000FF22002840F0CB80B6F83E339BB2934213
:1038B00040F2A080D6F81413A6F83C234B687B4A4C
:1038C00013407B4A43EA0A031A434A60B8E74FF0C1
:1038D000580A0AFB058A9AF85533202B7FF43DAF2E
:1038E0009AF85433012B3FF438AF0122D8F8007016
:1038F00019234FF400418AF8542320460097FEF71D
:103900008DF900287FF429AF0E9BCAF84803CAF846
:10391000383321238AF8553310238AF85633CAF8EE
:103920005803AAF83E63BAF83E339BB2FF2B00F26D
:10393000C780BAF83E339BB2AAF83C33002B40F064
:10394000F180DAF8141357484B685A4A0340039839
:1039500003431A434A605826AA4606FB0586B6F872
:103960003E3339469BB2002B00F0D480204674F0E1
:10397000B5F9002878D1D6F83813D6F8145311F8D1
:10398000012BB6F83C33AA62C6F83813013BB6F8EF
:103990003E139BB20139A6F83C3389B2A6F83E1318
:1039A000B6F83E1389B2002BD9D10029D7D00246F0
:1039B0000A23802120460097FEF730F9FF220028D5
:1039C00052D1B6F83E339BB2934225D9D6F81413A0
:1039D000A6F83C234B68354A1340039A1343344AF4
:1039E0001A434A60BBE75823002203FB058383F890
:1039F0005423B2E6B6F83E33D6F814239BB22B48D4
:103A00005168A6F83C33DBB201404AEA03430B435A
:103A100043F00073536013E7B6F83E33D6F814133F
:103A20009BB2039A2148A6F83C33DBB242EA034337
:103A30004A680240134343F000734B608FE7039DD5
:103A40008BE6BAF83E33DAF814139BB2039A1748A0
:103A5000AAF83C33DBB242EA03434A68024013430C
:103A600043F000734B60E3E6554676E63946204660
:103A7000039D74F005F900287FF46FAED6F8143377
:103A800020210D4CD9615A6822405A6058230022E7
:103A900086F8551303FB058386F8560383F85423F1
:103AA00066E600BF009800FC00200101009C00FCBD
:103AB0000000FF010020000200E800FE002E0024AC
:103AC000FF234FF47F00FE224FF08076AAF83C33AC
:103AD000039BDDF838E01E4358231EF801AB03FBBF
:103AE0000583DFF850C0D3F81413C1F828A0A3F859
:103AF0003C23B3F83E23C3F838E3013A92B2A3F86B
:103B00003E234B6803EA0C033343034343F400535F
:103B10004B6020E72046554674F0B2F800287FF449
:103B20001CAEABE7013B4FF000769AB2501CC0B21E
:103B30000004CDE7009800FC2DE9F04F441C85B04F
:103B400099469DF83C3000F096805825C64C0646B4
:103B500000FB05F504EB050B9BF810A3BAF1000F71
:103B600000F089802544FF2A90464FEA410705F579
:103B7000457540F08680002B00F083809BF855331C
:103B8000202B6FD19BF85433012B6BD00122D4F83A
:103B9000008019234FF400418BF854232846CDF8B8
:103BA0000080FEF73BF800285CD10E9BCBF8480361
:103BB000CBF8383322238BF8553310238BF8563348
:103BC000CBF85803ABF83E93BBF83E339BB2FF2BC8
:103BD00000F21781BBF83E33DBF814139BB2A34805
:103BE0004A68ABF83C33DBB2024047EA0343134375
:103BF0009F4A1A434A604FF0580909FB0649B9F831
:103C00003E339BB2002B00F08A81D9F814339A69B5
:103C1000520700F1378142460A212846FDF77CFF12
:103C2000002840F0FB80D9F814339A69910640F1DE
:103C300000819A699A6912F0100200F0F88010224F
:103C400020218C4DDA610422C9F85823D9615A68C1
:103C50002A405A6089F8551389F8540389F85603A5
:103C600022689B69B4F81834304601339BB2A4F83B
:103C70001834FFF791FB4FF0000A504605B0BDE83D
:103C8000F08F4FF0580B0BFB064B9BF85533202B56
:103C9000E8D10E9B002B00F0AC80B9F1000F00F0D2
:103CA000A8809BF85433012BDCD0236801224FF409
:103CB000004128468BF85423039300931923FDF702
:103CC000ADFF0028CED12223DBF814130E9A8BF817
:103CD00055334023CBF838238BF85633CBF85803B1
:103CE000ABF83E93DFF884914A68CBF84803284646
:103CF00002EA09023A4342F490324A60039973F0AF
:103D0000EDFF0246002840F0368140232846194640
:103D1000DBF81433C3F82880039B00930A23FDF7D4
:103D20007DFF002840F02781BBF83E339BB2FF2B7C
:103D300040F22881DBF81413FF234F4AABF83C33E1
:103D40004B6803EA09033B431A434A604FF05808A3
:103D5000B946039F08FB064805E0B8F83E339BB21E
:103D6000002B00F021810A2300220421284600971D
:103D7000FDF754FF00287FF475AFD8F81433596A63
:103D8000D8F838331970B8F83E13D8F838330139F9
:103D9000013389B2C8F83833B8F83C33A8F83E1379
:103DA000013BB8F83E139BB289B2A8F83C33002916
:103DB000D3D0002BD1D102460A2380212846009778
:103DC000FDF72CFFFF2200287FF44CAFB8F83E33FC
:103DD0009BB2934240F2BD80D8F81413A8F83C235C
:103DE0004B68264A1340264A43EA09031A434A60AD
:103DF000B3E758234FF4007203FB0643C3F858237C
:103E000030E7DBF81413FF231848ABF83C334B685A
:103E1000194A03403B431A434A60ECE6582303FB2C
:103E20000643D3F814339A6922689B691AE7C9F8E4
:103E300058232268A2EB08020A2A7FF6E8AE9A69A4
:103E400012F004027FF4E3AE582101FB0641D1F8E1
:103E5000580381F85423202240F02000C1F8580371
:103E600081F855239B69FDE6002E0024009800FC94
:103E70000024000200E800FE0024FF01009C00FC7A
:103E80000000FF015A6AD9F838331A70B9F83E3386
:103E9000D9F83823013B01329BB2C9F83823A9F87D
:103EA0003E33B9F83C33B9F83E23013B92B29BB2A2
:103EB000A9F83C33002A3FF4A2AE002B7FF49FAE5A
:103EC0000A23002280212846CDF80080FDF7A6FEB7
:103ED00000287FF4C7AEB9F83E339BB2FF2B0CD954
:103EE000D9F81413FF233B48A9F83C334B683A4AEE
:103EF00003403B431A434A6081E6B9F83E33D9F8A0
:103F000014139BB233484A68A9F83C33DBB2024031
:103F100047EA0343134343F000734B606FE64146A7
:103F2000284673F0ADFE00287FF49CAED9F8143318
:103F300020212A4DD9615A682A405A6089F85513C0
:103F400089F856035822002302FB064484F85433B0
:103F500093E6B8F83E33D8F814239BB21D48516855
:103F6000A8F83C33DBB2014049EA03430B4343F07A
:103F700000735360F1E65823002203FB064383F8E5
:103F800054236FE6BBF83E33DBF814139BB24A6848
:103F9000ABF83C33DBB202EA090247EA03431343BE
:103FA0000F4A1A434A60D1E60399284673F068FE27
:103FB000034600287FF456AED8F814232020074D7E
:103FC000D06151682940516088F8550388F856330C
:103FD000B8E700BF009C00FC0000FF0100E800FE05
:103FE000002400020348D0F8B4300BB1A8301847C1
:103FF000704700BF000000240348D0F8D4300BB154
:10400000C8301847704700BF000000240348D0F8AC
:10401000F4300BB1E8301847704700BF00000024AF
:104020000348D0F8143113B100F584701847704775
:10403000000000240348D0F8343113B100F5947027
:1040400018477047000000240348D0F8543113B1DA
:1040500000F5A47018477047000000240348D0F80A
:10406000743113B100F5B470184770470000002494
:104070000348D0F8943113B100F5C4701847704765
:10408000000000240348D0F8B43113B100F5D47017
:1040900018477047000000240348D0F8D43113B10A
:1040A00000F5E47018477047000000240348D0F87A
:1040B000F43113B100F5F470184770470000002484
:1040C0000348D0F8143213B100F502701847704756
:1040D000000000240348D0F8343213B100F50A7010
:1040E00018477047000000240348D0F8543213B139
:1040F00000F5127018477047000000240348D0F8FC
:10410000743213B100F51A7018477047000000248C
:104110000348D0F8943213B100F522701847704765
:104120000000002410B41C46436884466FF30F035C
:1041300023434360036843F001030360036843F4CF
:1041400000730360002C3AD040F2E930DCF8143000
:104150009B0748D5002A49D012F8013B40F2E930CC
:104160008CF82030DCF81430DB0720D40138F9D18A
:10417000214B9C450CD0A3F578439C4538D003F5E2
:1041800080639C4536D003F578439C450BD10320D2
:104190001A4A00EB400002EBC002B2F8BC32013315
:1041A0009BB2A2F8BC3200205DF8044B70479CF82B
:1041B0003000C0B209B101F8010B013CC4D1DCF8F8
:1041C00014301B07FBD5DCF8183001205DF8044BD8
:1041D00043F01003CCF81830DCF8003023F0010372
:1041E000CCF8003070470138B0D1C1E7FF23B5E704
:1041F0000120CDE70220CBE7003001400000002481
:104200002DE9F84300242C4E8046036856F83450BC
:10421000AB4209D001340E2CF8D1284A00210520E8
:1042200009F0A6F8002019E0254B03EB8409D9F822
:104230001C74AFB198F8051000204B1C01EB410233
:1042400003EB430307EBC202DB00C2F80C80C2E9B8
:104250000400F854182303FB01700830BDE8F8830C
:104260000721682009F00AF90146C9F81C04F0B1D9
:104270003946682281F08EFFD9F81C1406EBC4047D
:104280003B4689600C6009628963096556F83320F2
:10429000954205D001330E2BF8D14F600F46C9E788
:1042A000084F4C2202FB03774F600F46C2E7064AD5
:1042B000052009F05DF8B5E7B0740C08941C0D08F2
:1042C000002E002454320024BC1C0D0830B40C4CC9
:1042D0000022234603E0013214330E2A0CD093F857
:1042E00004C08445F7D1DD68294201D10029F2D10B
:1042F000142303FB024000E0002030BC704700BFE5
:1043000008030024F0B54468A37913F002025FD0DB
:1043100002224FF0080C036864795B689B482044D4
:1043200093F83C40012C90F8C80050D0012483F849
:104330003C40142848D8DFE810F01500470047003B
:10434000470084004700470047003B014700470003
:104350004700BB00470047004700F2004700470006
:1043600047004D0018688A4C056A8A4E25F0020500
:10437000B04242EA0502056A25F001050562476878
:10438000856904EA050444F0600407D0824DA84220
:1043900004D005F57055A84240F04D8122F0080286
:1043A00047F440774CEA020222F00402476084613D
:1043B00041630262826942F008028261826922F0EE
:1043C0000402826182698261002283F83C20F0BD90
:1043D0009446A0E718686F4E046AB04224F40014B3
:1043E00044EA0252046A24F4801404626B4C456867
:1043F000476D04EA070444F4C0440ED006F5806615
:10440000B0420AD0664F06F58046B04218BFB842A7
:1044100003D006F58066B04201D145F480254560A1
:104420004465C1650262426D42F400624265426DBC
:1044300022F480624265426D4265002283F83C208E
:10444000C5E71868574C056A524E25F02005B04262
:1044500045EA0215026A22F0100202624768826988
:1044600004EA020444F4C04400F0DE804A4A904268
:1044700000F0DA804A4E4C4A904218BFB04203D056
:1044800002F58062904201D147F440674760846141
:1044900081630562826942F400628261826922F46A
:1044A0008062826182698261002283F83C208EE70B
:1044B0001868384E046AB04224F4005444EA0232C8
:1044C000046A24F480540462364C4568C76904EADF
:1044D000070444F4C0440ED006F58066B0420AD00A
:1044E0002F4F06F58046B04218BFB84203D006F5FC
:1044F0008066B04201D145F480454560C4610164E5
:104500000262C26942F40062C261C26922F480623E
:10451000C261C269C261002283F83C2057E7186873
:104520001C4E046AB04224F4003444EA0242046A95
:1045300024F4803404621D4C4568476D04EA070486
:1045400044F060040ED006F58066B0420AD0144FE5
:1045500006F58046B04218BFB84203D006F5806623
:10456000B04201D145F48035456044658165026201
:10457000426D42F008024265426D22F0040242653B
:10458000426D4265002283F83C2020E758740C08F5
:104590008CFFFEFF0000014000040140FF8FFFFE82
:1045A00000400140FF8CFFFE004401408FFFFEFFF2
:1045B0001868264C056A264E25F4007EB0424EEA65
:1045C0000225026A22F4807202624768C26904EA24
:1045D000020444F0600420D01E4A90421DD01E4EBA
:1045E0001E4A904218BFB04203D002F5806290424A
:1045F00001D147F440574760C461C1630562C26995
:1046000042F00802C261C26922F00402C261C269BA
:10461000C261002283F83C20D9E625F4006E4EEA00
:104620000C2E2EF48065E4E725F0800545EA0C1594
:1046300025F0400528E705F58065A8423FF4AEAEB9
:1046400005F58065A8427FF4B1AEA7E68CFFFEFFBA
:1046500000000140000401400040014000440140CE
:1046600042685379032B0FD8DFE803F00B080502EB
:1046700010684030704710683C3070471068383020
:10468000704710683430704700207047D0E900024E
:10469000064B517992790B44406893F8C810530740
:1046A00001D577F0A1B877F01BB900BF58740C089A
:1046B000F0B54468374A2469C368C4F303245B68CF
:1046C00052F82460EFF31184102585F312884568B1
:1046D000314F95F805E0D0F80CC002EB4E02D5F84A
:1046E00000E0158CDEF80C2005F4F05522EA0502F6
:1046F000CEF80C2017F806E0DCF8102053F80E5026
:104700001F2A25F0010543F80E5039D9203A2025FB
:10471000DCF804C005FA02F2CCF80C20E2B282F315
:104720001188BA5DDFF874C003EB020E4668456974
:10473000DEF8044004EA0C0C4CEA0101CEF8041047
:104740007179032924D8DFE801F0181512023168C5
:104750004031CEF80C500124CEF80810995841F0A1
:10476000100199509958214399500474F0BD316853
:104770003C31EEE731683831EBE731683431E8E756
:104780002025DCF804C005FA02F2CCF80820C5E7C1
:104790000021DEE758740C08C8750C080000FFFF04
:1047A00003681A7E012A2ED0002293F830100129C6
:1047B00009D093F8481001290ED093F86010012910
:1047C0001BD02ABB7047022142F4806283F830106C
:1047D00093F84810012904D1022142F4006283F8C1
:1047E000481093F86010012907D01B6800211B684E
:1047F0005962D9680A43DA607047022142F4805254
:1048000083F86010F1E702214FF400721976CCE7CB
:104810004FF40072E9E700BF08B5204B98420ED074
:1048200003F5806398420AD01D4A03F580439842FD
:1048300018BF904203D003F5806398421BD1FDF767
:1048400051FA1849184BCA69C969C2F30222C1F367
:1048500002211A4492F8302002F01F02D040114A7F
:104860001269C2F3C03241EAC202134493F8CC3059
:1048700003FB00F008BDFDF735FA0A490A4BCA6987
:10488000C969C2F3021CC1F3021103EB0C0292F8D6
:10489000302002F01F02D040E1E700BF00000140DD
:1048A000004001400044025858740C0870B50E4690
:1048B00005EE102AD0E90031013E1A680868B6B248
:1048C0005C681568FFF7A8FF07EE900AB8EE455A36
:1048D0009FED5D7AF8EE677A87EE850A30EE070A7B
:1048E0007CF0D2FB23680138AB4280B268D0C4E9C7
:1048F000005000238022E660A360A261C4E9043373
:1049000094F83D3003F0FF02002B78D00223211DE4
:10491000284684F83D30FDF7CDFE4C4A0123B5F121
:10492000804FA5EB020284F84830B2FA82F284F894
:104930003E3084F83F304FEA521284F8403084F819
:10494000413084F8423084F8433084F8443084F8AD
:10495000453084F8463084F8473084F83D3034D010
:104960009ABB3B4B9D420CD003F580639D4208D01F
:1049700003F580639D4245D003F578439D4241D0C5
:1049800070BD94F83C30012BFAD00222314B01214A
:1049900084F83D20A8680340AB6084F83D1084F89B
:1049A0003D206B68A96823F0700321F0800101228B
:1049B0006B600023A96084F83D2084F83C3070BD12
:1049C000636883423AD0606093E794F83C30012BEF
:1049D000D6D002211F4B002084F83D10A9680B405F
:1049E0000121AB6084F83D10022384F83D306B68F0
:1049F000A9680AB90028D6D023F47003D3E784F855
:104A00003C2083E794F83C30012BB9D00221114BB4
:104A1000114884F83D10A968281A0B40B0FA80F0BC
:104A20000121AB600023400984F83D1084F83C303C
:104A30000A4B9D42D8D00028D6D170BDE368B3425E
:104A40007FF457AF70BD00BF0AD7233C0000014080
:104A5000000400408800CEFF00040140000C00402C
:104A6000024B0348D3F81C14FCF7D4BC002E0024DE
:104A700000000140034B4FF08040D3F82014FCF7B6
:104A8000C9BC00BF002E0024024B0348D3F82414F5
:104A9000FCF7C0BC002E002400040040024B034879
:104AA000D3F82814FCF7B6BC002E00240008004000
:104AB000024B0348D3F82C14FCF7ACBC002E0024A6
:104AC000000C0040024B0348D3F83814FCF7A2BC9A
:104AD000002E002400040140024B0348D3F8481480
:104AE000FCF798BC002E002400180040024B03483D
:104AF000D3F85414FCF78EBC002E00240040014073
:104B0000024B0348D3F85814FCF784BC002E002451
:104B100000440140024B0348D3F85C14FCF77ABC14
:104B2000002E00240048014010B5064C0648D4F879
:104B30003814FCF76FFCD4F84C140448BDE810405E
:104B4000FCF768BC002E002400040140001C00405B
:104B500010B5064C0648D4F83814FCF75BFCD4F8C2
:104B600050140448BDE81040FCF754BC002E00244B
:104B70000004014000200040BFF34F8F0549064B61
:104B8000CA6802F4E0621343CB60BFF34F8F00BFEB
:104B9000FDE700BF00ED00E00400FA050021012060
:104BA00008B50EF0CFF872B6FFF7E6FF2DE9F04337
:104BB000BFB0BFF35F8F9C4C0023626A22F4803247
:104BC0006262C4F894309DF843109DF84450090681
:104BD0009DF842200F9841EA057141EAC2419DF8D3
:104BE000452041EA82419DF8462041EA42419DF834
:104BF000472041EA02419DF8412041EA02219DF807
:104C0000402041EA4201C4F898300133D4F8A02092
:104C1000112B22F00102C4F8A020C4F89C00C4F8B3
:104C2000A010F0D10523C4F89430636A43F48033B4
:104C30006362BFF34F8FBFF36F8F7C487C4A7D491F
:104C4000121A80F07FF9D4F888107B4B00220120E3
:104C500041F47001C4F8881018601A61196841F0B5
:104C600080011960196801431960196841F48031A5
:104C70001960196841F4805119609A61DA611A6209
:104C80009A62DA621A635A639A63DA631A645A643C
:104C9000196821F4802119601A664FF00063674992
:104CA000C1F80801A36078F033FC654AD36813F0BB
:104CB000040FD36840F0A380624B0021604A059145
:104CC000D96A21F00101D962DB6A03F0010305937F
:104CD000936943F440439361936903F4404305931C
:104CE000059B93699E04FCD54C2200210EA8564CCE
:104CF00081F050FA554A42F20303A4F11001126800
:104D0000B3EB124F4FF000024FF00C0308BF0C46FC
:104D10000892E268A370002A4CD1494A494B916934
:104D200041F440419161926902F440420892DA6A8A
:104D300042F00102DA62DB6A03F001030893089B88
:104D40003F4A93699D04FCD53B4B4FF440354048A6
:104D50000321D3F8E02042F08002C3F8E0200122D2
:104D6000D3F8E03003F080030793079B85610D9B28
:104D7000CDE90013002378F059F8022301204FF405
:104D80008031A288CDE917330C231993A379CDE99B
:104D90000E01E079217A1C900EA81D91CDE91A230D
:104DA00008220023CDE91E23FBF75CFD032838D041
:104DB000A0B1FEE7234BD96A21F00101D962DB6A79
:104DC0001F4903F0010308938B6923F44043134305
:104DD0008B618B6903F440430893B0E71D4B1A685D
:104DE00012F00E0F3AD11A6822F00F0242F00202BE
:104DF0001A601B6803F00F03022B2FD0FEE723F08D
:104E00000703154C43F00203D360216805E02368D3
:104E10005B1AB3F57A7F3FF64FAF53689F04F6D520
:104E20004AE7FFF7BBFE00BF00ED00E00000000016
:104E300058370000509B0D08004402580080005174
:104E40000048025800040058300400240010005CA0
:104E5000001C025800200052002E00246D4A936965
:104E600003F070033F2B05D8936923F0700343F0E0
:104E700040039361674AD36903F070033F2B05D861
:104E8000D36923F0700343F04003D361614AD369CF
:104E900003F4E063B3F5806F05D2D36923F4E063D4
:104EA00043F48063D3615B4A136A03F070033F2BC2
:104EB00005D8136A23F0700343F040031362554B87
:104EC0009A69140705D49A6922F00F0242F0080289
:104ED0009A61504A936923F470639361136898014F
:104EE0008CD5136941F288314B4C23F0070343F012
:104EF00003031361206804E023681B1A8B4200F24D
:104F0000AA81136903F03803182BF5D1936903F0D4
:104F10000F03082B05D9936923F00F0343F008030F
:104F200093613E4A136803F00F03022B0BD91368F9
:104F300023F00F0343F002031360136803F00F0321
:104F4000022B00D05AE7334A936903F07003402BD9
:104F500005D9936923F0700343F0400393612D4A10
:104F6000D36903F07003402B05D9D36923F0700394
:104F700043F04003D361274AD36903F4E063B3F5F8
:104F8000806F05D9D36923F4E06343F48063D36170
:104F9000204A136A03F07003402B00F254811D4E27
:104FA000FCF77EFE1E4DB269B369C2F303221D4BAE
:104FB000134493F8303003F01F0320FA03F3D5F8BD
:104FC00080002B60FCF7FAFC002840F0458110239C
:104FD000159017900EA80E93FBF744FC002840F0A4
:104FE00031813368104A43F080033360D6F8F430DF
:104FF00043F00203C6F8F430D6F8F43003F00203AD
:105000000493049B136A43F001031362074B216866
:1050100011E000BF00440258002E0024002000527E
:105020000000002458740C08000400588038010067
:10503000013B3FF4F6AE22689142F9D02268236822
:105040009B1A0A2BFBD900214FF48020A64C4FF469
:1050500040130026002730934FF00208CDE90E01DF
:105060000EA877F009F8D4F8EC30A04941F2030219
:1050700043F002030EA8C4F8EC30D4F8EC3003F08F
:1050800002030393039BD4F8943043F00203C4F863
:105090009430D4F8943023F00203C4F894300B68B1
:1050A0009349B2EB134F934B934A28BF0A465A6079
:1050B0001A6822F47C5242F400521A601A6842F0D4
:1050C00060021A6003220023CDE92C67CDE90E238C
:1050D00076F0D2FF4FF4E04200230EA8CDE9266718
:1050E00000270326CDE90E233A9776F0C5FF182254
:1050F00000230EA82F973497CDE90E2376F0BCFF3E
:105100004FF4803200230EA81797CDE90E23052215
:105110004FF4FA73CDE91023042314934FF4803332
:10512000CDE915772293CDE9128676F0A5FFD4F864
:10513000E03042464FF4807143F001036F48C4F8F9
:10514000E030D4F8E03003F001030993099B3B46BB
:10515000CDE9006777F06AFE23694246684823F08C
:10516000FE7343F088732361D4F8E03043F0040306
:10517000C4F8E030D4F8E03003F0040306933B4673
:1051800006994FF40071CDE9006777F04FFE23696F
:1051900023F07E4343F0FC432361FCF781FD28604C
:1051A000BFF35F8F574C3E46574D4FF00108636A7F
:1051B00023F480336362C4F8947028E0002A49D055
:1051C0002F686B7A103515F8061C1B0643EA01732D
:1051D00043EA420315F8052C43EA824315F8042CF0
:1051E00043EA424315F8032CC4F89860013643EAB9
:1051F0000243D4F8A020032E43F0010322F0010261
:10520000C4F8A020C4F89C70C4F8A03025D06B6806
:105210002A7A002BD2D02F68002AD2D127F01F0281
:10522000A3EB0209B9F1200F38BF4FF0200948461F
:105230007FF0FEFD421E08FA02F1894508BF0246D2
:10524000D2B2BEE7FEE7136A23F0700343F04003D7
:105250001362A4E6FEE7D1E5D0E50523C4F8943057
:10526000636A43F480336362BFF34F8FBFF36F8F82
:10527000BFF34F8FBFF36F8F0022C4F85022BFF3EC
:105280004F8FBFF36F8F636943F400336361BFF3E4
:105290004F8FBFF36F8FC4F88420BFF34F8FD4F8C4
:1052A000805043F6E0761749C5F34E34C5F3C9057F
:1052B000640104EA06002B4640EA8372013BC1F810
:1052C0006022F9D2203C14F1200FF2D1BFF34F8FAE
:1052D0004B6943F480334B61BFF34F8FBFF36F8F44
:1052E0003FB0BDE8F08300BF004402580010005CEE
:1052F0007FBB2200008400407FBB223000000258A8
:105300000008025800ED00E0400400243F4B586DB7
:10531000012830B585B06ED03D494FF6FF003D4ABB
:10532000CC683D4B04403D4D3D482243CA605A6F16
:10533000C5F87C28D3F8F42042F00202C3F8F42028
:10534000D3F8F42002F002020392039AD3F8DC208F
:1053500042F00052C3F8DC20D3F8DC2002F0005207
:105360000292029AD3F8DC2042F08042C3F8DC209B
:10537000D3F8DC2002F080420192019AD3F8DC20BD
:1053800042F00042C3F8DC20D3F8DC20036802F0CE
:10539000004224480092009AD1F8FC40224A44F08E
:1053A0008074C1F8FC40A2FB03420024920CC5F8B3
:1053B00080281E4AC0F8B02F1D4A4460A2FB032378
:1053C00002689B0942F00102013B0260B3F1807F59
:1053D00007D34FF0E022136943F00403136105B0D3
:1053E00030BD4FF0E022F0205361072381F8230005
:1053F00094611361EDE700210DF0A4FC0D4B1A68D8
:1054000082F308885B689847FEE700BF00400058B9
:1054100000ED00E00003FA0500440258002E0024CD
:1054200000000024001000E083DE1B4355CEACC515
:10543000D34D62100098F01F2DE9F843374E98467F
:1054400006EB8003D3F8DC40002C65D004F1D203D6
:10545000FC360546B4F8D202A36104F5E973666030
:105460001746E3614FF48073261DE160C4E90433FD
:105470002368C4F8CC30A36300284AD194F8D10043
:105480000DF08AF918F0080F94F8D09034D1BA07CB
:1054900023D4FB0711D4052194F8D60272F0A0FCA6
:1054A00094F8D63201221E4903F01F005B098240A6
:1054B00041F823203046BDE8F883013548460DF019
:1054C0006BF9EDB218B140F206630572C38094F82F
:1054D000D42202210DF03EF9DDE76B1CDBB218B1DE
:1054E000037240F20653C38094F8D52202210DF0D6
:1054F00031F9FB07CFD5E0E70135EDB218B140F245
:1055000006730572C38094F8D52202210DF022F9AA
:10551000C1E772F00FF8B1E72646CBE758740C08E4
:1055200000E100E00148FDF771B900BF74040024F8
:105530000148FDF76BB900BF4C0700240148FDF797
:1055400065B900BF240A00240148FDF75FB900BF18
:10555000FC0C00240148FDF759B900BFD40F00240A
:105560000148FDF753B900BFAC1200240148FDF714
:105570004DB900BF8415002470B52422456B00236B
:105580008168C0F8BC2004462A6800F1340622F085
:1055900001022A602B606B60AB608279C0F8C43076
:1055A00080F8B830C0F8BC30C364C0F8C030436580
:1055B000C0F8A030C0F8A4309302816303F4805394
:1055C0004179C363130303F400530364130203F428
:1055D00080634364C36D01F00200C90745D400280D
:1055E0007ED1A06412F0080254D0D4F8BC20002A66
:1055F00000F08A802422C4F8BC202A6822F001022C
:105600002A60002B7CD13046FCF7DEFC012812D04A
:105610006B68304623F490436B60AB6823F0220341
:10562000AB60AB6843F00803AB602B6843F0010349
:105630002B6076F079F86279D6070DD5D4F8C830AA
:10564000196841F480711960996841F0010199600D
:10565000196841F020011960950705D5D4F8C820D4
:10566000136843F08003136070BD0421A16470B31C
:105670000C21D007A164B5D54FF4803143F002036B
:10568000616643F001034FF40031E365216612F0D7
:105690000802AAD1D4F8BC1009B194F8B82084F853
:1056A000B8202422C4F8BC202A6822F001022A6013
:1056B00013BB3046FCF788FC0128BCD06B68304631
:1056C00023F490436B60AB6823F02A03ACE7D10767
:1056D00088D543F002034FF48031E365616681E7CA
:1056E0000821A164D1077FF57DAF43F001034FF49A
:1056F0000031E3652166CAE73046FBF7E7FBD8E7F0
:105700003046FBF7E3FB7EE784F8B82072E700BF82
:10571000816031E741712FE781712DE72DE9F84371
:10572000434D3C20434C05F59872B5F83631C4F82A
:105730008428A4F89038B5F83A21B5F83E31A4F899
:105740009228A4F888380DF027F8074642200DF07B
:1057500023F8064638200DF01FF881461FB10D23AF
:10576000FB8000233B721EB10D23F38000233372B4
:10577000B9F1000F05D00D23A9F80630002389F8F0
:105780000830B5F842313920A4F88A38B5F84631E6
:10579000A4F88C38B5F84A31A4F88E380CF0FCFF28
:1057A00080463A200CF0F8FF05463B200CF0F4FF51
:1057B0000446B8F1000F05D00D23A8F806300023E9
:1057C00088F808301DB10D23EB8000232B721CB12B
:1057D0000D23E3800023237248460CF08DFF012146
:1057E00048460CF095FF40460CF086FF28460CF02A
:1057F00083FF20460CF080FF404601210CF088FF1B
:10580000284601210CF084FF012120460CF080FF86
:1058100038460CF071FF30460CF06EFF384601211F
:105820000CF076FF30460121BDE8F8430CF070BF64
:1058300058740C08002E002438B5134D41F20D1396
:10584000124941F28832D5F8D808D5F894480004B6
:10585000A060E068014020460B430D21E360FDF7A6
:105860000BFB38B1D5F8C828034600201343C5F810
:10587000C83838BD606900F4F050A0F50060B0FA97
:1058800080F0400938BD00BF002E0024C0E0FEFFBC
:105890002DE9F04FA74D7C2200219BB005F6940026
:1058A00080F078FC4FF48031D5F8844895F8C438FE
:1058B0002268C5F898184FF40031C5F89428C5F847
:1058C000A4180221C5F8A818002B00F08880042233
:1058D000994B85F8C428DA6C1B68D6030DD51801DE
:1058E00000F1D98001224FF0006385F8C428C5F883
:1058F000C83801201BB0BDE8F08F9C01F2D50AAB7F
:1059000018460193FCF760FD0B990029EAD0D5F801
:1059100094480A0A894B6668A3FB0232884B894F78
:1059200033401009B94243EA12136360236843F01D
:105930000303236040F2F9804300834AB1FBF3F391
:10594000B2FBF3F2296802322B685B1A9A42FBD849
:1059500000237E4A0493A3607D4BE16817680B40E7
:1059600043F48053E3607B4BA3FB073741F288335A
:105970007F0A03FB07F73B46002B00F0CB80626BEE
:10598000013B1106F8D5744B714AA3634FF4D573EC
:10599000A360E3681A4041F208131343E3604FB178
:1059A0003B46626B12F0450F02D0920440F1DC805E
:1059B000013BF6D10023C5F8D038A360644BE26800
:1059C000134043F48053E3603B46002B00F0A28079
:1059D000626B013B1106F8D55F4BA363E3E05F4BBD
:1059E0009A425FD05E4B9A4200F00F8195F8900882
:1059F0000CF0D2FE834695F892080CF0CDFE82465C
:105A000095F888080CF0C8FE814695F88A080CF0D5
:105A1000C3FE804695F88C080CF0BEFE074695F84C
:105A20008E080CF0B9FE95F8912806460E215846CE
:105A30000CF090FE504695F893280E210CF08AFE4B
:105A4000484695F889280E210CF084FE404695F8CA
:105A50008B280E210CF07EFE95F88D2838460E21FD
:105A60000CF078FE0E2195F88F2830460CF072FE6F
:105A70000221B4F9040072F0B3F9B4F90430002B38
:105A8000FFF625AF03F01F0001225B093549824074
:105A900041F823201BE70AAB18460193FCF760F995
:105AA0000C9932E7244BD3F8D42022F48032C3F887
:105AB000D420D3F8D42042F48032C3F8D420D3F8D1
:105AC000D42002F480320392039ADA6F42F48032D7
:105AD000DA67DA6F22F48032DA6787E72A684FEAFA
:105AE000134EA2EB09027346824213D8002B40F0FA
:105AF0003181C4F808E0E36803EA0A030B43E3607A
:105B00003B46626B12F0450F02D0920440F1F080E8
:105B1000013BF6D14FF00040012385F8C438D5F899
:105B2000C8380343C5F8C838E3E6074AB2FBF1F2C8
:105B3000296808E7002E002400440258598B4F01C1
:105B4000002CC0FFFF340C001021010000000024D5
:105B5000C0E0FEFFD34D6210C5002000007000526F
:105B60000024024800E100E0636B5B0700F16F83F3
:105B7000636BDE0769D4636B580601D54023A363CA
:105B80000123704A37212046C5F8D0380023A3608E
:105B9000E3681A4041F23713134341F28832E3605D
:105BA000FDF76AF970BB049A4FF6FE739A4200F251
:105BB0003982DFF890A1DFF89881634E002241F22C
:105BC000371337212046A260E26802EA0A02134333
:105BD00041F28832E360FDF74FF900289CD1C4F808
:105BE000088041F22913E26802EA0A021343E360E3
:105BF00047B13B46626B12F0450F01D0920427D5A6
:105C0000013BF7D14FF0805086E7504BD3F8DC20B2
:105C100022F40072C3F8DC20D3F8DC2042F40072D6
:105C2000C3F8DC20D3F8DC2002F400720292029A5E
:105C3000D3F8842042F40072C3F88420D3F884207F
:105C400022F40072C3F88420D0E60123A36397E70F
:105C5000636B5B0758D4A6636269049B002A03F157
:105C600001030493049B03DB4FF6FE718B42A5D91D
:105C700004994FF6FE73994200F21782500040F1EA
:105C8000D4814FF00108D5F80090C5F8CC8823687E
:105C9000990700F0C4810023DFF8A8A02046A36084
:105CA00041F20233E26802EA0A021343E360FBF7BF
:105CB0006BF900287FF430AF636941F20311C5F836
:105CC0000039A369C5F80439E369C5F80839236ABE
:105CD000C5F80C39A060E36803EA0A030B43E360EC
:105CE000002F3FF417AFDFF860C041F2873007E7BD
:105CF000636B5B0722D4636BDE071CD42369DBB2C2
:105D0000032B06D0012007E704234FF08050A36344
:105D100002E7C4F838C0636913F4604F3FF4DEAEA5
:105D2000590400F19D8213F4004F0CBF4FF48030F2
:105D30004FF48050F0E60123A363E3E70423184601
:105D4000A363E9E6C0E0FEFFC5002000004402585E
:105D5000000010C14FEA0E49C5F8D8E8D44A2046E1
:105D6000C4F80890E3681A4041F209331343E36032
:105D7000FBF70AF900287FF4CFAE6269C5F8F02876
:105D8000A369C5F8F438E769C5F8F878216AC5F859
:105D9000FC18D4F818C04FEA1C5CC5F8D4C84FEA08
:105DA000927C8DF828C0C2F3836C8DF829C0C2F3B1
:105DB000016C8DF82AC0C2F3074C8DF82BC0C2F3DA
:105DC000072CD2B28DF82CC08DF82D201A0DADF80D
:105DD0002E20C3F303428DF83020C3F3C0328DF878
:105DE0003120C3F380328DF83220C3F340328DF876
:105DF0003320C3F300328DF834208DF83500B8F12C
:105E0000000F00F01F811B0403F47C1343EA1743C7
:105E10000E934FF40073C5F8E0380E9B01339B02DC
:105E2000C5F8DC38C5F8E438C7F380334FF4007A9E
:105E300020468DF84130C7F3C61307F07F07C5F839
:105E4000E8A88DF84230CB0F8DF8437001278DF80C
:105E50004430C1F341738DF84530C1F382638DF84E
:105E60004630C1F383538DF84730C1F340538DF86A
:105E7000483000238DF84930C1F300438DF84A3093
:105E8000C1F3C0338DF84B30C1F380338DF84C3003
:105E9000C1F340338DF84D30C1F300338DF84E30EF
:105EA000C1F381238DF84F30C1F30123C1F34601C3
:105EB0008DF8503041F207138DF8511007218DF8FD
:105EC0005270C4F80890DFF8E891E26802EA09022B
:105ED000134341F28832E360FCF7CEFF00287FF4E1
:105EE0001BAEC4F808A041F2101BE36841F28832EF
:105EF0001021204603EA090343EA0B03E360FCF7A1
:105F0000BBFF002840F0948095F8C438032B3FF481
:105F1000F0AC2F6863699A017ED44FF0400A41F2D9
:105F2000883210212046C4F808A0E36803EA090378
:105F300043EA0B03E360FCF79FFF002843D1D5F849
:105F4000D838372120461B04A36041F23713E2689A
:105F500002EA0902134341F28832E360FCF78CFF46
:105F600088BB4FF0FF330D216362C4F828A0E36AB9
:105F700023F0FF0343F06303E36241F20D13A060DB
:105F80002046E26802EA0902134341F28832E360E4
:105F9000FCF772FFB8B9019E04E02B68DB1B0133EC
:105FA00000F08A80636B13F4957F636B40F0878009
:105FB0001B04F2D506F12002D4F8803046F8043BE9
:105FC000B242F9D1E9E7D5F8C838C5F8C838394B35
:105FD0000122A363D5F8C83818434FF40073C5F8FD
:105FE000C808204685F8C428A36041F21013E16870
:105FF0002F4A0A401021134341F28832E360FCF734
:106000003BFF00283FF475AC2A4A0123A263C5F880
:10601000C80885F8C4386CE44FF40060D7E74FF047
:10602000806079E5049A9A423FD84FF000082AE64A
:10603000204BA363D5F8C8380343C5F8C83885F8A2
:10604000C47856E440F6FC7202EA830343EA97738D
:106050000E93C7F3C2638DF83C30C7F302638DF82B
:106060003D30C7F342538DF83E30C7F382438DF87D
:106070003F30C7F3C2338DF8403001230E9A9DF8AC
:1060800040001A4400F00700023082409DF83000C2
:1060900000F00F00C5F8DC288340C5F8E0385B0A43
:1060A00002FB03F3C5F8E438BEE64FF0807033E539
:1060B000C0E0FEFFFF0FE01F4FF0004087E718072A
:1060C00000F1C880636B990700F1C880636B9A0682
:1060D00008D5C1E0D4F880202B6846F8042BDB1BE0
:1060E0000133E9D0636BDB04F4D40A9B5E4AA263FC
:1060F000C3F381128DF81420C3F340128DF81520DC
:106100001A0A22F0FF0242EA1362DDE90B1392B28F
:1061100009BAADF81620DAB206918DF81C20C3F347
:1061200007229DF83B108DF81D20C3F303521B0C72
:106130008DF81E200D9A23F0FF03D0B203432046B2
:10614000ADF82030C2F385238DF82230C2F301234D
:106150008DF82330C2F3031302F00F028DF82430C0
:106160004FF400738DF825208DF826101021A360C0
:106170003E4AE3681A4041F21013134341F2883259
:10618000E360FCF779FE00287FF43EAF9DF82430F1
:10619000B8F1010F9DF82520DBB2D2B205D113432F
:1061A00014BF4FF400784FF48078D5F8A008C5F8F4
:1061B000EC8871F067FC00287FF49BAB2C6803E04F
:1061C0002B681B1B013330D071F03AFC0428F7D147
:1061D00000230121D5F8DC28C5F8C838C5F8C03837
:1061E00085F8C418002A3FF484AB4FF4804071F066
:1061F00049FC00287FF47DABD5F8CC38F3B1012BF6
:106200007FF477AB02201A4C85F81009A4F124031F
:106210000FCB84E80F00A4F1140310340FCB84E8F3
:106220000F0000201BB0BDE8F08F4FF000420123AB
:10623000C5F8C82885F8C438FFF75BBBD5F8D03857
:10624000002BE0D0012B7FF454AB1846DBE704238E
:10625000A36395E40820BAE62020B8E60220B6E65B
:106260004FF4005058E400BF3A0F0018C0E0FEFFA2
:1062700014370024C74BD3F81419D3F8182970B574
:106280008C0F93F81059100EC2F3072C83F8404975
:10629000C1F383640001012D83F84149C1F3016416
:1062A00083F84249C1F3074483F84349C1F3072403
:1062B000C9B283F84449C2F3035483F84519A3F8DB
:1062C0004609C2F3C030B3F8461989B241EA040165
:1062D000C2F30344A3F84619C2F3403183F8484996
:1062E000C2F3803483F849094FF0000083F84A492B
:1062F00083F84B19C2F3003183F84C19D3F81C19F9
:1063000083F84D0940F2EF80022D00F0C3802A206F
:106310004FEA4C0C83F85949C1F3C01201F07F01D8
:106320000CF07E0C83F85AC94FF0010C93F85A49CF
:106330001443D3F8202983F85A49D40F83F85B1902
:10634000910D83F85C49C2F3417401F00C01C2F372
:10635000815583F85D49C2F3826483F85E4983F80E
:106360005F1993F85F19D3F82449294383F85F191B
:10637000C2F3405183F86019002183F86119C2F318
:10638000004183F86219C2F3C03183F86319C2F384
:10639000803183F86419C2F3403183F86519C2F380
:1063A000003183F86619C2F3812183F86719C2F3BB
:1063B0000121C2F3460283F86819C4F3074183F848
:1063C0006929220E090283F86AC983F86C29C4F38B
:1063D0000722A3F86E192406B3F86E1989B2114387
:1063E000A3F86E19D3F82819C3F870490C0ED3F826
:1063F000702942EA0442C3F870290A0AD3F87049A6
:1064000002F47F422243C1F30724C9B2C3F87029C2
:10641000D3F87059D3F82C292C43C3F8704983F86A
:106420007419110E83F87519110C0906C3F878193F
:106430001102D3F878490A4601F47F01214392B250
:10644000D3F83049C3F87819D3F878190A43C3F858
:106450007829C4F30352D3F8781941EA1461C3F8D8
:10646000781993F87C191143C4F3072283F87C1937
:10647000210A01F47061A3F87E19B3F87E1989B27C
:106480001143C4F34602A3F87E1983F8802983F8E8
:1064900081C970BD1204C1F3072C0D0E02F47C12E9
:1064A000C3F85029C1F30742D3F8504944EA052400
:1064B000C3F85049D3F8504922434FF40074C3F84D
:1064C0005029D3F85029C3F89049013240F1000413
:1064D000A40244EA92549202C3F88C49C1F3803476
:1064E000C3F8882914E74FEA8C2CC1F3C2659400E5
:1064F0000CF44062C1F3072C04F47F74C3F85029F4
:10650000D3F850291443CA0BC3F8504902F00602CD
:10651000D3F8504944EA9174C3F85049C1F3026476
:1065200083F85459012583F85549C1F3425483F83F
:106530005649C1F3824483F85749C1F3C03483F804
:10654000582993F85829224383F85829D3F85049F9
:1065500093F8582993F84869023205FA02F2B540D7
:10656000D617A2FB052EC3F8905905FB06EE04FBD7
:106570000EEE0134A2FB0424A644520AC1F3803477
:1065800042EACE52C3F888294FEA5E22C3F88C292A
:10659000BEE600BF002E002471F0AEB871F0ACB8BA
:1065A00010B51C200CF0F8F8044611210CF0B0F8DE
:1065B00020460CF0A7F8C8200EF00EF82046BDE8E3
:1065C00010400CF099B800BF1C48D0F80038D0F843
:1065D000082830B59B184FF01A040C8001D11848D8
:1065E00030BD174A0024D0F8040802F11005114606
:1065F0004FEA137EB3F1204FCC7001F102010EF18E
:10660000370C38BF0EF1300C8D424FEA031381F87E
:1066100000C0EDD10B4D0024010FB0F1204FD47418
:1066200002F1020201F1370338BF01F13003954254
:106630004FEA00101374EFD1014830BD00E0F11FA4
:10664000581800246018002400207047212808B53D
:1066500024D0222816D0202812D189B1072A0FD1A0
:10666000154A164B0868B1F804C012688979D861D8
:10667000A3F820C083F8221012B1014600209047F1
:10668000002008BD0029FBD0022AF9D10A4B5B6823
:10669000002BF5D0098800209847F1E70029EFD0BA
:1066A000072AEDD1054BD8691A8C93F8223008607F
:1066B00000208A808B7108BDA03700245818002460
:1066C00000207047034B93F82C00003818BF0120BE
:1066D000704700BFA0370024034B93F82C00032819
:1066E00094BF002001207047A03700240048704765
:1066F000D0370024164B002030B493F82A4014B150
:10670000DD698D4205D0013010330828F5D130BC49
:106710007047104BB2B1996F01EB40218A4201D111
:10672000022C08D093F8182212B9012283F81822FB
:10673000012283F8612003EB0013012283F88A20F1
:1067400030BC704703EB001383F88A20DFE700BFFB
:1067500000380024A037002430B40023194C04F181
:10676000600084F8043103E001331030082B1BD0A3
:10677000C5698D42F8D190F82AC0BCF1030FF3D15E
:10678000A2B1A16F01EB43218A4208D094F81822EC
:1067900012B9012284F81822012284F8612004EB46
:1067A0000314012384F88A3030BC7047D4F80021E8
:1067B00004EB03130421013283F88A10C4F800218A
:1067C000F2E700BFA0370024C0B1836823B10F4BAC
:1067D000072283F8622070470C4A042192F8600077
:1067E00082F87430032882F86210C2E91B3314BFA8
:1067F0004FF480738023C2E919337047034B0122A1
:1068000083F8182283F86120704700BFA037002466
:10681000244910B5CC8C91F824C0644531D9634625
:106820002431E646624603E0944238D991F800E00C
:106830007144724491F801E092B2BEF1050FF3D1B8
:1068400091F802E0BEF1810FEED1174A03E0A342B6
:106850001BD292F800C06244634492F801C09BB21C
:10686000BCF1050FF3D192F802C0BCF1010FEED1DB
:1068700019B1002402230C714B7100210223117104
:10688000537120230380084810BD0029F9D002234A
:1068900000224B7120230A710380034810BD0021A0
:1068A000D3E700BF581800247C180024244910B5F1
:1068B000CC8C91F824C0644531D963462431E64636
:1068C000624603E0944238D991F800E07144724482
:1068D00091F801E092B2BEF1050FF3D191F802E018
:1068E000BEF1810FEED1174A03E0A3421BD292F80A
:1068F00000C06244634492F801C09BB2BCF1050F32
:10690000F3D192F802C0BCF1010FEED119B100240D
:1069100040234C710B7100214023517113712023CE
:106920000380084810BD0029F9D0402300220B71D4
:1069300020234A710380034810BD0021D3E700BF24
:10694000581800247C180024244910B5CC8C91F8E8
:1069500024C0644531D963462431E646624603E0EB
:10696000944238D991F800E07144724491F801E002
:1069700092B2BEF1050FF3D191F802E0BEF1810FA2
:10698000EED1174A03E0A3421BD292F800C0624442
:10699000634492F801C09BB2BCF1050FF3D192F8A9
:1069A00002C0BCF1010FEED119B1002440234C719B
:1069B0000B7100214023517113712023038008487B
:1069C00010BD0029F9D0402300220B7120234A7109
:1069D0000380034810BD0021D3E700BF58180024EE
:1069E0007C18002403460A2201481A80704700BF21
:1069F0009C18002438B5D0F8D432B03350F8235066
:106A00007DB195F81C32044623B9D5F818320BB184
:106A10006B7A8BB18121204674F0EAFB6B7A022BF2
:106A200000D038BD2046812174F0E2FB20460121D0
:106A3000BDE8384074F0DCBB012174F0D9FB20467E
:106A40008121BDE8384074F0D3BB00BFD0F8D42218
:106A500000EB82022DE9F041D2F8C0420646002C3C
:106A60004ED0B4F8643204F11007D4F870520846DE
:106A7000D2F8C422394603FB05F5D2F81080B5F5EB
:106A8000007FD4F86C2228BF4FF40075B5FBF3F3F8
:106A90009BB2C04700281BDB2B463A46812130467B
:106AA00074F064FDB4F86422B5FBF2F2D4E99B13F0
:106AB00011449B1AD4F83822521BC4E99B13C4F822
:106AC000382213B10020BDE8F08103232372F9E7D7
:106AD000D6F8D432B03356F823208AB192F8613216
:106AE0000424112003F148010133DBB202F83140E4
:106AF00002EBC101A342888008BF002382F8613203
:106B00004FF0FF30DFE700BF10B50E4B0E4C03F126
:106B100050021B6DD4F8AC15B4F8B005C4F8482683
:106B200088619847D4F84836002BFBD01B699847FA
:106B30000028F7D0B4F8B0350020D4F8AC251B04F9
:106B4000936110BD58180024A037002438B5084BB5
:106B5000D3F8483653B1DB6914460D4698474FF4D5
:106B60000073026800202A60238038BD1B68FFDEA6
:106B7000A037002408B5064BD3F8483623B11B696B
:106B80009847013840B208BD4FF0FF3008BD00BF44
:106B9000A0370024002070472DE9F041194C15461C
:106BA000B4F8BC25D4F8B8051604866123B30E46A4
:106BB00003EB050804E0D4F848360BB31B6998478B
:106BC000D4F84816E1B100234F68284631461A46EA
:106BD000B8470028EFD0D4F84836002BFBD01B690B
:106BE00098470028F7D0013506F50076A845E7D18B
:106BF000D4F8B805B4F8BC2582610020BDE8F08166
:106C0000FEE700BFA03700242DE9F041184C1546DF
:106C1000B4F8BC25D4F8B8051604866123B30E4633
:106C200003EB050801E01B699847D4F8481651B1F9
:106C30000023CF68284631461A46B847D4F848366C
:106C400010B1002BEFD1002313B11B69984710B985
:106C5000D4F84836F8E7013506F500764545E4D125
:106C6000D4F8B805B4F8BC2582610020BDE8F081F5
:106C7000A03700240020704708B520B9044870F000
:106C80002BFC044808BD044870F026FC014808BDF0
:106C9000D81C0D08EC3D0024FC1C0D08024808B56A
:106CA00070F01AFC014808BD201D0D08EC3D0024C1
:106CB000024808B570F010FC014808BD281D0D08F9
:106CC000EC3D0024024808B570F006FC014808BD00
:106CD000341D0D08EC3D0024D0F8D432B03370B52B
:106CE00050F823402CB30026124B054684F83C1282
:106CF000C4F8303204F50C7226720D23812104F59C
:106D0000047474F033FCD5F8C8321F220121C3F893
:106D10008C62A3F8781203F51E711868C3E9A142CA
:106D20009A79012A08BFC3F89442BDE8704074F014
:106D3000D5BA70BD55534253D0F8D42200EB82022D
:106D40002DE9F041D2F8C0420646002C67D0B4F8D5
:106D5000643204F11007D4F870520846D2F8C42205
:106D6000394603FB05F5D2F81480B5F5007FD4F859
:106D70006C2228BF4FF40075B5FBF3F39BB2C047FC
:106D8000002834DBD4F83802B4F86422401BB5FB89
:106D9000F2F5D4E99B13C4F8380229445B1BC4E91B
:106DA0009B13FBB1D6F8C80202FB03F301220021BA
:106DB000B3F5007FC0F88472A0F87822827928BFEA
:106DC0004FF40073C0F88C1200F51E71012AC0F850
:106DD000883208BFC0F89472006874F07FFA00200F
:106DE000BDE8F08119463046FFF776FFF7E7D6F8A1
:106DF000D432B03356F823208AB192F86132042499
:106E0000032003F148010133DBB202F8314002EB09
:106E1000C101A342888008BF002382F861324FF08D
:106E2000FF30DDE7D0F8D43200EB83032DE9F043E7
:106E3000D3F8C04283B0002C00F0B7801646127819
:106E400005460F465A2A5FD85A2A00F29B80DFE88F
:106E500012F04601990099005A0199009900990091
:106E6000990099009900990099009900990099005A
:106E70009900990099008E01990099009900990054
:106E8000990099009900AC01CD01990099003D014C
:106E90009900990099009900100299003602990012
:106EA0009900FA0099005E029900990099009900F2
:106EB000E1019900990099009900990099009900C1
:106EC00099009900990099009900990099009900FA
:106ED00099009900990099009900990099009900EA
:106EE00099009900990099009900990099009900DA
:106EF00099009900990099009900990099009900CA
:106F0000990099009900F001A82A53D0AA2A00F00C
:106F100064829E2A36D1D3F8C432084604F5197229
:106F200004F51A715B6898470146002840F0098310
:106F300094F86232022B00F00483D6F80A301ABAB1
:106F4000E2601BB104F110007FF024F9D4F868323C
:106F50000022013B190E61F30702190C61F30F22A5
:106F6000190A61F31742B4F8641263F31F624BBA53
:106F70006383002362612383D6F80A301BBAE3607F
:106F8000002014E094F86122052620250221531CDC
:106F90004832DBB204F8326004EBC200042B858077
:106FA00008BF0023617284F861324FF0FF3003B0F4
:106FB000BDE8F08394F80880B8F1000F7DD194F912
:106FC0001C22002A80F2058394F86222022A00F033
:106FD0008083D3F8C43208469B689847002840F065
:106FE000DE82D6F80230D5F8D4121BBAB031C4F81C
:106FF0006C32D6F8062055F8211012BAC4F8702267
:107000000029D2D01344D1F86802834200F24783AA
:10701000B4F8643202FB03F3D4F818229A424AD03F
:1070200091F861320524202003F148020133DBB2DC
:1070300001F8324001EBC202042B908008BF00230C
:1070400081F86132B1E794F80880B8F1000F34D1CB
:1070500094F91C22002A80F2BC8294F86222022A4F
:1070600000F03783D3F8C43238469B68984700282D
:1070700040F09582D6F80220D5F8D41212BAB03179
:10708000C4F86C22B6F8073055F821105BBA9BB2F1
:10709000C4F87032002988D01A44D1F86862B2422C
:1070A00000F27383B4F8642202FB03F3D4F81822CD
:1070B0009A4240F0E182022323724FF40073394672
:1070C0002846E36003B0BDE8F043BFE43379002213
:1070D0009B1AE26018BF012384F8623250E7D4F8AB
:1070E0001822002A40F0398294F86212022900F036
:1070F0004683D3F8C43238469B689847002840F04E
:10710000D382E0603CE7D4F81832002B00F02582EF
:107110007021002294F8603221740C21C4F81520EB
:10712000E17594F86112C4F811209942C4F819204D
:10713000C4F81D2084F8212011D004EBC30191F87C
:107140004012A17404EBC3010133B1F84412DBB265
:10715000A183042B14BF84F8603284F860221223C8
:10716000E36032799A4298BF1346E36008E7D4F8A7
:107170001822002A00F0F1817278D20740F1B18123
:10718000B378002B00F0CF81802B40F0E081082104
:10719000CC4A04F1180304F11000E16012F8011D5B
:1071A00003F8011D8342F9D1EAE6D3F8C432384628
:1071B000DB689847002840F074813279042A13462E
:1071C00028BF0423E360002A3FF4DAAE013BBD4A46
:1071D00004F1100099B201F111030A44234412F89A
:1071E000011903F8011D8342F9D1C9E694F862221E
:1071F0003379012A03F0030300F06A81012B00F0C8
:107200006C81022B00F06A81032B00F06681002361
:10721000E360B5E6737813F0020340F09881D4E997
:107220009B210A44D4F868128A4200F2E581E360A7
:10723000A6E6D3F8C4323846DB689847002840F009
:107240003881337A082B194628BF0821E160002BCA
:107250003FF496AE9C4A01F1100304F110000A4479
:1072600054FA83F312F8011D03F8011D9842F9D175
:1072700086E6D3F8C4320DF10202384601A95B68F4
:107280009847002840F06F8194F86232022B00F09A
:107290006A81BDF802200821206152BA019BA061D9
:1072A000013B62830C22E174E375190EE2601A0C53
:1072B0001B0A217562750222A375227677E6D3F840
:1072C000C43204F51972384604F51A715B689847A0
:1072D000002840F0368194F86232022B00F03181B0
:1072E000D4F868320822A082013BE260190E1A0C21
:1072F00061F30700190A62F30F20B4F8642261F306
:10730000174052BA63F31F60E282206138E694F8B6
:107310000890B9F1000F40F00081D4F81822002A3B
:1073200000F08A8194F91C22002AC0F21582D3F859
:10733000C43238469B6898478046002840F0F18167
:10734000D5F8D432384605EB8303D3F8C432DB6872
:1073500098470146002840F08281D6F80220D5F8EF
:10736000D40212BAB030C4F86C22B6F8073055F81F
:1073700020005BBA9BB2C4F8703200283FF415AE0F
:107380001A44D0F86862B24200F2C681B4F86422AE
:1073900002FB03F3D4F81822934240F0EC80B3F5DB
:1073A000007F4FF0010004F1100428BF4FF4007378
:1073B00004F8080C1A46D5F8C832C3F888229A791E
:1073C000C3F88C1203F51E718242C3F88442A3F8FD
:1073D000780262D1C3F894425FE0227A002A40F03A
:1073E0009C80D4F81812002900F0838194F91C12B3
:1073F0000029C0F22181D3F8C43238469B689847EF
:10740000D5F8D432002840F05A8105EB8303384682
:10741000D3F8C432DB689847002840F0F280D6F8F1
:107420000230D5F8D4121BBAB031C4F86C32D6F899
:10743000062055F8211012BAC4F8702200293FF432
:10744000B4AD1344D1F86802834200F22881B4F845
:10745000643202FB03F3D4F8182293427FF4E0ADC8
:10746000B3F5007F4FF0010104F1100028BF4FF485
:107470000073217200241A46D5F8C832C3F8882256
:107480009A79A3F8781203F51E71012AC3F88402D1
:10749000C3F88C4208BFC3F89402186873F01EFF4B
:1074A0006EE50A4A92F8823063F07F0382F88230F8
:1074B00083E6064A92F8873063F07F0382F88730CC
:1074C000BFE600BFD8180024DC1800245818002498
:1074D000022B3CD0012B7FF497AE002384F862325C
:1074E00095E6D3F8C43207EBC7013279D86900EBCF
:1074F000810003790533934228BF1346E360002BD4
:107500003FF43EAD03F110020344224413F8011D81
:10751000834202F8011DF9D132E53946284603B00D
:10752000BDE8F04308E406219A4A04F1160304F189
:107530001000E16012F8011D03F8011D8342F9D12A
:107540001EE53A220221284673F07CFB2DE5242219
:107550000521284673F076FB27E5202205212846E1
:1075600073F070FB21E528463A22022173F06AFB92
:107570004FF0FF301BE590F861320525202403F120
:1075800048020133DBB200F8325000EBC202042B98
:10759000948014BF80F8613280F8611205E5D5F857
:1075A000D432B03355F82320002A3FF4FEAC92F8D1
:1075B000613202243A2003F148010133DBB202F8C0
:1075C000314002EBC101042B888075D082F8613212
:1075D000EBE494F861320520202103F148020133E5
:1075E000DBB204F8320004EBC202042B91807FF47A
:1075F000DAAC84F86182D8E42122052173F022FB01
:10760000D3E4D5F8D432B03355F823208AB192F8B8
:1076100061320225272003F148010133DBB202F871
:10762000315002EBC101042B888008BF002382F88F
:10763000613205232372B8E494F8613205252020D5
:1076400003F148010133DBB204F8315004EBC1010E
:10765000042B88807FF4A7AC84F86122A5E4D5F8D8
:10766000D432B03355F82320002A3FF49EAC92F870
:107670006132022427209EE791F8613205252024FB
:1076800003F148020133DBB201F8325001EBC202D0
:10769000042B94807FF4D4AC81F8610285E491F8E6
:1076A000613205242120BFE43A220221284673F0EA
:1076B000C9FA0523237278E482F8618275E4B03355
:1076C00055F82320002AB4D092F8613202253A20DE
:1076D000A1E794F8613203F148010133DBB204F809
:1076E000312004EBC1013A22042B8A807FF45BAC89
:1076F0007FE794F861320525202003F14802013329
:10770000DBB204F8325004EBC202042B90807FF409
:107710004AAC84F8611248E490F8613205252124CE
:107720002DE7D5F8D432B03355F82320002A3FF4A2
:107730003CAC92F8613202243A2003F14801013353
:10774000DBB202F8314002EBC101042B88807FF4E8
:107750003DAF82F8619228E494F86132052020213F
:1077600003F148020133DBB204F8320004EBC20239
:10777000042B91807FF417AC84F8619215E43A22CF
:1077800073F060FA052323720FE491F86132052546
:10779000212475E7CE180024D0F8D432B03350F845
:1077A0002330CBB110B51A7A022A07D0033A012A46
:1077B00002D80021FFF790FA002010BD03F21F222B
:1077C00093F81D120446FFF72DFB0028F4DA01217F
:1077D0002046FFF781FAEFE700207047D0F8D43257
:1077E000B03370B550F8235025B12B7A044683B1DD
:1077F000012B01D0002070BD05F21F2295F81D124B
:10780000FFF710FB0028F5DA01212046FFF764FAA4
:10781000F0E7D5E98523C5F83832D0F8C832C5F885
:107820003422D3F88C321F2B04D12F4BD5F81022E1
:107830009A421AD095F861324FF0050C202120466B
:1078400003F148020133DBB205F832C005EBC20296
:10785000042B91804FF0020208BF00236A7285F862
:107860006132FFF7C7F8002070BD95F81D1201299D
:10787000E0D895F81E32013B0F2BDBD805F21F2212
:10788000FFF7D0FA00282B7A22DB013B022BB1D97B
:10789000EE681EB3D4F8D432B03354F82310002964
:1078A000A8D02046D1F83842D1F8183205F110029C
:1078B000A41BB342C1F838424FF0000428BF33463E
:1078C00081F83C4204240C72812173F04FFE91E751
:1078D000052B99D02046FFF78DF88BE731462046DF
:1078E000FFF7FAF986E700BF55534243554B002195
:1078F000554A1B685548A2FB032330B5DB0C544C9A
:1079000083B0013BC4F85C17C4F8541742F20F71FE
:1079100094F88927C4F84C07C4F85817C4F85037AE
:10792000002A00F08A8002254A49484884F889578D
:10793000FAF7C0FE0123484A0621372084F894371D
:1079400084F88A3784F88B3784F88C3784F88D373D
:1079500084F88E3784F88F3784F8903784F891371D
:1079600084F8923784F8933784F88937D2F8E8306E
:1079700043F02003C2F8E830D2F8E83003F02003E7
:107980000193019B70F02CFA344B4FF400025A60C3
:1079900094F88937012B3BD1D4F84C27304B314830
:1079A000B2F1804F18BF9A4284F88957D1680CBF52
:1079B0000123002341F00101824208BF43F001038B
:1079C00000F58060D160824208BF43F0010300F5FA
:1079D00080602549824208BF43F0010300F57840EA
:1079E000824208BF43F001038A4208BF43F001030B
:1079F00013B91E4B9A4207D191681D4B0B40062BC1
:107A000006D0B3F5803F03D0136843F00103136041
:107A1000184AD2F8D432B03352F8233043B1164862
:107A20000021164AC3F80802C3F81012C3F8042252
:107A30000020C4E9000003B030BD02F0FF0084F86C
:107A4000880770E70000002483DE1B430014004019
:107A5000A0370024F03E00240044025800E100E07A
:107A600000000140000400400018004000400140B8
:107A700007000100082E00242C5400242C4400246C
:107A800010B50B68054A064C136020600BB100204E
:107A900010BD73F033FD002010BD00BF042E002484
:107AA000EC30002410B50F4CA36D23B119689A88EF
:107AB0000B691A420AD0FDF7EBFE38B994F8203072
:107AC0000133DBB2072B84F8203003D9002384F87C
:107AD0002C3010BD044A0123126884F82C30E26176
:107AE00010BD00BFA0370024F030002410B50C4CAE
:107AF000A36D23B119689A880B691A420BD0FDF760
:107B0000C7FE40B9074B012284F820001B6884F8A7
:107B10002C20E36110BD002384F82C3010BD00BF81
:107B2000A0370024F030002470B5164D0021164E09
:107B30006B6C2C681B04B162144A0D21A3602046B3
:107B4000E3681A4041F20D13134341F28832E360B7
:107B5000FBF792F950B16B6B03436B630C4A09233B
:107B60000020126886F82C30F26170BD636903F45E
:107B7000F053B3F5006FF1D10423022086F82C30C6
:107B800070BD00BF94360024A0370024C0E0FEFF83
:107B9000F030002470B50C4D04460E4695F82C309C
:107BA000042B0AD0082B06D16B6A83420AD0FFF758
:107BB000BBFF022801D0012070BD0823C5E909469A
:107BC00085F82C30022070BDA037002470B5804CA1
:107BD00094F82C506B1E082B1BD8DFE803F06C6068
:107BE000701A4705321A24007A4B5B6A002B60D169
:107BF000794B072265691B6884F82C20E361002D0E
:107C000057D0A3690120D4E90221A84794F82C5049
:107C10006B1EDBB2022B46D9042D18BF082D0CBFFA
:107C20000120002070BDFDF707FE002840F0C48051
:107C3000694AE3691268FA339342EDD2FFF732FFE3
:107C4000C6E7FDF7F9FD0028F2D0A36A0022012B58
:107C500084F8202040F2B480626A013B082101329E
:107C6000A36284F82C106262012070BD594B1E6A19
:107C7000002E65D1FDF7E0FD002868D0042365697A
:107C800084F8206084F82C30002DEDD0A3693046B4
:107C9000A268E168A84794F82C506B1EB9E76FF012
:107CA000CFFE04285FD04C4BE2691B689B1AC82B9F
:107CB00077D8002070BD022384F82C3088E7FEF7C7
:107CC000D9FA0028EFD1454B0421A06293F82C206B
:107CD00084F82C10D88D196B84F83620090E1A6B95
:107CE000A086120C84F83710196B186B84F83820B2
:107CF000090A84F83A0093F8340093F8352084F8A0
:107D00003910120984F83B0093F8350084F84020BC
:107D1000996B00F00F00DD8FDA8FE163D98FC2F32A
:107D20000B1384F8410043EA152301F00F0203F01E
:107D30000F0384F8442003F5FA63A4F8423047E7C0
:107D4000254AE369126864339342BFF465AFFFF7D5
:107D5000A9FE6569002D3FF43BAF0022A369E168ED
:107D60001046A84734E7FEF785FA00289BD11C4B44
:107D70001B78002BA3F10203B3FA83F308BF01259C
:107D80005B0984F8215084F82230FEF773FA00284A
:107D90007FF454AF114B03229B6C84F82C20236397
:107DA00016E7FFF77FFE94F82C00042818BF082878
:107DB0000CBF0120002070BD042384F82C3053E751
:107DC000FAD1FFF7B1FE94F82C506B1E21E700BFEB
:107DD000A037002414370024F0300024403700245A
:107DE000103700242DE9F04106460D4690461F4607
:107DF0004E4C94F82C1004290AD0082906D1636A45
:107E0000B34205D0FFF790FE0228F2D0012084E0B3
:107E100006220123C4F8148084F82C20444A2374D9
:107E20005362EB06A761C4E9025660D1BFF34F8FDE
:107E3000404A05F500712B46C2F8683220338B4268
:107E4000FAD1BFF34F8FBFF36F8F002D67D0DFF8EC
:107E5000F08098F83030012B49D1731CD8F85010BD
:107E600000228B42C8F834204CD80323D8F8007085
:107E7000C8F81C50182188F830304FF40073FA62AB
:107E80003846C8F82030D8F838302B4A012B4FF04C
:107E9000FF337B624FF4007318BF7602BB62FB6A4C
:107EA00023F0FF0343F09003FB62FB6843F04003C1
:107EB000FB609023BD6501253D65C8F82C30BE6090
:107EC000FB681A4041F21813134341F28832FB60F9
:107ED000FAF7D2FFE8B1194B0022BB63D8F834306F
:107EE0000343C8F8343088F83050C8F82C20FFF726
:107EF000D9FD656925B1A3690022E1680120A84781
:107F000003200AE0D8F8343043F00073C8F8343066
:107F1000EDE7FB6B43F48D73FB63BDE8F081084A2A
:107F2000536B43F000635363E1E700BFA0370024C5
:107F30001437002400ED00E0C0E0FEFFFF0FE01F5B
:107F4000943600242DE9F84F544F0C4680461646CF
:107F500097F82C101D46042908D0082902D00020CB
:107F6000BDE8F88FFFF7E0FD0228F8D114F01F02FA
:107F700069D101234A49C7F89847C7F8A0370B626F
:107F80004FF40073474941F8043C002C79D0DFF8E6
:107F900024B19BF83010012955D108F10100DBF81C
:107FA0005010CBF83420884271D8DBF800A04FF095
:107FB000010911215046CBE9094303238BF83030E6
:107FC000DBF83830CAF82C20012B4FF0FF33CAF809
:107FD00024304FF4007314BF4FEA48224246CAF8D7
:107FE0002830DAF82C3023F0FF0343F09203CAF86C
:107FF0002C30DAF80C3043F04003CAF80C308123FF
:10800000CAF85840CAF85090CBF82C30CAF808206B
:10801000254ADAF80C301A4041F21113134341F2A9
:108020008832CAF80C30FAF727FFB8B11F4B00228C
:10803000CAF83830DBF834300343CBF834308BF8EF
:108040003090CBF82C20FFF72DFD7C69002C86D0DA
:108050000022BB69F9681046A04780E70523144A4F
:1080600048467E6187F82C30DAF83C30BD6143F435
:108070009573CAF83C301368C7E90248FB61BDE854
:10808000F88F0C4A536B43F000635363DBE7DBF874
:10809000343043F00073CBF83430D4E7A0370024F9
:1080A00014370024403F0024C0E0FEFFFF0FE01F14
:1080B000F0300024943600242DE9F04104464FF4BA
:1080C0001D707DF097FF054600285BD0D4F8D47270
:1080D00004EB8707C7F8C002237CC4F8BC02002B5E
:1080E00045D0402302220121204672F079FF01226F
:1080F00040234FF001082046A4F878218121022274
:10810000002672F06DFFA4F83880D7F8C4323046EC
:108110002E81A5F8606285F862621B689847D4F8E2
:10812000C84294F894342768434508D03846FAF793
:108130006DFF41463846FAF741FF84F8946405F52F
:1081400004751F220023384604F51E71C4F88C32D2
:108150000123C4E9A152A279A4F878329A4208BF57
:10816000C4F8945273F0BAF80020BDE8F0814FF4DF
:10817000007302220121204672F032FF01224FF4E7
:108180000073B6E7D4F8D4320220B03344F8235059
:10819000EBE700BFF0B5002383B0ADF80630D0F8B0
:1081A000D43200EB8303D3F8C0524DB10A780446B1
:1081B00012F0600036D0202805D0204673F054F825
:1081C000032003B0F0BD4878FE2849D0FF28F4D141
:1081D0004B88002BF1D1CE88002EEED11006ECD4C6
:1081E0004FF4807381212B8105F50475D4F8C842C2
:1081F000204674F0C1FD2046012174F0BDFD1F2210
:10820000012304F51E712068C4F88452A4F8783262
:10821000C4E9A226A2799A4208BFC4F8945273F026
:108220005DF846E04B780B2BC7D801A252F823F03B
:10823000B782040827830408BB810408BB810408B3
:10824000BB810408BB810408BB810408BB8104080E
:10825000BB810408BB810408EF820408A7820408DC
:108260004E88002EA9D1CF88012FA6D11206A4D501
:10827000D3F8C4329B699847022328604FF4807179
:10828000C4F89432D4F8C832C4E906779A7999824E
:1082900003F11401012A5F621D629E6241D01868D9
:1082A00073F01CF805E094F89C32032B85D18B7891
:1082B0006B60002085E794F89C32032B7FF47DAF40
:1082C0000222D4F8C8320020C4F8942203F1140129
:1082D000C4E906220DF106049862C3E908424FF48E
:1082E00080729A829A79012AD9D11C63D7E794F8CF
:1082F0009C32032B7FF461AFD4F8C83201220221F3
:1083000004350020C4F894124FF48071C4E90622A9
:10831000C3E908529A79998203F11401012A9862FB
:10832000BDD11D63BBE794F89C32032BC1D14B88B0
:10833000002BBED1D4F8C8628F8896F89434012BF4
:108340000AD001233906306886F8943410D4FAF73D
:108350005DFE002386F894346B7A022B0DD03A062A
:10836000A7D5012BA5D001212046FEF7B5FCA0E73B
:1083700007F00F01FAF722FEEBE72046812172F0A9
:1083800037FF0121204672F033FF92E7F8B5D0F8AD
:10839000C85201260446002295F89434A5F8786264
:1083A000B34227D03146286885F89464002773F0DB
:1083B0005DF940F20113A4F878713246314628681D
:1083C00085F894642B8773F051F985F89474D4F888
:1083D000D4320025B033258754F8230040B17DF016
:1083E00011FED4F8D432B03344F82350C4F8BC5250
:1083F0000020F8BD40F20113A0F878212B87E6E7B2
:108400002DE9F04FDFF8B4B38BB0DBF8A4A7DAF8AE
:10841000143013F0010902D00BB0BDE8F08FDAF888
:108420001420DAF818301A42F6D0DAF808280AF5DB
:108430000061DAF81430C2F30D220291CBF8782CE7
:10844000DAF8182013409D0705D5DAF8143003F048
:108450000203CAF81430DAF81430DAF8182013409E
:10846000DC061BD5DAF8183023F01003CAF81830F0
:10847000DAF8203003F4F01203F00F05B2F5802F84
:1084800000F04985B2F5402F00F02583CDF804A017
:10849000019A936943F01003936101E0CDF804A0C1
:1084A000019A536992691340180300F19C82019A62
:1084B0005369926913405F0300F1D281019B5A69AD
:1084C0009B691A4200F1EA80019A5369926913404C
:1084D0001B0509D5029B9B68DF0700F16485019AA3
:1084E000536903F40063536101994B698A6913402E
:1084F0001E0116D54B6903F000634B619BF8703C7D
:10850000002B00F0C282DBF8843C93F89C22042A02
:1085100004D093F89C22D2B283F89D22042283F8DF
:108520009C22019A536992691340DD0400F148814D
:10853000019A5369926913409C0400F1D780019A13
:10854000536992691340190700F1C38001994B697F
:108550008A6913401A067DD44B698A691340DB028D
:1085600028D59BF8A887B8F1010F1ED9924D0AF5BE
:108570001267012604E0013620372435464514D021
:1085800095F83C303A68012BF5D1002AF3DA66F011
:108590007F0085F83B30C0B26FF04EFCEBE7019AEC
:1085A000536992691340DA0204D5019A536903F4BE
:1085B00080135361019A5369926913409F0231D528
:1085C0009BF8A877012F28D90AF532627A4B01214E
:1085D00003E0B94203F124031FD093F87C02013178
:1085E000146820320128F4D1002CF2DADBF8785C30
:1085F00085EA1445EE07ECD483F87B02DAF818001C
:1086000040F08000CAF81800DAF814000506E0D43B
:10861000029A536843F400735360019A536903F458
:1086200000135361019A5369926913405C0000F191
:10863000BD8001994B698A69134058077FF5ECAEFC
:108640004C68610700F1BF84DBF8A4375A68144313
:108650005C60E1E6DAF818309BF8A88723F0800325
:10866000B8F1010FCAF8183099D9534D01262F4699
:1086700003E001362437464507D097F87B32012BBB
:10868000F7D1F0B26FF0D8FBF3E7019B5A699B6911
:108690001340DB028ED59BF8A88768E7029A5368DF
:1086A00023F0010353609BF8703C012B00F0018222
:1086B000DBF8843C93F89C22042A04D193F89D2291
:1086C000D2B283F89C22019A536903F000435361AC
:1086D000FAE6DBF8840C90F89C32032B00F0ED8175
:1086E000019A536903F0080353612FE7019AD2F806
:1086F00000396FF30A03C2F8003902F50063D2F8BB
:10870000042842F480725A609B68980700F1F78150
:1087100013F0060F0CBF00230F238BF8AB37F9F7CC
:10872000E1FA9BF8AB67022E00F06F844FF4105310
:108730000199003EDBF8845CCA6818BF012622F468
:108740007052CA60CA681343CB600123002185F8C8
:108750009C32D5F8B8326960C5F8A41285F8A01229
:10876000C5F894121BB15B680BB1284698470022EC
:108770004024012740231146284672F031FC23464D
:10878000002280212846C5F86041A5F8647172F086
:1087900027FCDBF8843CDBF8A427AF842C621E7432
:1087A0005369019203F400535361C8E6019A536977
:1087B00003F0804353613CE7443F0024A03700248A
:1087C000029A10210198536823F001035360FAF7CD
:1087D000F5FB9BF8A807E0B10AF510634FF67F316F
:1087E000996009F101091A682033814522F40012C9
:1087F00043F8202CC3F8E811D3F8E02122F400124A
:10880000C3F8E021D3F8E02142F00062C3F8E02190
:10881000E6D1029AD36943F00113D3619BF8B337D1
:10882000002B00F03B81029AD2F8843043F00B0316
:10883000C2F88430536C43F00B035364DAF8003809
:10884000019C23F4FE63B44A2046CAF800389BF822
:10885000AA1772F047FC636903F48053636167E60B
:10886000019AD2F81878D2F81C381F40BFB2002FF6
:108870003FF424AE0AF510614FF00008CDF80CA0CB
:108880001346A64D44468A46CDF8109008E07F086E
:1088900004F1010405F124050AF1200A00F03181F8
:1088A000FE07F4D5D3F8102804F00F01D3F834688C
:1088B0004FEA4419CE40F601F6B2164303F51062B2
:1088C00002EB441292681640E2B2F007019221D501
:1088D0000120029ADBF8848C526B00FA01F122EA43
:1088E000010202994A639BF8AA17CAF8080081425C
:1088F00000F078832B6A0593002C40F0FA82D8F8B8
:108900009432022B00F0E88398F8A03213B10023D0
:1089100088F8A032320702D50823CAF80830F306D7
:1089200002D51023CAF80830700602D54023CAF8D1
:108930000830B10700F110813206DBF8A437A6D564
:10894000D5E909068642A2D8811BEA6903F5106EB3
:108950008A42CE4428BF0A46DEF81810033289B294
:10896000B1EB920F31D39BF8AA8703F5805C019499
:1089700042460CEB043C98461346B04240F29083CA
:10898000811BEA69914228BF11462A6A01F1030955
:108990004FEA990973B98CB20334A4080AD002EBE8
:1089A000840452F8040BA242CCF80000F9D12A6AE0
:1089B000D5E909060A440E442A62DEF81820AE62A0
:1089C00092B29145D9D9019C4346B0423FF65FAF80
:1089D00004F00F0201219140D3F8342822EA010269
:1089E000C3F8342853E70198D0F81838D0F81C2879
:1089F00013405FEA13483FF45AAD484B0AF530661E
:108A0000CDF80CA000279A46CDF8149008E05FEA54
:108A1000580807F1010706F120060AF1240A74D06C
:108A200018F00109F3D0FBB200F530627D0101932B
:108A300002EB47139C68D0F814180C40E1076FD480
:108A4000210700F19580E50601D51023B360A0074A
:108A50000FD5039B5B69190604D5029A536843F44A
:108A6000806353609AF85732012B00F01C83022375
:108A7000B360A20601D52023B360A30402D54FF44E
:108A80000053B360DBF8A407C1E701238BF8703C07
:108A90004B6DC3F38303CBF8743C42E5029942F279
:108AA0002B034A6913434B610B6943F00B030B61C2
:108AB000C4E600238BF8703C05E6D0F8B832002BF2
:108AC0003FF40EAEDB69002B3FF40AAE9847DBF8AB
:108AD000A437019304E605EBC5020AF58051C3F300
:108AE0000A130BEB8202D2F80C0A03440868CBF895
:108AF000400C0968C2F80C3ACBF8441CC6E40223C7
:108B00000BE6DDE903A90193D8E4DDF80CA0DDF85C
:108B100014900190CBE400BFE0430024443F0024C4
:108B20000121B1609BF8AA17D0F840E00129D3F8E1
:108B300008C000F0A582B6498E4500F09B83DBF8A3
:108B4000083A3B4300F04984DAF860220199DBF8E7
:108B5000840C72F031FD73E721460398FAF72EFA80
:108B6000EB7D012B00F091830223CAF80830E3E685
:108B7000DBF8A4270823B36002F53063126C2B44A2
:108B800010460492A34A9968904204D90A0402D577
:108B90004FF400429A60DBF8845C01219BF8403C72
:108BA00005F2AA2085F8AA329BF841EC079085F8D7
:108BB000ABE2BBF8422CA5F8AC22BBF844CC069241
:108BC000A5F8AEC2BBF8462CC5F8941203F01F01FD
:108BD000A5F8B0220129C5F8982200F0A582022943
:108BE00000F00783002940F0DE8203F06003202BB1
:108BF00000F0E983402B00F0E683A3B9BEF1090F32
:108C000011D8DFE81EF0E800C1001000D800100005
:108C10007D00640010003E002300D5F8B4325B698B
:108C2000002B40F0C285284672F01EFB794B049A57
:108C30009A427FF608AF9BF8AA1701297FF403AF89
:108C4000754ADBF8A40772F04DFAFCE69DF818901F
:108C5000B9F1010F8BF8889CE5D895F89C32DAB20F
:108C6000022B069200F00385032A00F0D7842846E1
:108C700072F0FAFAD5F8B832494628465B68984748
:108C8000D4E7012ACFD195F89C120229CBB200F289
:108C9000A684002BC7D0D5F8C832002128464FF053
:108CA000020C40F8081FC5F894C2C5E90622C3E9C2
:108CB000092118624FF4807203F114019A829A79A3
:108CC000012A08BF1863186872F008FBAEE7069B1C
:108CD00000221B0AADF82620013B062BA3D801A2D7
:108CE00052F823F0C58E0408A98E04087F8E04086C
:108CF000278C0408278C04081D8E0408D78E0408CE
:108D000052EA0C0C8FD1069B7F2B8CD895F89C32A5
:108D1000032B88D00698D5F8C8325FFA80F985F819
:108D20009E9293F89424012A12D01A684FF0000CF6
:108D300083F81190D2F8001821F4FE61C2F80018EF
:108D4000D2F8001841EA0011C2F8001883F894C460
:108D50000422002003F11401C5F894224FF480721C
:108D6000A8619A829A799862012AC3E9080008BF2B
:108D70001863186872F0B2FAB9F1000F40F072840B
:108D8000012385F89C3251E795F89C32013B022B78
:108D90003FF649AF069B012B7FF448AF0020D5F882
:108DA000C832C5F8A402A8610422C5F894229862CA
:108DB000C3E908007EE7069B012B00F06F84069B49
:108DC000022B7FF430AF4FEA1C2CD5F8C8320020BC
:108DD00085F8A0C2E7E795F89C32013B022B3FF6ED
:108DE00022AF022A7FF41FAFD5F8A4322846002B09
:108DF00018BF4FF0030940F80C9FD5F8C832C5F8EA
:108E00009422C5E90622C3E9080200229A6251E7CA
:108E10000A31544F0A30544FE04300242B7C002B7E
:108E20007FF401AFD5F8B8320DF126005B6B98479F
:108E30000346B5F8B002002800F03884BDF82620BB
:108E4000002A3FF4F0AE82424FF0020128BF0246F2
:108E5000D5F8C802C5F8941200F11401C5E906223C
:108E6000C0E90832002282624FF4807282828279E5
:108E7000012A08BF0363006872F030FAD6E69DF855
:108E8000180005283FF6CFAE01A353F820F000BF2D
:108E9000E3970408D5970408C7970408B99704080E
:108EA0001B8C04089F9704082A7CD5F8B832002A46
:108EB00040F072849B6A0DF1260098470222034617
:108EC0004270B6E7D5F8B4320DF12601287C1B6854
:108ED00098470346ADE72B7C002B7FF4A4AED5F872
:108EE000B8320DF126001B6B9847072203464270EB
:108EF0009FE798F89C32032B7FF40CADD8F8B8327A
:108F00005B69002B3FF406AD002240460199C8F88A
:108F1000D4229847FEE447F6F07213423FF4B6AA13
:108F200005EBC502C3F388144FEA131CC3F3011306
:108F30000BEB8202EE00D2F8047A002C00F00083E2
:108F40000AF5805E002239460132DEF800009442C4
:108F500041F8040BF8D107EB8404002B00F0BC812E
:108F60000AF5805223441068002220FA02F10832E8
:108F700004F8011B9C42F8D173190BEB8303D3F85F
:108F8000047ADBF8A43701937319CCF30A0C0BEBCA
:108F900083036744D3F80C2AC3F8047A6244C3F805
:108FA0000C2AFFF775BADBF8843C93F89C22042A5C
:108FB00004D093F89C22D2B283F89D22042283F835
:108FC0009C22FFF78CBADBF8840C0122D0F8B8326F
:108FD00080F89C22002B3FF437AB5B6801799847FF
:108FE000FFF732BBD5E9070202442A62002C80D188
:108FF000DBF8C407DBF8C8270590002A7FF47FACB4
:109000001846B74A72F06EF879E4B64BB64A034494
:10901000934240F25281B54BB54A0344934240F229
:109020005781B44BB44A0344934240F23582B34B68
:10903000B34A03449342C0F06B82B24BB24A03443A
:10904000934240F29182B14BB14A03449342C0F043
:109050008F82B04BB04A03449342FFF467ABAF4BEF
:10906000AF4A03449342C0F0D582AE4BAE4A0344AC
:1090700093422CBF4FF4C0534FF4E053FFF758BB5B
:109080001CF0080F00F01D81A84A96457FF6D8AC69
:109090001CF4004F3FF4D4AC4FF400429A60CFE48C
:1090A000019C434694E400238AF85732DBF8840C91
:1090B000D0F8D432AE3350F82330002B3FF4D7AC85
:1090C00090F89C22032A7FF4D2AC5B6A002B3FF419
:1090D000CEAC01999847CAE4D8E90732934200F22E
:1090E000278100F0988198F89C32032B00F0C8810A
:1090F0008021404672F07CF805230020C8F89432A5
:10910000D8F8C8329A7903F51571C3F86802012AB4
:10911000A3F85402C3E9980008BFC3F870021868A6
:1091200072F0DCF8FFF7F0BB03F060025B0602D5DB
:10913000402A7FF478AD95F89C32013B022B3FF634
:1091400072AD5FFA8CFCBCF1030F3FF66CADD5F845
:10915000B8329B68002B3FF469AD4FF000090799C6
:109160002846C5F8D4929847B5F8B022002A7FF473
:109170005DAD00287FF45AAD0422D5F8C832C5F899
:109180001890C5F894224FF4807203F11401C3F8CB
:1091900028909A829A79012AC3E908997FF493ADBD
:1091A000C3F830908FE51B06D5F8C85200F12D8129
:1091B000002385F8553205F5157301224FF000099B
:1091C0009A7083F8009095F8941491423FF42EAD74
:1091D000286885F894245A781978069071F0CEFFA3
:1091E000069805F29C42A97971F07CFF85F8949469
:1091F0001CE503F06003202B00F07C81402B00F085
:109200007981002B7FF40FADBEF1010F5FFA8CF175
:1092100000F04681BEF1030F00F07E81BEF1000F29
:109220007FF401AD95F89C32022BDAB200F0A481F4
:10923000032A7FF4F8AC01F00F0314221CF0800F16
:1092400002FB035340F0B281B3F86431002B3FF4CA
:10925000EAAC02FB015202F5AA70002940F02B8211
:1092600000230360D5F8C8320222C5F89422C5E96C
:109270000622C8E51CF4004F7FF40EAF1CF0200F4F
:109280003FF462AC20229A605EE40023EB75DBF8C9
:10929000840CD0F8D432AE3350F82330002B3FF496
:1092A00063AC90F89C22032A7FF45EAC1B6A002B0F
:1092B0003FF45AAC0199984756E44FF47053FFF7C6
:1092C00037BA1CF0200F60D020229A60FFF7B8BB9D
:1092D0004FF46053FFF72CBACDF804A054E600BF5A
:1092E000E0430024405327FFFF340C00401E1BFFC7
:1092F0003F420F0000DC0BFF7F4F1200808CF9FE15
:1093000020D6130060B6E5FE5FE3160000D3CEFE64
:1093100040771B00C05BB3FEC091210000CA91FEE4
:1093200020753800E05459FEE09C41000A30544F4B
:109330009A1AD8F8C832C8E906225A6203F1140111
:10934000059A1A6200229A624FF480729A829A7980
:10935000012A01D1059818631868CDE9050371F059
:10936000BDFF069B00209A7903F51571C3F86802CA
:10937000012AA3F85402C3E9980008BFC3F8700299
:10938000059871F0ABFFFFF7BFBAC64A964503D9FF
:109390001CF4004F7FF480AE1A69DAF87432C2F31D
:1093A00012029B1ACAF86832002F7FF4CDABDBF8AB
:1093B000082A002A00F0D280DBF8042A1A44CBF8ED
:1093C000042AFFF7C1BBD5F8D43228460799AE333B
:1093D00055F823309B68984728E4016CB14B9942BB
:1093E00003D91368002BFFF6AFAB00231361136999
:1093F00043F400231361136943F0180313611369E5
:1094000043F0C0431361FFF79FBB4FF001036B753F
:1094100005F11403D1E6D8F8182093423FF663AE65
:10942000D8F898329A42BFF45EAED8F8C83200201D
:109430004FF48072C8F8180003F114019A829A79E7
:109440009862012AC3E9080008BF18631868CDE9CB
:10945000050371F043FF069B4FF0000C059803F5E0
:109460001571C8F898C29A79C3F868C2012AA3F89E
:1094700054C2C3E998CC7FF453AEC3F870C24FE630
:10948000D8F8B832DB68002B3FF432AE00224046F9
:10949000C8F8D42298472BE64FF45053FFF748B949
:1094A00095F89C32022BDAB24CD0032A7FF4BBAB86
:1094B000069B002B7FF4BAAB4806D5F8C89240F063
:1094C00006810422002309F11401D9F80000C5F82F
:1094D00094224FF48072AB61A9F8142099F8062009
:1094E000C9F82830012AC9E9083308BFC9F8303063
:1094F00071F0F4FED5F8B83200229B68C5F8D4228A
:10950000002B3FF493AB079928469847FFF78EBB93
:109510004FF44053FFF70CB995F89C32022B5FFAD9
:1095200083FC0FD0BCF1030F7FF47DAB480603D062
:10953000069B134300F0C780D5F8C832002032E400
:109540003C460AE54B0628463FF46EAB71F050FEF0
:109550002846802171F04CFEFFF768BB524A01217A
:1095600071F0C0FDFFF7F0BA4FF43053FFF7E0B8E9
:109570004FF42053FFF7DCB84A067FF454AB1CF0DD
:10958000800FD5F8C8324FF002024FF0000114BF2F
:1095900005F1140005F5AA700160C5F89422C5E92B
:1095A0000622C3E909211862FFF784BB9B8C002BBC
:1095B0003FF439AB01F07F01481C00EB800005EB64
:1095C000800000293FF44CAE2422D5F8C83202FBBB
:1095D00001318A7D003A18BF0122026044E6032B64
:1095E0007FF421ABD5F8C8320221C5E90622C5F8BF
:1095F000941204355A62002203F114011D629A622A
:109600004FF480729A829A79012A7FF45CAB1D63D1
:10961000FFF759BB4FF40053FFF78AB8B9F1000FB9
:1096200000F0AE806968012986D0D5F8B832C9B299
:1096300028465B6898479BF8881CD5F8B832696063
:10964000002B3FF479AF1B682846984700283FF469
:1096500073AF284671F008FED5F8B832297928464C
:109660005B689847022385F89C32FFF7DFBAB9F1AF
:10967000000F3FF481AD0121D5F8B8326960002BAD
:109680005AD01B6828469847002855D0284671F0C4
:10969000EBFD069B85F89C32FFF7C8BAC5F8A432EB
:1096A0004AE700BF0A30544FE0430024D5F8C832DF
:1096B000A861FFF779BB2422D5F8C83202FB01313B
:1096C00091F8562286E7284671F092FD34E701F0C2
:1096D0000F0199F804308B42FFF4F3AE01EBC103A4
:1096E0001CF0800F4FEA830341D103F5157300226C
:1096F00009EB030C242303FB019383F855224FF05D
:1097000000038CF800108CF8023099F89434012B87
:109710003FF4D7AE0123D9F8000089F894349CF8BF
:1097200004309CF801209CF8001071F001FD4FF00E
:10973000000389F89434C4E60422D5F8C832002026
:10974000C5F894224FF48072A86103F114019A8243
:109750009A799862012AC3E9080008BF186318685B
:1097600071F0BCFD032385F89C32FFF75FBA143318
:10977000012209EB030C242303FB01935A75BEE776
:10978000022349462846C5F8049085F89C32D5F84E
:10979000B8325B689847EFE4DB6AFFF78CBBD5F81B
:1097A000B4329B69002B3FF43EAA0DF12601287CC0
:1097B00098470346FFF73DBBD5F8B4321B69002B31
:1097C000F3D1FFF730BAD5F8B432DB68002BECD117
:1097D000FFF729BAD5F8B4329B68002BE5D1FFF723
:1097E00022BAD5F8B4325B68002BDED1FFF71BBA82
:1097F0002DE9F8434B4BD3F84C57EE682C69A7077B
:1098000001D5B00736D4610701D572072AD42707DE
:1098100001D530071ED4E10601D5F20612D4E707C0
:1098200001D5F0073BD414F4025F2BD031066FD47E
:10983000600601D5710671D4A20601D5B30629D4FC
:10984000BDE8F8836FF010022A610022E96983F80D
:109850006827E4E76FF008022A610022E96983F8CB
:109860006827D8E76FF004022A610022A96983F80B
:109870006827CCE76FF002022A610022A96983F809
:109880006827C0E7E305D3D53706D1D56FF48073D9
:109890002B61CDE76FF020032B61BDE8F883224BED
:1098A0006FF001029D422A61BDD1DFF88C801F4B11
:1098B000D8F800201F68BA42B5D01D4888BFC2F54D
:1098C00080571C4B98BFBF1A1A44D0F8D432B0331B
:1098D00050F82330002BA6D0D3F81492C3F80822F6
:1098E000C3F81072B9F1000F9DD10121C762C3F80E
:1098F00014123B46812171F039FED8F800301F4424
:10990000B7F5805F14BF3B464B46C8F800308AE786
:109910006FF40253E2052B618AD5B7E76FF040037D
:109920002B6189E7A037002400140040E8300024B0
:10993000082E00242C540024E43000242DE9F84F94
:10994000234B81468A46D3F8BC32D3F81422002A2E
:10995000FBD1BAF1000F37D009EB0A031D4E09F114
:10996000FF39DFF8788003F1FF3B7027326819F880
:10997000011F531C1848C3F30B0381543360EFF3EA
:10998000118287F31288D8F80030D2B2316882F39E
:1099900011888B42A3EB01038CBF0022012203EB51
:1099A0000233012B0ED10AF0E9FD04460D460AF000
:1099B000E5FD001B61EB0501B0F57A7F71F1000157
:1099C000F5D3DCE7D945D1D15046BDE8F88F00BFCB
:1099D000082E0024E83000242C540024E430002415
:1099E00002784368022A0FD00B490269D1F87C0241
:1099F000023A184010B4400AD1E99C1404FB02005A
:109A00005DF8044B08447047034AD2E9992102EB00
:109A1000410202EB53207047A03700242DE9F04F9C
:109A200083B002F00207844D019308B9002F6AD178
:109A3000D5F86C42002C53D14FF0FF3E7F4C4FF0D5
:109A4000000CF146F046F246E36994F82A60984229
:109A500000F0A080002E3BD0012E05EB0C1B0AD19C
:109A60009BF88B60F30706D416F07E0F03D1F6093E
:109A700000F09380E0460CF1010C1034BCF1080FAB
:109A8000E2D1BEF1000F04DAB8F1000FC0F2978006
:109A9000C646D5F8FC400EF1020605EB0E1801345F
:109AA00005EB061CC5F8FC400CF1600CCCF804403A
:109AB000C8E91F040024CCF8084005EB061494F80C
:109AC0006A40042C1FD8DFE804F029441A444600F9
:109AD000E6460CF1010C1034BCF1080FB4D1D0E70C
:109AE000D5E99C3606FB0434A042A5D395F818327C
:109AF00013B9012385F81832012385F8613000205D
:109B000003B0BDE8F08F95F81832002B53D0012335
:109B1000022085F8613003B0BDE8F08F12F0010437
:109B2000D5F878C073D105EB0610019B4FEAE20C23
:109B300090F86B80032B6CF3C71880F86B8064D9A6
:109B40004FF6FF70834228BF034605EB0610A0F8CE
:109B50006830002F45D1500707D505EB061090F867
:109B60006B3043F0010380F86B30D3060AD505EB68
:109B7000061696F86B30C3F34502013262F34603D2
:109B800086F86B30AB6F012003EB4E230B6003B004
:109B9000BDE8F08FC6B9E6467BE7666A1034B24589
:109BA00088BFE1460CF1010C88BFB246BCF1080F3A
:109BB0007FF44AAF65E7012385F81832A7E7B9F1CA
:109BC000000F9CDBCE4664E7D5F8FC400CF10206A2
:109BD000E646013405EB061CC5F8FC40CCF86440B1
:109BE0006BE7D5F80001D5F8FC3001300133C5F83A
:109BF000000105EB0E10C5F8FC30C0F8803005EB15
:109C00000613042083F86A00A5E723469DE7D5F8EC
:109C10004836002B3FF473AF5C680CEB4E210023F9
:109C2000074AA04700283FF46AAF05EB0616022357
:109C300086F86A3063E700BFA037002400380024AC
:109C4000F566040870B5114D82B00E4695F8603087
:109C5000022B16D1020AC4B2D5F86402002301A96E
:109C600010440322FFF7DAFE012808D195F860308E
:109C7000019A022B0CBF22F8146042F8246002B053
:109C800070BDC0F3D41200F07F04E5E7A0370024D4
:109C90002DE9F04F444E0D4683B0174696F86010FC
:109CA0002B6803293ED0022961D14FEA13294FF4D2
:109CB000807A5FFA83F8421E012A23D84FF0010B05
:109CC0009F421AD901288CBF00240124D6F8DC2138
:109CD0001AB1D6F8F81199424CD0D6F86402002394
:109CE000092201A94844FFF799FE012823D0022840
:109CF00014D020B12B689F42E8D803202F6003B016
:109D0000BDE8F08FB8F1000F13D096F8183213B9F0
:109D1000012386F81832012386F86130022003B04F
:109D2000BDE8F08F4FF0800AC3F3D41903F07F0829
:109D3000C1E7D346C4E796F86010022913D003297F
:109D4000ECD1019B53F8282022F07042B2FA82F243
:109D50002B685209A2421FD0D8445B44D0452B60E7
:109D60001DD20229EDD1019B33F81820EEE74FF404
:109D7000807AD9E7D6F87412013A02EB41224902FF
:109D8000B2FBF1F21344B3FBFBF20BFB12320AB14C
:109D90005B449B1A2B60AEE79F42B0D8ADE709F158
:109DA00001094FF00008A6E7A03700242DE9F04F85
:109DB000DFF884918B4685B0174699F860C0096832
:109DC000BCF1020FD9F8645240F08280CEB24FF459
:109DD000807305EB1125A6EB010890449844B94225
:109DE00008F1FF38B8FBF3F84AD200F00103A844A9
:109DF0006FF0404A0193BCF1030F07EB0604A8EB98
:109E00000503284614BF4FF480728022641A03A908
:109E1000944228BF1446944228BF002E14BF01224A
:109E200000220A32FFF7FAFD01282AD199F860C012
:109E3000DBF800E0BCF1020F0EF1010324D0B442C4
:109E400055D9039806EB0A02011F00EB820201EBD1
:109E5000840142F8043F8A4203F10103F9D1DBF89F
:109E60000030A11B19448F42CBF8001002D1019B96
:109E7000002B48D18F4205F101054FF00006BAD8FA
:109E8000012005B0BDE8F08FB44246D903986FF0C9
:109E90000042811E324401EB440100EB420222F8F1
:109EA000023F914203F10103F9D1A11B71448F429A
:109EB000CBF80010DED1019B002BDBD086466FF083
:109EC00000434FF6FF72012023442EF81320D8E7F9
:109ED00001F07F06C1F3D413BCF1030FA6EB010818
:109EE0001D4414BF4FF480738023904476E7AEEB9B
:109EF000060E0EEB04018F42CBF80010BAD1019B85
:109F0000002BB7D003986FF040434FF0FF3223444B
:109F100040F82320DBF80010ACE7AEEB060E0EEBAA
:109F200004018F42CBF80010A4D1019B002BA1D0DB
:109F3000DDF80CE0C3E700BFA037002430B50446CD
:109F4000C06983B010B9012003B030BD0D460023B5
:109F5000032201A9FFF762FD0128F5D1B4F9202001
:109F6000002A19DB019B012D4FEA421103EB42123B
:109F700003D0022D1BD1E5205854A368D361237868
:109F8000032B04D10023137753779377D377636A36
:109F9000190C53839182D6E7064A92F8181209B930
:109FA00082F818020123022082F86130CCE7E368CE
:109FB000E4E700BFA03700242DE9F041044682B059
:109FC0000D4694F83C30042B7ED8DFE803F02B03D9
:109FD00069493A003D4E4FF6F777DFF8F48016E016
:109FE000BA425BD86DF04CFA01284FF0000134D131
:109FF000206BFFF727FE01282FD1019AD6F878129F
:10A00000531E22638B4228BF0B46C6F8783296F85F
:10A01000602001A9236B032A18469AB2E0D1434578
:10A02000E0D93BE06900204601F0FE01FFF786FF22
:10A0300001283FD1636B002B18BF022084F83C003D
:10A04000BFE794F82830042B02D1002384F828308D
:10A05000A36B0BB120469847012002B0BDE8F08108
:10A060001A4E0021E26AD6F8F83106F5EA70C6F811
:10A07000F8219B1AD6F8742202FB03F3D6F8DC21F0
:10A0800002EB4322C6F8DC21D6F8E02102EB4322A2
:10A09000C6F8E021FFF752FF01280BD10420CDE7DD
:10A0A000626B04F130010020FFF780FE012801D12E
:10A0B0000320C3E70228D0D194F82830042BCCD158
:10A0C000002384F82830C8E70220F5E7A0370024F1
:10A0D000F7FFFF0F38B5044694F83430052B60D8ED
:10A0E000DFE803F031251D130D0394F82830082B09
:10A0F0003FD02D4B0122022083F8192238BD94F85D
:10A100002830082B30D0012038BD00212046FFF731
:10A1100015FF012845D1042084F83400DCE7D4E998
:10A120000B01FFF78FFD01283BD10320F4E74FF02F
:10A13000FF31206BFFF786FD012832D1E36A002B47
:10A14000F3D00220E8E7184D04F130010120D5F8E2
:10A150006C220232FFF79CFD012813D00238C0B2F6
:10A1600001281ED80520D7E70023012084F82830D5
:10A17000CAE700230122022084F828300A4B83F822
:10A180001922BBE7E368D5F87412226B03EB412375
:10A19000C5F87822C4E90332E36A002BBCD16262BD
:10A1A000BAE7002038BD00BFA0370024F8B5044648
:10A1B00094F83830032B4CD8DFE803F021180B0259
:10A1C00000212046FFF7BAFE431EDBB2012B41D926
:10A1D000F8BD0120626B04F13001FFF7E7FD0128B3
:10A1E0004FF00303F0D184F83830E1E700211E4836
:10A1F000FFF7A4FE01284FF00203F4D0E4E71B4B65
:10A20000E66893F86020D3F87412032AD3F8DC517F
:10A21000D3F8F80114BF4FF480728022206102FB52
:10A2200001F1871A0244A5EB412506EB4126E660C1
:10A23000C3F8DC51D3F8E051C3F8F821A5EB412174
:10A24000C3F8E011E36AC4E90C025BB96062012360
:10A25000C9E7022094F82830062BB9D1002384F8EE
:10A260002830F8BD2763F2E774390024A0370024B2
:10A270004368C3F308020A44B2F5007F2DE9F041B8
:10A28000054682B00C4605D223446B60012002B023
:10A29000BDE8F08190F91A10481C0AD0474A02EB39
:10A2A000011292F88B1021F0010182F88B10FF222D
:10A2B000AA7695F91B20511C16D0404E023206EBAF
:10A2C000021191F86B10C1F34501012944D90139FC
:10A2D00001F03F0106EB0212FF2692F86B0061F3DA
:10A2E000460082F86B00EE762A78022ACCD0334EF4
:10A2F000D6F87422B4EB422F4FEA42282EDCD6F86F
:10A300007C721F407A42A24228DCE2192869424549
:10A3100013D32A7E12072DD5D6F8F821411C8A4284
:10A320001ED300D100214344A4EB0808686108460D
:10A33000DB1B08EB070429616B600028A6D096F8A8
:10A340006020032A35D080B24FF6F77290429DD834
:10A350001A4614446C6099E70021BBE7002096E799
:10A3600096F818220ABB012386F8183286F8613065
:10A370006B68D8E701A96DF083F80128EED16B680E
:10A38000A4EB080428699844297868613C44A8EB48
:10A390000703019802291A466B602861CDD1D6F8CF
:10A3A0008412B3EB412FD4D370E7012286F86120E9
:10A3B000B9E7034A90423FF669AFC9E7A0370024E6
:10A3C000F7FFFF0F2DE9F0474FF0010882B0044678
:10A3D00094F83830032B00F2A680DFE803F055171D
:10A3E0000C020020236C84F8280003B19847022057
:10A3F00002B0BDE8F0870022236C84F828200BB15E
:10A4000020469847012002B0BDE8F08723786768AE
:10A41000022B03D0454BD3F87C321F40C7F34F27A4
:10A420002046FFF7DDFA414E3F1A0546BFB207EB63
:10A43000050C022201A9002328461FFA8CF9FFF718
:10A44000EDFA01284FF400724FF00001D0D10198CD
:10A450007BF0A0FEE3694FF4007120460BB1636806
:10A46000EBB1D6F874325A1E914547D20135FFF749
:10A47000FFFE0028DBD196F8183213B9012386F8C5
:10A48000183286F86180D2E72046FFF723FE0128C4
:10A4900002D0022847D1032084F8380098E7019BB6
:10A4A0004FF020324FF0100E4FF02E0C42F62E6A75
:10A4B000C3F80120C3F80520A3F8092083F800C0E1
:10A4C000D4F824C0A3F820A083F80BE0C3F822201E
:10A4D000C3F8262083F82A20E26BA3F81AC02CFACE
:10A4E0000EFC5A8722FA0EF2A3F814C09A8683F85B
:10A4F0002BE0D6F874325A1E9145B7D3C3EBC35341
:10A500002046590201F50071FFF7B2FE28B996F80E
:10A51000183223B1012386F861300220BCE7012301
:10A5200086F81832F6E7002062E700BFA037002463
:10A53000B1F904300F2B2DE9F0410D4682B00446ED
:10A54000164632D02046FFF74BFA94F91B80B8F13B
:10A55000FF3F3BD05B4F07EB0813DB6F984212D0F5
:10A5600097F81832002B6ED0012387F861302378DA
:10A57000022B5ED02269002A73D1002301203360B0
:10A5800002B0BDE8F081B96F01EB4821002966D027
:10A59000AB88204601331BB201EB4311AB80316025
:10A5A000FFF71EFA28600120EAE74FF40071FFF779
:10A5B0005FFE002843D04FF6FF732046AB80FFF7C5
:10A5C0000FFA94F91B80B8F1FF3FC3D12378022B17
:10A5D0003DD02269002AD0D03A4F97F86030032B43
:10A5E00066D093B24FF6F7718B4294BF00230123DC
:10A5F000002BC0D130B997F81832002B4BD0012373
:10A6000087F861300023112201A9FFF707FA01281A
:10A6100025D10199BB6FCB1A48BF03F2FF13B3F5E5
:10A62000805F4FEA63222CD24FFA82F884F81B80B5
:10A63000ACE7D7F884226368B3EB422F9DD20020A9
:10A6400002B0BDE8F081012387F818328CE71D4F76
:10A650006368D7F88422B3EB422FCBD38DE72378FE
:10A6600086E797F86030032B19D093B24FF6F77254
:10A67000934294BF00230123002B7FF47EAF002080
:10A68000DEE797F8183213B9012387F8183201234F
:10A6900087F86130CAE7012387F81832AFE70A4B21
:10A6A0009A4294BF00230123002B7FF466AFE6E7B4
:10A6B000054B9A4294BF00230123002B7FF45BAF2C
:10A6C00098E700BFA0370024F7FFFF0F2DE9F04700
:10A6D000044688B094F83030042B11D8DFE803F03A
:10A6E000501361035A00237E9A0640F1F88000233C
:10A6F000112204A9E069FFF791F9012800F0EF8029
:10A7000008B0BDE8F087C44D03AE04F11C0705F5A1
:10A710000779324639464846FFF70AFF012800F01C
:10A72000F9800228ECD195F936325F1C0AD005EB8E
:10A730000313FF2193F88B2085F8361222F00102D3
:10A7400083F88B2095F937325E1C17D0023305EB66
:10A75000031292F86B20C2F34502012A40F25A819B
:10A76000013A02F03F0205EB031393F86B1062F31A
:10A770004601FF2283F86B1085F83722042306E098
:10A78000A6486DF013FC4FF6FF720123228484F873
:10A7900030309FE70020E36A207008B0BDE8F04742
:10A7A00018479D4D95F84432002BA9D104F11C07A0
:10A7B00005F5077803AE324639464046FFF7B8FE46
:10A7C000012840F01581039B002B00F0F0801A78DF
:10A7D0000AB1E52AEFD1AA6F9A1A48BF02F2FF1216
:10A7E000B2F5805F4FEA622180F0498109018C4A0D
:10A7F0000A44917B04290CD0D5F8FC100131C5F82E
:10A80000FC10516004219173D5F800210132C5F884
:10A81000002195F93622501C0AD005EB021292F85D
:10A820008B1021F0010182F88B10FF2285F836226F
:10A8300095F93722511C17D0023205EB021191F81D
:10A840006B10C1F34501012940F26181013901F02A
:10A850003F0105EB0212FF2085F8370292F86B00EA
:10A8600061F3460082F86B002022002118467BF03D
:10A8700091FCD4F831100346D4F8352005A81960AE
:10A880005A6094F83B20B4F839109A721981627EAC
:10A890000193DA7203F0C6F8019B002800F0D8801B
:10A8A0009DF816009DF817209DF8191042EA4012F5
:10A8B000BDF814004901A0F2BC7042EA40229DF8A4
:10A8C0001A0041EA50019DF8180092B241EAC021F5
:10A8D00088B2D9811A821A83D882032357E7204687
:10A8E0006DF064FB2369002B00F08780237E03F06A
:10A8F000F70213F00403227640F09480122A00F04D
:10A90000AA800022E36A204684F8282008B0BDE827
:10A91000F0471847DDF80C80B8F1000F00F0BB805D
:10A9200098F80030002B00F0B68098F80BA01AF0D1
:10A93000080F7FF4EEAE0B2204F1310140467AF0AD
:10A940007DFA00287FF4E5AE637E8AEA0303DF0622
:10A9500040F1E18095F936325E1C0AD005EB031315
:10A96000FF2193F88B2085F8361260F3000283F8FC
:10A970008B2095F93722511C3FF400AF023205EBD2
:10A98000021393F86B30C3F34503012B40F20681A9
:10A99000013B03F03F0305EB021292F86B1063F3E7
:10A9A0004601FF2382F86B1085F83732E6E695F80A
:10A9B0001C320922022B3FF4E1AE95F84432002B01
:10A9C0007FF4DCAE85F85432404685F8503285F885
:10A9D0004422C5E99633D5F83032C5F84832D5F867
:10A9E0007832C5F84C32FFF7EDFC01283FF4E3AEB6
:10A9F00002287FF485AE0423C9E6237E1B0780D599
:10AA0000054B93F8FC21002A7FF47AAE072283F8E5
:10AA1000FC2176E70022A6E6A0370024BC390024FA
:10AA20001C3800240023A5682046E66A294684F8DD
:10AA30002830FFF71DFC002863D194F82830002B44
:10AA40007FF45EAE0223C4E90B6584F8283057E634
:10AA500044F281723EE7E06A0421626AA063204604
:10AA600084F83C3084F8281063636362C4E90B22E5
:10AA7000C4E9023308B0BDE8F0476DF097BA95F825
:10AA8000182212B9012285F8182201226FF00F0155
:10AA900085F86120ABE695F93632591C0AD005EBF2
:10AAA0000313FF2193F88B2085F8361222F0010260
:10AAB00083F88B2095F937325A1C16D0023305EBF8
:10AAC000031292F86B20C2F34502012A21D9013A00
:10AAD00002F03F0205EB031393F86B1062F346019B
:10AAE000FF2283F86B1085F83722237EDB067FF583
:10AAF00045AE2C486DF05AFA4FF6FF7202232284BD
:10AB000045E6002E3FF4FCAD2046334645E60021E5
:10AB10009FE60022DEE7B8F81420B8F81A3043EABE
:10AB20000243D5F8742263625202D8F81C30B3FB9A
:10AB3000F2F102FB1131A36009B113445B1AE36027
:10AB400084F819A095F936325A1C0AD005EB031384
:10AB5000FF2193F88B2085F8361222F0010283F84A
:10AB60008B2095F93722531C3FF4B7AE023205EB28
:10AB7000021393F86B30C3F34503012B10D9013B4B
:10AB800003F03F0305EB021292F86B1063F34601EA
:10AB9000FF2382F86B1085F837329EE60023FAE631
:10ABA0000023EFE7BC39002410B50378044690F881
:10ABB00018C0023B012B02D91CF0060F6ED11CF00D
:10ABC000200F44D194F91A20511C0AD03A4BFF218E
:10ABD00003EB021393F88B2022F0010283F88B2001
:10ABE000A17694F91B305A1C16D03349023301EB7D
:10ABF000031292F86B20C2F34502012A4BD9013AA5
:10AC000002F03F0201EB031393F86B1062F346016D
:10AC1000FF2283F86B10E2761CF0080F0ED0264955
:10AC200091F8FC31072B06D091F81832002B3DD05B
:10AC3000012381F86130002381F8FC310023E26AAE
:10AC4000237084F8283042B3BDE8104010471B4AF7
:10AC50000023E069D1691032884206D00133082B05
:10AC6000B0D0D16910328842F8D11349023301EBD8
:10AC7000031292F86B20C2F34502012A1AD9013A55
:10AC800002F03F0201EB031393F86B1062F34601ED
:10AC900083F86B1096E70022B4E710BD0121FFF79F
:10ACA0004DF90128F9D194F818C088E7012381F8FB
:10ACB0001832BDE70022E5E7A03700240038002461
:10ACC00038B51A4C94F844322BB970B190F828205A
:10ACD0001AB1184638BD002038BD0146442204F59B
:10ACE00007707AF02FF9012038BD04F50775014689
:10ACF000442228467BF04EFA94F8603003224FF647
:10AD0000FF71022B2846A4F8361218BF1346D4F858
:10AD1000801284F83422102284F81C32C4F84012C5
:10AD200084F835226DF042F9DDE700BFA03700243A
:10AD3000304A4FF0FF31F8B5A2F1600C00230C4609
:10AD400003E001331032082B14D092F82A000428B3
:10AD5000F7D10CEB031090F88B00C607F1D4651CFB
:10AD6000106A01D08142ECD91C46013301461032F1
:10AD7000082BEAD1002C01DA0120F8BD1E4DA61CDB
:10AD800005EB0613D5F84826B3F86810D9B92701A2
:10AD90002F44A96FD5F84836F86F01EB4421D3B1A1
:10ADA000DC680023154AA047A8B1022809D1D5F8CC
:10ADB000003105EB06160122013B86F86A20C5F832
:10ADC00000310020F8BD05EB04132701D86F12B144
:10ADD00093689847DCE7D5F8003105EB06160321A8
:10ADE0000122013B86F86A1085F80421C5F800317C
:10ADF000E7E700BF00380024A037002459670408A3
:10AE00002DE9F04390F8283083B00446013B082B2D
:10AE10000BD8DFE803F0383C1F2305290A2E330046
:10AE20000121FFF7C9F8012802D003B0BDE8F08383
:10AE300000222378216C84F82820002BF5D00322EF
:10AE4000E162D4E9010384F82820834238BF034635
:10AE50002046A36003B0BDE8F043A5E6002103B09F
:10AE6000BDE8F043FFF7A8B803B0BDE8F043FFF733
:10AE70009DB903B0BDE8F043FFF72CB903B0BDE8BE
:10AE8000F043FFF79FBA03B0BDE8F0431EE4DFF8DC
:10AE900034914368D9F87C62026B19461E40D9F898
:10AEA000740294F800C0B5184702B5EB402F41D3A7
:10AEB0004FF6F778BCF1020F14D025692846002D13
:10AEC0005AD16168A3680020E26A8B4284F82800A6
:10AED00038BF0B46A360002AA7D0204603B0BDE8C8
:10AEE000F04310476168D9F88402B1EB402F5CD27F
:10AEF0002069217E090732D5D9F8F811451CA942ED
:10AF00002AD299F81812002943D1012389F818325E
:10AF100089F86130226B636894F800C0D21B3B440F
:10AF200032449B1B00269742194663602263C4E9A2
:10AF30000450BFD9BCF1020F37D02569002DC1D014
:10AF400099F86030032B36D0ADB24FF6F7739D42BF
:10AF5000B8D811446160B5E7E0D10025DEE701A96A
:10AF60006CF08EFA01287FF460AF2069019D94F89F
:10AF700000C06368226BD1E799F8601003290ED0F6
:10AF8000A9B2414594BF002101210029B1D06168D7
:10AF9000D4E7012189F8611094F800C0BEE70849A0
:10AFA0008D4294BF00210121EFE7D9F88432B1EB43
:10AFB000432FCED386E7024B9D4283D8C9E700BF1B
:10AFC000F7FFFF0FA0370024704700BF00797047DC
:10AFD0000079C0F34010704700794009704700BF06
:10AFE000704700BF704700BF03685A1C02601970A9
:10AFF000704700BF03685A1C02601970704700BF99
:10B00000024B186803681B68184700BF406400249F
:10B010002DE9F0413A4E33787E2B03D00027384695
:10B02000BDE8F08108214FF4FC4341F221041AB23B
:10B030005B00002A84EA42009BB2B8BF83B20139A8
:10B04000F5D1B6F80140002C37D02E4A2E4DAA4239
:10B05000E4D2052CA2F106028CBF0027012714447C
:10B06000AC4228BF47F00107002F46D141F2210E24
:10B07000A24214D0501E04F1FF3810F8011F08221C
:10B0800083EA012319B25B0000298EEA410C9BB2CE
:10B09000B8BF1FFA8CF3013AF4D14045EDD12188B5
:10B0A00061B1A21DAA42BAD2052904EB01002246D1
:10B0B000B5D9A842B3D20446DAE7144C671E41F270
:10B0C0002105BC4617F8012F83EA0223082219B292
:10B0D0005B00002985EA41009BB2B8BF83B2013A08
:10B0E000F5D16445EDD16788094AFF1A231DB7FAE7
:10B0F00087F79B1B7F09938091E70F468FE700BF7F
:10B10000000002080700020800000408010002080D
:10B110004064002490F83C20034602F0FF0012B186
:10B12000002283F83C2070474FF48053838170479E
:10B130004FF40063838170474FF40063838170474D
:10B140004FF40063838170474FF40063838170473D
:10B15000074B10B403F11001002453F8042B824272
:10B1600008BF43F8044C8B42F7D15DF8044B70479D
:10B170004864002470B5374CE08C238BB4F9305010
:10B180001B1AA08CB4F91EC000FB03F3B4F92E0007
:10B19000E66B05EBE335C00290FBF5F000EBE33026
:10B1A000B4F92A30A0F57A6E60630EFB0EF50EFB43
:10B1B0000CFC2D134FEAEC2C05FB03F30CEBE32CFA
:10B1C000B4F9283005FB03F3B4F920501B140EFB2F
:10B1D00005F503EB6533B4F91C5002330CEB850C19
:10B1E000B4F938509B10648C0CFA05FC03F500434D
:10B1F0000CF1020C04FB03F34CF25034A6EBAC0C44
:10B200002C41DB0B04FB0CF4002C1EDB6400B4FBB4
:10B21000F3F389B11C1240F6DE3504FB04F405FBA0
:10B2200004F40D4D241403FB05F504EB254404F64A
:10B23000CF6403EB24130B602AB100EB80004000C5
:10B24000083000111060012070BDB4FBF3F35B0007
:10B25000DFE700BF4064002443E3FFFF01207047A5
:10B26000012070472DE9F04F734D85B00F46286CD3
:10B27000B5F844300092C3EB2014B5F948205B00C8
:10B28000B5F950E004FB04F4B5F84A80C3EBE003E1
:10B29000CDF80CE02413B5F95260B5F9541002FB57
:10B2A00004F4B5F94620029602FB03F3A413B5F9A2
:10B2B0004C2004EBE3242B6EA4F5FA300193B5F98E
:10B2C0004E3080FB00EA4FEAE37B82FB002C03FB5D
:10B2D0000AF94FEA0C3CEC650EFB0B99A3FB0E3B05
:10B2E0004CEA125C1203CB441B0A43EA0B639B1823
:10B2F0004CEB2B2BA3FB08320BF5004B08FB0B2B65
:10B300004FEAEB734FEA6B0953EA6B0B00F0928044
:10B31000029E01FB0AFA019A86FB0008039EC2F511
:10B32000801C4A464FEA48484FEAE17948EAD0385B
:10B330000EFB09A94004A1FB0E1E4118F1444FF079
:10B3400000000CF0004E49EB08094EEA5C0E411873
:10B350004FEACC7C09EBC609BCEB010C6EEB090E85
:10B360001CEB0C084EEB0E0118EB0C084EEB010128
:10B370004FEA88104FEA811918EB000049EA9869F2
:10B3800041EB0901890041EA9071800010EB0C004B
:10B390004EEB0101890041EA9071800010EB0C0036
:10B3A0004EEB010173F04EF9B5F95A304FEA6138AE
:10B3B00084464FEA503EB5F956204FEAE37A03FB44
:10B3C00008F94EEAC14EB5F958000EFB0A99A3FBE5
:10B3D0000E35A94403FB08F50EFB0955A3FB0E3EF1
:10B3E00075445B0E4FEAE07E43EAC51313EB0C0392
:10B3F00041EB656500FB01F10EFB0C11A0FB0C0C91
:10B400006144C00C40EA41301B1845EBE1451B0A82
:10B4100043EA056303EB02130FB11B0A3B60009B79
:10B4200023B104EB8404803424121C60012005B095
:10B43000BDE8F08F0023EFE74064002431B10A4BF0
:10B44000D3ED207AFDEEE77AC1ED007A52B1064BDA
:10B450009FED067AD3ED217A67EE877AFDEEE77AE3
:10B46000C2ED007A01207047406400240000C84209
:10B470002DE9F04F5F4D934685B0B5F89630D5F87D
:10B4800088001B02B5F894E0B5F89240C21AB5F8EE
:10B490009030019167EB0707AEFB020C1B04B5F877
:10B4A0008E100EFB07CCC009B5F89860C90340EABE
:10B4B0004C604FEAEC1CC018A4FB023E04FB07EEF4
:10B4C0004FEA13234CF1000C43EA0E634FEA2E2E91
:10B4D0005B18A6FB021406FB07444FEAD1514EF15C
:10B4E000000E41EA4421E41511F5FA6844F1000622
:10B4F000B8F5FA6F029676F1000630DA01FB04F631
:10B500000394A1FB014A0AEB460AA6004FEA8A0906
:10B51000361949EA9479384C4AEB09094FEA560A38
:10B52000B6084AEAC97A46EA8976B0EB0A0A6CEBB1
:10B53000690C9E1B50466EEBA90E3346A045029E39
:10B540004FF0FF34A64126DB02FB07F7A2FB0221E6
:10B5500001EB4701D20F42EA4102B8EB0208019C1D
:10B5600084B1D5F89C10A1FB033201FB0E225B0DC8
:10B5700043EAC22352151B1A62EB0C02DB0B43EAAF
:10B5800042432360BBF1000F01D0CBF800800120C3
:10B5900005B0BDE8F08F40F6AC56039C891944F124
:10B5A000000401FB04F4A1FB016101EB4401F40080
:10B5B0004FEAC109341B49EA567961EB090924189D
:10B5C0004CEB090C2046B41941EB0109A41941EBDD
:10B5D00009094FEA890949EA9479A400A41B69EB97
:10B5E0000109610841EAC971591A6EEB690E0B46EF
:10B5F000AAE700BF4064002424FAFFFF012070473F
:10B60000104B10B4104C1B68D4F8A0001B1AFA2B76
:10B610000BD811B1D4F8AC300B6012B1D4F8B03003
:10B62000136001205DF8044B7047D4F8A430002269
:10B6300023F00403104684F8A820C4F8A4305DF871
:10B64000044B7047F0300024406400242DE9F84397
:10B650000D46D0E9003113448B4220D80446AE1881
:10B66000076BCAB14FF0000900F10C0801E0AE42CF
:10B6700012D0E36A5A1C2344E262202A15F8011B07
:10B680001973F4D14146204617B9F7F70BFD074669
:10B69000AE42C4E90B97ECD13846BDE8F8834FF0D1
:10B6A000FF37F9E72DE9F04F5422044600218BB013
:10B6B0009F487AF06FFD9F4A611EE01C144611F806
:10B6C000013F5D1E052D88BF0023884244F8043BDE
:10B6D000F5D102F11003114651F8040B012800F0D6
:10B6E00019818B42F8D1114651F8040B022800F061
:10B6F00007818B42F8D1114651F8040B032800F062
:10B70000F5808B42F8D152F8041B042900F0E48044
:10B710009342F8D105204FF01A094FF0000ADFF8E4
:10B720001082854DFFF714FD844F0620FFF710FDB2
:10B7300098F80C407CB3204698F90D6007F02CF87F
:10B7400028B1052380F80790837100230372032139
:10B7500006F0DEFF002302E001331C2B3DD015F87C
:10B760003320A242F8D105EBC3035868F421062325
:10B770000122C8F8100001FB067688F816309244C2
:10B78000D6F8F03088F8152086F8EC209A1888F85A
:10B790001430C6F8F02009F1010908F10C085FFA2D
:10B7A00089F9B9F1200FC3D1BAF1000F12D0DFF837
:10B7B0008CA14FF0000BDFF89C81D14699F8EC305A
:10B7C0006BB90BF1010B09F1F40908F58C78BBF1A9
:10B7D000030FF3D10BB0BDE8F08F0020C6E7B9F836
:10B7E00006006BF0A7FEB9F804006BF0A3FED9F8D1
:10B7F000F0304FF4403CF421012BC9F8283001FB14
:10B800000BA1D9F80020D4BF002301234FF0030E71
:10B81000C9F81020C9F81C300023C9F8383089F85D
:10B820002C30C9F83030C9F8203089F848300493FA
:10B830000823C9E905C34FF48063C9F834304FF4D5
:10B840008073A9F824304FF48053C9E90FE34B6E9D
:10B85000002B69D093689F0003D59168384B0B404B
:10B8600093609368DE0014D4364B37491B689068A8
:10B87000B3FBF1F335490133014041F08051916050
:10B880000493049B2BB1049B013B0493049B002B6A
:10B89000F9D19368DD001CD4F423012103FB0BA331
:10B8A0000191596E41F010015966996E41F0010104
:10B8B0009966F423916803FB0BA301F00401586E11
:10B8C00000F01000014347D05A6E42F010025A6651
:10B8D00077E700230193ECE71D4B342193F808210F
:10B8E00083F8E410013283F8082113E7184935245E
:10B8F00091F8080181F8D840013081F8080102E789
:10B900001349312491F8080181F8CC40013081F8C5
:10B910000801F0E60E49302491F8080181F8C04092
:10B92000013081F80801DEE68B6689F8603091E726
:10B93000F46400244864002400760C08E81800240D
:10B94000C0FFFF5F00000024400D0300C0FFFF6F39
:10B950004064002400000030596E21F4817141F0F0
:10B96000020159669368DC0713D4784B9A4200F0C1
:10B97000178303F580739A4200F01283744B9B681F
:10B98000D90706D473498B6823F47C1343F44033FE
:10B990008B60714B71491B68D368194043F20803EF
:10B9A0000B43D3609168936801F0040103F008032E
:10B9B000194300F06182D9F81000D9F81C30012B2E
:10B9C00000F05583036B23F00F030363F42303FBA1
:10B9D0000BA35A6E22F0030242F001025A66019A4A
:10B9E000002A7FF4EEAE019A059299F86020012AB0
:10B9F0003FF4E7AE82680121940789F860108168FE
:10BA000002D4CA0700F18882F421554A554B01FB44
:10BA10000BA14C6E224042F002024A66826813403B
:10BA200043F00043836083684F4A002BC0F2E581F6
:10BA3000F4214E4B4E4C4FF4806C01FB0BA14D4852
:10BA400003274D4D4A6E22F0030242F001024A667E
:10BA5000D9F80820D9F80C60A24218BF9A424FF4D6
:10BA60000054C9F878600CBF01230023C9F89C700A
:10BA7000824208BF43F001031830824208BF43F0FE
:10BA800001031830824208BF43F00103183082429C
:10BA900008BF43F001031830824208BF43F001039E
:10BAA0001830824208BF43F0010300F5567082420D
:10BAB00008BF43F001031830824208BF43F001037E
:10BAC0001830824208BF43F001031830824208BF99
:10BAD00043F001031830824208BF43F001031830DD
:10BAE000824208BF43F001031830824208BF43F08E
:10BAF0000103002089F86000C9F89800C9E91F0017
:10BB0000C9E928004FF40060C9E921C04FF48070F2
:10BB1000C9E923404FF400304C46C9F89400286826
:10BB200044F8742F1BB9154B9A4240F0BE84F4239D
:10BB3000022103FB0BA383F8A9100021136889F8E5
:10BB4000A81023F0010313601FE000BF0020024093
:10BB500000600258006302580010005C03C0F0FF50
:10BB6000FDEEFFFFC0FFFE3F00F8C32510000240BE
:10BB70002800024040000240002E0024B804024089
:10BB80002B681B1A052B00F2BD811368DF07F7D461
:10BB9000A44913680868A4496FF30F001940A34B28
:10BBA000B0F1005F43EA01030BD32E2E40F21F8356
:10BBB0003F3E132E05D89E48F040C00701D59D4B4F
:10BBC0000B4313602046536923F007035361F5F7D5
:10BBD00021FFD9F8D02002F01F013F228A40826065
:10BBE000D9F87420944B9549954E8A4218BF9A42D1
:10BBF00001F11801A2EB06000CBF012300238A42C9
:10BC000008BF43F0010318318A4208BF43F0010323
:10BC100018318A4208BF43F0010318318A4208BF35
:10BC200043F0010318318A4208BF43F00103183181
:10BC30008A4208BF43F0010301F556718A4208BFEA
:10BC400043F0010318318A4208BF43F00103183161
:10BC50008A4208BF43F0010318318A4208BF43F00B
:10BC6000010318318A4208BF43F0010318318A42A8
:10BC700008BF43F0010318318A4208BF43F00103B3
:10BC80007049511AD1F1000C4CEB010C6E498A42FB
:10BC900008BF43F001036D494642A2EB010701F1E1
:10BCA000140146414CEA0303D7F1000EA2EB010058
:10BCB00043EA06034EEB070E41424EEA03034141BD
:10BCC00063480B4302916349571A794279410B4308
:10BCD0000391111A484248415F49571A0343794278
:10BCE00079415E4FBA4214BF002701270B4301D1AF
:10BCF000002F3BD046EA0C06029B4EEA060E039E3E
:10BD000043EA0E031E43D3B230430143394300F0EC
:10BD10005D831422083B0126514FB3FBF2F3514AD5
:10BD20009E401A449200D9F87C30C9F8DC60802B20
:10BD3000C9E9352700F00881D9F87830D8B2013B3D
:10BD4000072B10607E6000F20481461E002900F07F
:10BD50006885454B454903449B0001220020B240C1
:10BD6000C9E93831C9F8E82018604A60F423012194
:10BD700000204FFA8BFE03FB0BA30A460295C3F883
:10BD8000C80083F8A91009F11003C9F85C40C9F88C
:10BD9000AC30374B04E001320C33072A00F00A8143
:10BDA000597D0029F7D093F90D107145F3D1002189
:10BDB00001989D7D06912F49039501EB800118693B
:10BDC000D1F8E04099F8601001293FF4FAAC4FF047
:10BDD000010189F86010D9F810108D686F0740F1E3
:10BDE0000F81F42303FB0BA35A6E42F020025A6624
:10BDF0004FF0000389F86030E3E4059B01330593BD
:10BE0000059B9342FFF40FAEF422002102FB0BA22C
:10BE1000536E23F0120343F01003536689F8601049
:10BE2000CFE400BF0010005C3F8010FE002D020038
:10BE30000F030F00002D12001000024028000240E6
:10BE40001C54025808540258B80402403054025896
:10BE50006C54025858540258805402589454025852
:10BE600080580258009600163F9600164059025816
:10BE7000F464002400760C08D068AA4B0340D9F87B
:10BE8000440043F00303D360136923F001031361FB
:10BE9000136923F0704303431361A34B9A4277D095
:10BEA00003F580739A4273D0A04B9B6813F4403F14
:10BEB00014BF01230023002B00F0EA80F5F712FFE6
:10BEC000D9F814300146B3F5003F00F01E82B3F5F7
:10BED000403F00F01E82B3F5803F00F01682944B85
:10BEE000D9F810001A6841F20303B3EB124FC0F007
:10BEF000C780904B9942836800F20F8123F48073CE
:10BF000083605AE5F423202203FB0BA3C3F8C82067
:10BF1000032283F8A92054E4826802F00D02012A6A
:10BF20001DD05A6E002142F010025A669A6E42F0FD
:10BF300001029A66F42303FB0BA35A6E42F010022F
:10BF40005A6689F860103CE40023C9F87830136021
:10BF50007E600023C9E93833C9F8E83006E7826813
:10BF6000754B764D134043F0020383600323036057
:10BF70002A688368DE077FF547AD2B689B1A022B82
:10BF8000F7D98368DF07F4D5F42303FB0BA3C8E7D5
:10BF90006B4B9B6813F4403F14BF012300238AE7D7
:10BFA000614B68499B6889680B43D8073FF5F1AC42
:10BFB0006349E8E4D9F810105B4B029D9942D9F827
:10BFC000F07052D003F5807399424ED05748826882
:10BFD0008B685E073FF5F5AB99F86030012B3FF4B5
:10BFE000F0AB02F01F0240F221230124D34089F874
:10BFF0006040234040F0FF8089F86030FFF7E1BBEC
:10C0000000284FEA906709DBC0F31305002D40F0CC
:10C01000E6800125BD40CE692E43CE61A50901F120
:10C02000300604F01F0407F01F0705F00C054FF061
:10C030001F0CA7400CFA04FC745924EA0C043C437E
:10C0400074518D688C6805F0040504F008042C43D5
:10C0500000F082808C68E60732D501990131C9B2BF
:10C060000191002189F8601095E63548AFE7026B31
:10C07000D9F8283022F00F02013B13430363A5E4F3
:10C08000314B994242D8836823F44073836094E42F
:10C090002E4B9A6D02F44032B2F5803F00F0888159
:10C0A000B2F5003F00F06981002A7FF418AF1B68E9
:10C0B0001A017FF514AF07A8F5F752FE07990EE7AE
:10C0C000D1F8C040C0F31305002824EA0504C1F8E4
:10C0D000C040C2DA144CA14200F01D8104F5807406
:10C0E000A14200F01881114C194EA568B668F607F8
:10C0F00040F11B81F423002103FB0BA35A6E42F095
:10C1000020025A6689F86010FFF75BBB114B994219
:10C1100000F22881836823F4407343F480738360C2
:10C120004BE400BFFCBFFFFF002002400063025849
:10C130000010005C002D3101C0FFFF7F002E0024A5
:10C14000002302400021024021BCBE0000440258EE
:10C150000060025841787D01C0F30454039FC50D6F
:10C1600001F1140607FA04FC072705F00405A740AF
:10C17000745924EA070444EA0C0474519F4C24685F
:10C1800004F07044B4F1805FCC6800D0CC680C6ED1
:10C19000850604F0F844B4EB806F03D10C6E24F0F4
:10C1A00000440C664C6E04F0F844A54203D14C6E7A
:10C1B00024F000444C668C6E04F0F844A54203D190
:10C1C0008C6E24F000448C66CC6E04F0F844A542DA
:10C1D0007FF440AFCC6E24F00044CC663AE790FA8E
:10C1E000A0F50126B5FA85F506FA05F513E7282E20
:10C1F0007FF6E7ACE3E48B68DC0733D48C68804BD4
:10C200001C421FD18C687F4B234043F001038B609D
:10C210002C688368DB0602D07B4B994222D0794898
:10C220000B68DE071ED48B68DE0704D48B680340DE
:10C2300043F001038B602B681B1B022BF0D90B68AA
:10C24000DB07EDD4F42303FB0BA35A6E42F010027C
:10C250005A669A6E42F001029A66002389F86030AD
:10C26000FFF7AFBAF420694B00FB0BA0446E2340EC
:10C2700043F48073436612B1634B994206D0F423B2
:10C2800003FB0BA35A6E22F480125A66F42303FBBD
:10C290000BA35A6E12F4805200F0A8809A6E22F01E
:10C2A00006029A66D9F85C000024594BD9F83C2064
:10C2B000C363584B0364584BC3641C230B604B6827
:10C2C00089F8604043F010034B60CB6823F0030310
:10C2D0001343CB6090F83430012B0CD0012380F84D
:10C2E000343090F83530012B00F02C814FF400638E
:10C2F00080F834404365D9F81020424B91680B40D8
:10C3000043F004039360FFF75CBA1B0CB1FBF3F13D
:10C31000E5E58108E3E5414C414E3B4FA568B66831
:10C32000BF683E43F7073FF5E5AE3E4F05F0E076C8
:10C33000B84200F08D803C4FB84200F0A7803B4FE0
:10C34000B8427FF48AAE6F023FF587AE384881422B
:10C350007FF483AEA16821F0E071314341F48001A4
:10C36000A1607AE6334B994283682AD823F440735C
:10C3700043F400738360FFF720BBDA6C186802F0A7
:10C380004052470701D5002A32D02B4B1B68DE05EF
:10C3900003D5B2F1805F00F0D380274B1B689D036B
:10C3A0007FF59DAD254BB2F1005F08BF194696E5BC
:10C3B0001B689B007FF593AD07A8F5F76BFD099906
:10C3C0008DE543F440738360FFF7F7BA1C48103BD8
:10C3D00010441822A828B3FBF2F300D80833194AF6
:10C3E0000126194F1A449E4092009CE49A6659E730
:10C3F0001B681649C3F3C103D94070E50010005C07
:10C400003F000080C0FFFF7F00210240FEF0FFFFE1
:10C4100001000408550004085900040800230240E4
:10C4200000200240000084CB000052C70000B8CFBB
:10C430000060025881F0FA020044025840787D0101
:10C44000F0FBFDBF00820010800802400090D00386
:10C450002D023FF502AE9F4881427FF4FEAD9E491A
:10C460009E480968B1FBF0F1A068013120F0E0704E
:10C470004900304340F40000A060069102E00699B4
:10C480000139069106990029F9D1E6E5E8013FF561
:10C49000E4AD904881427FF4E0ADA16821F0E07105
:10C4A000314341F08071A160D7E58D4B8D488242C8
:10C4B00018BF9A4200F114000CBF012300238242EE
:10C4C00008BF43F001031430824208BF43F0010368
:10C4D0001430824208BF43F001031430824208BF87
:10C4E00043F001031430824208BF43F001031BB93B
:10C4F0007D4B9A4240F09B81F42102207B4B01FB53
:10C500000BA1134481F8A9001421B3FBF1F383407C
:10C51000106842F2A0516FF310100143002089F817
:10C52000A80020461160C9F8D030F5F773FAD9F8A1
:10C53000D02002F01F0101228A404260FFF750BB69
:10C540006B49CCE4036840316A4A6B4DAB4218BF7B
:10C55000934205F118050CBF01220022AB4208BF2F
:10C5600042F001021835AB4208BF42F00102183513
:10C57000AB4208BF42F001021835AB4208BF42F09F
:10C58000010205F55675AB4208BF42F001021835AD
:10C59000AB4208BF42F001021835AB4208BF42F07F
:10C5A00001021835AB4208BF42F001021835AB4218
:10C5B00008BF42F001021835AB4208BF42F0010249
:10C5C0001835AB4208BF42F001021835AB4208BF34
:10C5D00042F00102142505FB07F7022580F83550CB
:10C5E000464D4465464CAB4218BFA342856D0CBF17
:10C5F0000124002401950AB9002C37D01D6825F0CC
:10C600000105D0E919EC1D60C56E002C40F0FF80DB
:10C61000456EC5F804C0C56E002D75D0D0E91C5616
:10C620006E60002C70D0C56D019E05F01F0C3F257B
:10C6300005FA0CF5B5601D6825F480251D60856838
:10C640005F60402D00F0DF809960C3F80C8014B962
:10C65000002A00F09580196821F01E0141F01601B2
:10C660001960196841F008011960B9E01C4DDFF844
:10C6700074C0634518BFAB420CF1140C0CBF01250C
:10C680000025634508BF45F001050CF1140C634516
:10C6900008BF45F001050CF1140C634508BF45F0D7
:10C6A00001050CF1140C634508BF45F00105D3F8F2
:10C6B00000C02CF0010CC3F800C0DFF848C063458F
:10C6C00008BF45F0010515B9074DAB4258D1D0F868
:10C6D00068C09DE70060025800000024400D030080
:10C6E000085402581C54025894540258F8ABFDA741
:10C6F00000093D004000024058000240280002406E
:10C700001000024080540258002A8CD14B4DDFF8B3
:10C7100034C1634518BFAB420CF1140C0CBF0125AA
:10C720000025634508BF45F001050CF1140C634575
:10C7300008BF45F001050CF1140C634508BF45F036
:10C7400001050CF1140C634508BF45F001050CF11F
:10C75000140C634508BF45F0010515B9384DAB42CF
:10C760000ED1C56D019E05F01F0C012505FA0CF5D3
:10C77000756085685F60402D4FD09960C3F80C806C
:10C7800030492E4DAB4218BF8B4205F128050CBF36
:10C7900001210021AB4208BF41F001011D6825F0D5
:10C7A0000E0545F00A051D60274DAB4208BF41F05C
:10C7B00001011435AB4208BF41F001011435AB4211
:10C7C00008BF41F001011D6845F004051D601F4DC3
:10C7D000AB4208BF41F0010111B919498B420DD19B
:10C7E000016E0D68EA0303D50D6845F480750D6090
:10C7F000C16E19B1086840F4807008601A6842F090
:10C8000001021A6077E5C3F80880D9601FE7CEF807
:10C8100004C0002D7FF402AF05E7C3F80880D9609B
:10C82000AEE70B4B0B4903449B00FFF796BA40233E
:10C83000C1F8C83081F8A970FEF7C3BF0854025888
:10C84000945402581C5402584454025880540258BC
:10C850003F8200104009024038B51446002944D0F8
:10C86000344B0D469FED344A93ED437AD3ED466A3F
:10C87000B8EEC76AB3F92821B8EEE60AD3ED447AD8
:10C8800004EE902AB3F92421C6EE046A93ED477AA8
:10C8900005EE902AB3F9262105EE102AB3F92221DC
:10C8A000B3F92031F8EEE44A06EE102AF8EEE55A24
:10C8B000F8EEE77AB8EEC55AB8EEC77AC7EE843A12
:10C8C00007EE903AB8EEC66AE6EEA45AF8EEE77ABA
:10C8D000A6EE856AA6EEA57AE6EE867AA6EE870A29
:10C8E000A3EEA70A74F0D0FB28600CB3114BF6EE50
:10C8F000005A9FED115AD3ED446AB3F91621F8EEB0
:10C90000E66AB3F9143107EE102A9FED0C6A07EEC0
:10C91000903A86EE850AB8EEC77AF8EEE77A20EE0E
:10C92000070AA7EEA50A20EE060A74F0ADFB206008
:10C93000012038BD406400240000F04A0000C842D5
:10C940000369416853EA0102F0B43B4E5DD0C56A09
:10C95000013390ED067A6A1C876830EE077A03612E
:10C96000012AC26280ED067A42D090ED075A07EEA6
:10C97000902AD0ED096A70EE455A3468B8EEE76A3D
:10C98000611AC5EE867AB94277EE857A30EE670A8B
:10C99000C0ED087AC0ED077AF0EE667AE5EE807AAF
:10C9A000C0ED0A7AC0ED097A01D8F0BC7047012ABF
:10C9B00028DD06EE905AF8EEE66A87EEA66AB5EE36
:10C9C000C06AF1EE10FA1DDBF1EEC67AF4EE677A7A
:10C9D000F1EE10FA16D6D0ED056AF4EEE76AF1EE44
:10C9E00010FA15D5037BFBB10323F0BC037070472D
:10C9F000326880ED080A521A002180ED070ABA4217
:10CA00004162D2D9DFED0D7AE5E7316841609EE7FA
:10CA100007EE903A0223F8EE677A0370F0BCC7EE97
:10CA2000276AC0ED066A7047316800220361C3625D
:10CA300041608261B9E700BFF030002400000000CF
:10CA400010B5DFED4F4A844600F1480E0346DA6A1E
:10CA5000B1EC017AD3ED067A013277EE877A012ABA
:10CA6000DA62C3ED067A71D093ED075A07EE902A89
:10CA700093ED096A77EE455AF8EEE77AC5EEA76AB4
:10CA800076EE857AF0EE466A37EE677AC3ED087A7D
:10CA9000E5EE876AC3ED0A6AC3ED077A1833C3ED82
:10CAA000036A7345D3D1374C416822680369521A2F
:10CAB000816801338A42036147D990ED056A0022FB
:10CAC000DFED2F5ADCF82C10F0EE657ADCED0A6A07
:10CAD000012901F1FF3E11DD07EE90EAF8EEE77A59
:10CAE00086EEA77AB5EEC07AF1EE10FA45DBF1EEEC
:10CAF000C77AF4EE677AF1EE10FA3ED6B4EEE76A42
:10CB000001320CF1180CF1EE10FA26D4022AD9DD0C
:10CB1000B4EEE76AF1EE10FA1FD407EE903AD0EDCA
:10CB2000066A90ED0C7A0223F8EE677AD0ED125A7D
:10CB3000037086EEA76AC7EE276A85EEA77A80EDB6
:10CB4000066AC0ED0C6A80ED127A10BDF0EE477AED
:10CB500083ED087AF0EE646A9EE7037B13B103234A
:10CB6000037010BD002221680361C36241608261CD
:10CB7000026343648264C36510BDDFED017ABDE7E3
:10CB800000000000F0300024B0EEC06AF0EEE05A81
:10CB9000F0EE407AF4EEC65AF1EE10FA0EDCB5EE85
:10CBA000400AF1EE10FA4AD0F4EEC65AF0EE466AA8
:10CBB000F1EE10FA4FD5B0EE655A03E0F0EE656A7B
:10CBC000B0EE465A85EE267A9FED242A9FED243A50
:10CBD0009FED244ADFED244ADFED242ADFED243ADD
:10CBE000B7EE005ADFED236AF4EEC65AF1EE10FA02
:10CBF000A7EE023AE7EE223AA7EE034AA7EE235A3F
:10CC0000E7EE044AE7EE246AB1EE667A87EE050A9B
:10CC100010D4F5EEC00AF1EE10FA03D59FED167AA6
:10CC200037EE400AF5EEC07AF1EE10FA48BFB1EEE9
:10CC3000400A70479FED117A37EE400AE9E7F5EEBA
:10CC4000C00ADFED0F7A9FED0F0AF1EE10FA58BF20
:10CC5000B0EE670A7047B0EE465AB3E739094E3D69
:10CC6000E3B59EBE88FA16BE45FE7FBF99FB243F02
:10CC700069A2163EA7DFA8B4DB0F4940DB0FC93F0E
:10CC8000A7DFA834DA0F4940D1ED007AF7EE002A89
:10CC9000D0ED043A90ED054AE7EEA73AD0ED064A0A
:10CCA00090ED075AD0ED085A90ED096AD0ED0A6A66
:10CCB00090ED0B7AC0ED043A91ED003AD1ED013AD6
:10CCC000D0ED0C7AA3EE234A80ED054AD1ED003A6F
:10CCD00091ED024AE3EE844AC0ED064AD1ED004AE6
:10CCE00035EE245A80ED075AD1ED014A91ED005AF4
:10CCF000E4EE855AC0ED085AD1ED015AA5EEA56AB9
:10CD000080ED096AD1ED015A91ED026AE5EE866A7D
:10CD1000C0ED0A6AD1ED016A37EE267A80ED0B7A12
:10CD2000D1ED026A91ED007AE6EE877AC0ED0C7AD9
:10CD300091ED027AD1ED017A90ED0D3AD0ED0E3AF7
:10CD4000A7EE273A90ED0F4AD0ED104A90ED115A18
:10CD5000D0ED127AD0ED135A90ED006A80ED0D3AC5
:10CD600075EEA25A91ED023AD0ED016AE3EE033A74
:10CD700090ED027AC0ED0E3AD1ED023A34EE234A3C
:10CD800080ED0F4A91ED004A74EE844AC0ED104ADE
:10CD9000D1ED014A35EE245A80ED115A91ED025A37
:10CDA000C0ED135A77EE857AC0ED127AD1ED017A93
:10CDB000D1ED005A67EEA77A91ED025AE5EEA57A19
:10CDC000E5EE057AA5EEA76A80ED006A91ED016AAD
:10CDD000E6EE276AC0ED016AD1ED026AA6EEA77AF7
:10CDE00080ED027A90ED037A77EE277AC0ED037A30
:10CDF000704700BF2DE9F04F4FF00009864600F163
:10CE000010050646034689B000F13008074648463B
:10CE10002C468B469C46B246CDF80CE000283CD10F
:10CE20000CF1040CA445FBD1032800F1010151D001
:10CE30009C46AA46029398B1DCED047AAAEB09035A
:10CE4000B64601927246F3EC016A0EF1100E92EDB5
:10CE5000007A5345E6EEC77ACCED047AF2D1019A16
:10CE6000DCED046A0CF1100C15ED047A0AF1100ADD
:10CE7000C445C6EE877ACCED007ADCD1029B04363D
:10CE8000084608F10408143314351034103709F13A
:10CE900004099C46B2460028C2D0DCED007AD64692
:10CEA000394601927246F1EC016A0EF1100E92EDD4
:10CEB000007A9942E6EEC77ACCED007AF2D10CF115
:10CEC000040C019A0AF1040AA445E6D1032800F1F2
:10CED0000101ADD1DDF80CE00023594604AD7646E2
:10CEE000774600200493059306930793F2EC017AAA
:10CEF000E5EC017AB0B104AC3B46B4EC017AF3EC5A
:10CF0000016AE6EEC77AB34245ED017AF5D1013008
:10CF100004280BD0F2EC017A10371436E5EC017AD4
:10CF20000028E8D1103714360120DFE708AD1031B2
:10CF30000EF1400E042875ED017AA1F10402744649
:10CF400041ED017A1ED07346F3EC016AB1EC017A2F
:10CF5000A342E6EEC77AC2ED007AF5D15EED016A32
:10CF6000013887EEA67A82ED007A17D0AEF1140E62
:10CF7000103C114675ED017A0428A1F1040241ED3F
:10CF8000017AE0D15EED016A103CAEF1140E03208F
:10CF900087EEA67A01ED017A1146EBE709B0BDE80C
:10CFA000F08F00BF60EEA00AE0EE000AF5EEC00AC6
:10CFB000F1EE10FA07DBB1EEE00AB4EE400AF1EE52
:10CFC00010FA00D670479FED010AFBE70000000051
:10CFD00060EEA00AE0EE000AE1EE010AF5EEC00AFA
:10CFE000F1EE10FA07DBB1EEE00AB4EE400AF1EE22
:10CFF00010FA00D670479FED010AFBE70000000021
:10D00000DFED297AB4EEE70AF1EE10FA28DD9FEDA4
:10D01000277A30EE470AB4EEE70AF1EE10FAF8DCB0
:10D02000DFED237AB4EEE70AF1EE10FA2FDD30EEF1
:10D03000670A37EEC00A60EE007ADFED1E5A9FEDF8
:10D040001E6ADFED1E6AA7EEA56A9FED1D7A60EEEF
:10D05000275AE7EE866AA7EEA67AA5EE870A7047FA
:10D06000DFED187AB4EEE70AF1EE10FAD8D59FEDAD
:10D070000F7A30EE070AB4EEE70AF1EE10FAF8D4B0
:10D08000DFED0B7AB4EEE70AF1EE10FACFDC9FED9C
:10D090000E7AB4EEC70AF1EE10FACCD530EE270ABC
:10D0A00037EE400AC7E700BFDB0F4940DB0FC9403E
:10D0B000DB0FC93F9A7C2E36FAAF4FB93587083C53
:10D0C000A4AA2ABEDB0F49C0DB0FC9BF10B5404C74
:10D0D000B4FBF2F4A14219D3DFED3E7AF7EE005A29
:10D0E000B0EE677AB0EE676AF0EE676A0023C0EDD3
:10D0F000005AC0ED017A80ED027A80ED036AC0ED3E
:10D10000046A836143610362C36110BD07EE902A24
:10D11000DFED315AB7EE006ADFED306AB8EE677ABC
:10D1200007EE901AB0EE405AF8EE677A27EE257AAD
:10D1300067EEA67AC6EE076AC7EEA64AFDEEE47A67
:10D1400017EE902A2032402A3FD8B0EE640AFFF74B
:10D1500057FFB0EE404ADFED227A34EEA70AFDEE2B
:10D16000C07A17EE902A2032402A29D8FFF748FFCC
:10D17000F8EE006A60EE266A012B1CD0B7EE006A5A
:10D18000F6EE004A36EE406A66EE244A35EE055A5F
:10D19000F7EE007A84EE057A77EE275A37EEC75A13
:10D1A00084EEA57AC6EE257A86EEA56AC5EE256AD6
:10D1B000F0EE475A9AE7F7EE004AB0EE666AE5E706
:10D1C000DFED086A9FED030AD6E79FED024AC2E74A
:10D1D00020A1070000000000BD378635DB0FC940E5
:10D1E000DB0FC93F00000080DFED077A30EE270A31
:10D1F000FDEEC07A17EE903A2033402B00D8FFE6C0
:10D200009FED020A704700BFDB0FC93F000000001E
:10D210002DE9F84F9DF828408946DDF82CB00546E9
:10D22000002C17461BF8011B0CBF4FF020084FF0D5
:10D2300030081C1E08463ADB00295CD0002C53D075
:10D240004FF0000A5B4600E064B313F8016B013C49
:10D25000002EF9D1BAF1000F2FD1264644B14D4529
:10D260004146284600D2B847013CF8D10B9B1878BC
:10D270000146A0B14FF0FF344FF0000A00E09B469A
:10D280004D45284600D2B8475B4613F8011B0029DC
:10D29000F5D10B9BF61A5E44BAF1000F10D130465F
:10D2A000BDE8F88FBAF1000F1BD15646E0E76342A4
:10D2B00029B31C464FF0010AC4E70028E0D1064616
:10D2C000002C04F1FF3AEADD54464D45414628461C
:10D2D00000D2B847013CF8D2013656443046BDE88A
:10D2E000F88F30B12646CBE726464FF0FF34B246E2
:10D2F000C6E70646D3E72646002CB0D1CFE76FEA53
:10D30000040A0E46E0E700BF0FB430B583B00B4C03
:10D3100006AB53F8042BD4E94B01019370F020F9CC
:10D320000546206803685B6998470028F9D02846BD
:10D3300003B0BDE8304004B0704700BF4064002433
:10D340000EB410B583B00446084905AB01A853F8E4
:10D35000042BCDE9003470F003F90022019B1A7010
:10D3600003B0BDE8104003B0704700BFF5AF04083C
:10D370000CB4F0B53C4CADF5277DD4F83431002B1E
:10D380006DD094F83C3199420BD90123D4F8402157
:10D390008340134205D10DF5277DBDE8F04002B072
:10D3A0007047324B4FF47A71314A1B68A2FB03027B
:10D3B00006A8920901FB12332E49FFF7C1FF06AB05
:10D3C000AC9A064603442C4901A80193ADAB0093E7
:10D3D00070F0C6F8019B0A2100225D1C01951970AE
:10D3E000019BD4F83451591C01911A70ADB12B68CE
:10D3F0005B6A1BB128469847D4F834519DF8181041
:10D400000029C8D00DF119042B6828461B689847DD
:10D4100014F8011B0029F7D1BDE7D4F83871002FAB
:10D42000B9D0304426ABFD2206A9841C1846ADF8BD
:10D4300010202246CDF81250ADF8165077F082FD3C
:10D4400002220346044402A93846CDE9023433F0EF
:10D450009BFF0DF5277DBDE8F04002B07047D4F882
:10D460003831002B8DD196E740640024F030002441
:10D47000D34D6210441D0D08E9AF040838B5184CAF
:10D480000330D4F8442102EB9003B3F5007F18D8A1
:10D4900004EB810104F5A47520F00300C4F84431C5
:10D4A00005EB8205D1F84829C3F5007310440D4AF5
:10D4B0009B00C1F8480904210020FFF759FF2846C6
:10D4C00038BD0021084A00250846FFF751FFD4F86F
:10D4D000D039284643F00073C4F8D03938BD00BFB6
:10D4E00040640024501D0D08741D0D0838B50568F2
:10D4F0000446EB69F3B1987800B938BDB3F90A2056
:10D50000012007EE902AF8EEE77AC4ED057AB3F928
:10D510000C2007EE902AF8EEE77AF1EE677AC4ED78
:10D52000047AB3F90E3007EE903AF8EEE77AC4EDDC
:10D53000067A38BD09211420FFF7A0FF0346E861F1
:10D54000D9E700BF38B505680446EB69E3B19878C0
:10D5500000B938BDB3F90420012007EE902AF8EE97
:10D56000E77AC4ED047AB3F9062007EE902AF8EEC4
:10D57000E77AC4ED057AB3F9083007EE903AF8EE91
:10D58000E77AC4ED067A38BD09211420FFF776FF4B
:10D590000346E861DBE700BF38B505680446EB6980
:10D5A000E3B1987800B938BD9A880120D2BA07EE65
:10D5B000902AF8EEE77AC4ED047ADA88D2BA07EE58
:10D5C000902AF8EEE77AC4ED057A1B89DBBA07EEFC
:10D5D000903AF8EEE77AC4ED067A38BD09211420B6
:10D5E000FFF74CFF0346E861DBE700BF38B505688D
:10D5F0000C46EB697BB1987800B938BD5B89012096
:10D60000084ADBBA82FB0312DB17C3EB221303F2D7
:10D610006D13238038BD09211420FFF72FFF034627
:10D62000E861E8E7797878782DE9F04103EB430683
:10D63000964686B0034602EB4606754612F9067B0F
:10D64000A3EB070C92F80080BCF1000FA3EB0804D9
:10D65000B8BFCCF1000C002CB8BF6442644502DABC
:10D6600015464FFA88F70632B242E9D1688803E0DE
:10D670000EF1060E764518D09EF800208446BA4278
:10D68000F6D10A1ABEF80280002AA1EB0804B8BF3E
:10D690005242002CB8BF64429442E9DA75460EF15A
:10D6A000060E4046C4467645E6D16879CDF808C0F6
:10D6B0002A78049028790192039001200091032197
:10D6C000034AFFF755FE284606B0BDE8F08100BFCB
:10D6D000841D0D0803685A1C02601878704700BF4B
:10D6E00003681A46591C016012F8021B0260587840
:10D6F00041EA0020704700BF02681346511C0160D8
:10D7000013F802CB0360D31C5178036093781B0499
:10D7100043EA0123111D43EA0C030160D07843EA78
:10D720000060704712B370B50446864604E0981B4B
:10D7300017D114EB0C0C15D01EF8013BA3F14100DE
:10D74000A2EB0E0C192811F8010BA0F1410598BFAE
:10D75000203300F12006192DE9D91B1A04D1002825
:10D76000E7D170BD604670BD184670BD1046704769
:10D77000038800211A4A30B503F0030E90F802C066
:10D78000184CA3F5FA630EEB4E0E0CF1FF3C40F281
:10D79000B5550CEB8E0C04EB4C044FEA930CB4F82B
:10D7A0002031847905FB0C3390F803C022444FF4F8
:10D7B0007A740CF1FF3C634490F804C003EB43031C
:10D7C0000CEBC30C43790089CCEB0C1C03EB8C03F2
:10D7D000C3EB031302EB8302C2FB040130BD00BFA5
:10D7E00080436D3800760C08F8B516461F46404D4C
:10D7F0000446394630464FF47A72002370F022FF17
:10D800003C4B05443C4F3D4E83FB0510E917284433
:10D81000C1EB601183FB0103C8170B44C0EB63101D
:10D8200087FB003CC317C3EBAC0386FB03764FEAD0
:10D83000E37ECEEBE61EC1EB0116A5EB860CC0EB3A
:10D8400000154FEA8E0684F806C0A1EB85016171D0
:10D8500003EB4301A0EBC10040F2B55101FB1E33C5
:10D860002071B3F5896F37DA40F2DA218B4239DC67
:10D87000B3F5B77F2249B4BF4FF0000E4FF0010E51
:10D880000EEB4E0075464FEA4E0701EBC001B1F8B2
:10D8900036011C4907EB0E0C01EBCC0C0B210CF1F3
:10D8A000160C01E03CF8020D984212DD0139F9D165
:10D8B0007744134901EBC701B1F82001012106F5B6
:10D8C000FA6E0133A17075441B1A22812580E37022
:10D8D000F8BD0131C9B2F2E7032540F296500627A0
:10D8E000AE46D6E7022540F229400427AE46D0E7EF
:10D8F00080BC92C789888888ABAAAA2A73B06D16A3
:10D9000000760C0820770C0830B5304C8DB0864678
:10D910000D46EC461EF0030F0FCCACE80F000FCC09
:10D92000ACE80F0094E80F008CE80F000FD1284BF3
:10D93000284A03FB0EF3B2EBB30F44D3264AB2EBF3
:10D94000331F34BF01220022C2F11D0200E01C225D
:10D950000EF1FF33019240F26D122048002B194660
:10D9600002FB0EF21E4CB8BF0EF10201EE4602EBB6
:10D97000A10280FB0310DB17ADF1040101EB85016F
:10D98000A3EB6015C3EBE0132A441A44253284FB51
:10D990000230D3171044C3EBA003C3EBC303D31A65
:10D9A0005EF8040FC218714584FB023C4FEAE27333
:10D9B0009444C3EBAC03C3EBC303A2EB0303EFD16B
:10D9C000C01A0DB030BD1D22C2E700BF80770C0821
:10D9D000295C8FC2285C8F020AD7A3001F85EB51F8
:10D9E000932449920D4B10B553E9024354EA0302C4
:10D9F0000AD10146002340F2011218460B80C1F8FB
:10DA000002208B710B8110BD054A1268121943F177
:10DA10000003FFF7E9FE012010BD00BF206E0024C7
:10DA2000F030002430B5144D83B00446D5F8D81931
:10DA3000D5F8DC3951EA03020AD1002340F2011281
:10DA400018462380C4F80220A371238103B030BD9F
:10DA50000A4A1268521843F10003FFF7C5FEB5F8F1
:10DA6000E03920460DF106022146ADF8063069F096
:10DA700067FC012003B030BD40640024F030002476
:10DA800088422DE9F04198464FF0010439D301FB5B
:10DA900004F4B0FBF4FC8C45F9D264B30025BCF16E
:10DAA000000F04FB1C00B4FBF1F7D4BF00260126D5
:10DAB0006DB966B9A142354619D9C6460CF1300C8C
:10DAC0000EF801CB00238EF80030BDE8F081BCF1E8
:10DAD000090F18DD002A0CBF57233723C6466344BD
:10DAE000A14205F101050EF8013BF046EAD83C469B
:10DAF000B0FBF7FCD3E7C64600238EF80030BDE844
:10DB0000F0818446CAE73023E8E700BF2DE9F04101
:10DB10000446154608469442B4FBF2F607D205FBCC
:10DB20001644134B1B5D00F8013BBDE8F0819642A3
:10DB3000B6FBF2F70CD20E4B05FB176705FB16443C
:10DB4000DA5D1B5D00F8012B00F8013BBDE8F081B8
:10DB5000BA42B7FBF2F807D905FB1878044B13F863
:10DB6000082000F8012BE7E74046FFF7CFFFF3E777
:10DB7000C01D0D08B5EEC00ADFED357A0023F1EEC9
:10DB800010FA30B5C8BF30EE270A87B0D8BF30EEE4
:10DB9000670ADFED307A054603A9029320EE270AD3
:10DBA000CDE90033FDEEC07A17EE904A84EAE470C6
:10DBB000A0EBE4706AF098F9002C03A8B4BF2D2301
:10DBC00020238DF800306FF023FF01282AD002288F
:10DBD00034D003281ED003A9684679F09BF9684623
:10DBE0006FF016FF044669462846033CE4B222461D
:10DBF00077F0A8F9002328462B556FF009FF2E2255
:10DC0000431C0DEB04012A54E81879F0F8F9284672
:10DC100007B030BD302303A968468DF8013079F094
:10DC200079F9DCE743F23002302303A96846ADF806
:10DC300001208DF8033079F06DF9D0E743F230031D
:10DC400003A96846ADF8013079F064F9C7E700BF71
:10DC50006F12033A00007A440378202B03D110F8A6
:10DC6000013F202BFBD0092BF9D02D2B63D02B2B80
:10DC7000B7EE000A08BF01300278A2F13003D9B232
:10DC8000092961D8F2EE046ADFED4D7A07EE103A09
:10DC900010F8012FB8EEC77AA2F13003D9B2A7EE7F
:10DCA000A67A0929F0EE477AF0D92E2A50D00378C7
:10DCB00003F0DF03452B3BD110B442782D2A73D0FB
:10DCC0002B2A62D0A2F130030130092B63D8002443
:10DCD000002303EB830302EB430310F8012FA2F1AF
:10DCE0003001303B0929F4D9B3F59A7F1A46B7EED3
:10DCF000007A28BF4FF49A72072B09D91346DFED3B
:10DD0000316A083B27EE267A072BFAD802F0070281
:10DD10002AB1F2EE046A013A27EE267AFBD1002CF2
:10DD20003BD0C7EE877A5DF8044B20EE270A704798
:10DD300020EE270A704742780130BFEE000AA2F1B8
:10DD40003003D9B209299DD92E2ADFED1D7AAED133
:10DD500043780130A3F13002D1B20929A8D8B2EE3C
:10DD6000047AF0EE475A06EE902A10F8013FB8EE1A
:10DD7000E66AA3F13002D1B2C6EE076A092927EE9E
:10DD8000257A77EEA67AEED992E782780230A2F170
:10DD90003003092B9BD9B7EE007A67EE877A5DF8DE
:10DDA000044B20EE270A704782780230A2F130033C
:10DDB000092B01D801248BE7B7EE007AB1E700BF49
:10DDC0000000000020BCBE4C0378092B01D0202BA2
:10DDD00005D110F8013F202BFBD0092BF9D02D2BBA
:10DDE00009D001784FF0010CA1F13002D3B2092B18
:10DDF0000AD900207047417801304FF0FF3CA1F173
:10DE00003002D3B2092BF4D8002310F8011F03EB22
:10DE1000830302EB4303A1F13002D1B20929F4D903
:10DE20000CFB03F0704700BFAB4BAC4A2DE9F04F41
:10DE30004FF0000A97B09E1A41F221051F462C228E
:10DE400000210DEB020078F0A5F9A44AA44B08923A
:10DE5000CDE90976DA68D10707D5A24A5A6002F1FE
:10DE600088325A60DB68DC070DD49D4BD3F80C2157
:10DE7000D20708D59B4AC3F8042102F18832C3F8BF
:10DE80000421D3F80C31002101227E2308A814912B
:10DE900005A98DF854208DF81430FDF7D7FB002824
:10DEA000C0F2298108214FF4FC4303E05B000139F3
:10DEB0009BB207D01AB2002AF8DA85EA4202013989
:10DEC00093B2F7D1884AADF81630884B934280F070
:10DED000518198460DF11809CDE902A7B8F8022042
:10DEE0004FF0000CB8F80030C2F30B0B10048DF8A3
:10DEF0001DC00BF10601ADF81810C3F30B014FEA7A
:10DF00001333ADF81A108DF81C3000F19180062201
:10DF1000494608A8FDF79AFB0028C0F2FD80BDF82D
:10DF2000164049460DF11E0011F8013B082284EA13
:10DF3000032403E06400013AA4B207D023B2002B0B
:10DF4000F8DA85EA4303013A9CB2F7D18842EBD173
:10DF50005A46D8F8041008A8FDF778FB0028C0F24C
:10DF6000DB80D8F8041001EB0B00814215D0013999
:10DF7000013811F8013F082284EA032403E0640019
:10DF8000013AA4B207D023B2002BF8DA85EA4303A2
:10DF9000013A9CB2F7D18142EBD1ADF8164008F1BD
:10DFA0001408514B984599D3DDE902A700230222BA
:10DFB000494608A8ADF81830FDF748FB0028C0F224
:10DFC0009A80BDF816300DF11A0041F2210119F8BE
:10DFD000012B082483EA022303E05B00013C9BB28F
:10DFE00007D01AB2002AF8DA81EA4202013C93B261
:10DFF000F7D14845EBD102220DF1160108A8ADF882
:10E000001630FDF723FB002875DB1398002840F03D
:10E010008980149800286EDB9DF85420002A40F077
:10E02000978000280DBF012200220123002364E015
:10E03000E2466746019601370622494608A8FFB224
:10E040008DF81D70FDF702FB002851DBBDF816406E
:10E0500049460DF11E0011F8013B082284EA032411
:10E0600003E06400013AA4B207D023B2002BF8DA2F
:10E0700085EA4303013A9CB2F7D18842EBD1D8F844
:10E0800004105A4608A801EB0A063146FDF7DEFAED
:10E0900000282DDB06EB0B00864215D0711E0138DF
:10E0A00011F8013F082284EA032403E06400013AE6
:10E0B000A4B207D023B2002BF8DA85EA4303013A71
:10E0C0009CB2F7D18142EBD1032FDA44ADF8164070
:10E0D000B1D1019E63E700BF000004080000020800
:10E0E00000200052230167455CD80D08A8D20D0816
:10E0F000DDE9016A039F012300220AF1010ABAF156
:10E10000020F02DC002B7FF49AAE12B1FCF780FF05
:10E1100028B9052006F010FFDDE902A7EBE717B0EC
:10E12000BDE8F08F089B099A03449342E3D80BABF8
:10E13000C0F120022146184478F02CF8149818B940
:10E140000BA908A8F4F7AEFF00221490139261E720
:10E150000A4AD16841F00101D160D168C9077FF551
:10E1600060AFD2F80C1141F00101C2F80C11D2F8E5
:10E170000C2156E70DF1180918E700BF00200052E6
:10E1800070B545880B4604460021C5F30B051846BB
:10E190002A4677F0FFFF0A4A21690346914206D3D7
:10E1A000084A914206D31846BDE870400847002946
:10E1B000F9D170BD2A46BDE8704076F0C3BE00BFFD
:10E1C0005CD80D087FDD0D0810B50446C06900B1AC
:10E1D00010BD09211420FFF751F9E06110BD00BF07
:10E1E000174B03EB8000806838B300EB400003EB73
:10E1F000800292F9B5C0BCF1FF3F1FD092F8BD007C
:10E20000D8B103EB0C00002310B590F808E18C2086
:10E2100092F8BC10142200FB0CFC0A4C0CEB010021
:10E22000013A714434F8100013FA80F3F6D1064A2B
:10E23000A2FB0320C0F30F1010BD704700207047F1
:10E240004064002400000030CDCCCCCC036810B575
:10E250001A790446022A03D000232360237110BDDB
:10E26000987A04F099FA0028F6D040F61A61002254
:10E27000C1802021027204F04BFA00232360237135
:10E2800010BD00BF2DE9F04FBA4E85B0BA4CA64282
:10E2900056D21D4602E00C36A64251D273798B420B
:10E2A000F9D13379834201D00028F4D1F379934234
:10E2B000F1D13468002C43D0002326606360A36052
:10E2C000E36023616361A361E36133792371012B0F
:10E2D00096F806B0C4F808B0317AE16032D0022B6B
:10E2E0002ED1F07A04F058FA96F90970A061B07A4C
:10E2F000277404F051FA06466061F0B1DFF89482A9
:10E3000007EB47017B0058F8319008EBC1010193FE
:10E31000B9F1000F11D0887DE8B10E2200230D2144
:10E320003046F2713372B57104F0F2F93368B28895
:10E330009A61204605B0BDE8F08F2046FFF786FFC2
:10E340000024F6E7F07A04F027FA727AB37AA06133
:10E3500022746374EDE7B1F808A0504669F0EAF85A
:10E3600001214FEA5A100AF01F0A023801FA0AF195
:10E37000092812D8DFE810F0F6001100EE001801AD
:10E380001001E600E000D800D0000A007B4BD3F873
:10E390009C0020EA0101C3F89C107B00D91908EB0E
:10E3A000C101487904F0F8F9791CCBB20146019318
:10E3B00018B1037240F60A30C8807B000291D81968
:10E3C00008EBC000C07904F0E7F902990346039016
:10E3D00020B1019A027240F60A50D8807B00029167
:10E3E000D81908EBC000807904F0D6F9029982466A
:10E3F00028B1019B037240F60A40AAF806007B0090
:10E40000D8191BF0040308EBC0000293807A02467F
:10E41000084614BF4E212E2104F09CF903987B007E
:10E420002E2103EB070B08EBCB0B9BF80B2004F022
:10E4300091F950469BF80C200E2104F08BF99BF8C3
:10E4400004A0BAF1000F40F0ED80D9F8002022F0CE
:10E450000102C9F800204A4A914500F0C180494AAA
:10E46000914540F0AC80454AD2F8901041F480418B
:10E47000C2F89010D2F8901021F48041C2F89010A8
:10E48000029B002B40F098804FF000714FF080729B
:10E49000D9F80C0040F00040C9F80C00D9F8080089
:10E4A00020F4F070C9F80800D9F80000C00727D49C
:10E4B000D9F80800344B034034481843C9F8080021
:10E4C000D9F80C00C30005D4D9F8000040F48050FE
:10E4D000C9F80000D9F80C0011432D4A02400A4344
:10E4E00042F08862C9F80C20D9F8002022F40062BA
:10E4F000C9F80020D9F8502022F00102C9F85020B4
:10E50000BAF1000F40F09B807B003B4408EBC3084E
:10E51000012388F8163000E7184BD3F8880020EA6A
:10E520000101C3F8881038E7144BD3F88C0020EAB7
:10E530000101C3F88C1030E7104BD86F20EA0101BD
:10E54000D9672AE70D4BD3F8940020EA0101C3F8FC
:10E55000941022E7094BD3F8800020EA0101C3F8A8
:10E5600080101AE7054BD3F8980020EA0101C3F8A0
:10E57000981012E7A0020008800400080044025826
:10E580000030014000380040E0FFBF8F070000204E
:10E59000FFFF39D8A80200243E4BD3F8900020EAB0
:10E5A0000101C3F89010F8E63A4BD3F8840020EA52
:10E5B0000101C3F88410F0E600210A4668E7364AF4
:10E5C00091451BD1334AD2F8901041F40041C2F872
:10E5D0009010D2F8901021F40041C2F890104FE74B
:10E5E0002C4AD2F8981041F48051C2F89810D2F811
:10E5F000981021F48051C2F8981041E7274A9145BC
:10E6000027D0274A914532D1224AD2F8981041F4B6
:10E610008011C2F89810D2F8981021F48011C2F835
:10E6200098102DE7504604F0B7F820B1019B40F652
:10E630000A620372C2800D2104F06AF805E75046B1
:10E6400004F0AAF800283FF45FAF02688388936162
:10E650005AE7104AD2F8981041F40051C2F89810C5
:10E66000D2F8981021F40051C2F8981008E70D4A2A
:10E6700091457FF405AF02F50C32D2F89C1041F0C1
:10E680002001C2F89C10D2F89C1021F02001C2F8A1
:10E690009C10F5E600440258003C00400034014064
:10E6A0000050014000140058104B70B5104CA342AC
:10E6B00019D2054602E00C33A34214D293F805C0E8
:10E6C0008C45F8D193F804C00DB1AC45F3D1D8799D
:10E6D0009042F0D1186890F804E0E645EBD1066866
:10E6E0009E42E8D170BD002070BD00BFA0020008AE
:10E6F000800400080379022B00D0704790F91020A5
:10E7000008311C4802EB420210B41B4C83B050F895
:10E71000322000946944194C11F808CCA24224D04C
:10E7200017498A4223D001F580618A4205D0154BF2
:10E730009A420CBF03234FF0FF33116803EB4303EE
:10E7400021F0010100EBC30011600169936851F8E9
:10E750002C1023F0E0430B439360136843F0010354
:10E76000136003B05DF8044B70470023E5E7012315
:10E77000E3E700BFA80200240001020300300140CB
:10E78000003800400034014090F91030F0B503EB40
:10E790004303284E154683B056F833600446836819
:10E7A0009A0719D501230DF106028DF8061030469F
:10E7B0000DF10701F5F7B6FC01230DF106020DF18D
:10E7C000070130468DF80650F5F7ACFCA3689B07AF
:10E7D00016D5012003B0F0BD43691BB19A881868B3
:10E7E00012048261144B154A1868154BC000576813
:10E7F000A3FB003080095368DB1B9842FBD2D1E7B2
:10E800000D4A4FF4FA700E4B12680C4900FB02F2ED
:10E810004868A3FB023292094B681B1A9A42FBD24A
:10E820006369002BD5D01A6801209B88936103B0DF
:10E83000F0BD00BFA802002480360024001000E0D4
:10E84000D34D621010B5037984B084468E46012BF7
:10E850000DD0022B02D0002004B010BD8368DB076E
:10E8600058BF01F07F0104B0BDE810408CE781681B
:10E870000DF10F001446724601F001018DF80F40B2
:10E88000CDE900019CF811109CF91000F4F738FF55
:10E8900004B010BD2DE9F0410768642682B0B622AD
:10E8A0007E2180463846FFF7CDFF05F067FE04461F
:10E8B0000D4605F063FE001B61EB0501B0F57A7FA4
:10E8C00071F10001F5D3013EEFD102213846FFF787
:10E8D00011FF7B691BB19A88196812048A6105F0DF
:10E8E0004DFE04460D4605F049FE001B61EB050197
:10E8F000B0F57A7F71F10001F5D37B6913B11A6825
:10E900009B8893610A2605F039FE04460D4605F002
:10E9100035FE001B61EB0501B0F57A7F71F1000156
:10E92000F5D3013EEFD132467C213846FFF78AFF0E
:10E9300005F024FE04460D4605F020FE001B61EBA9
:10E940000501B0F57A7F71F10001F5D3002259215C
:10E950003846FFF777FF05F011FE04460D4605F037
:10E960000DFE001B61EB0501B0F57A7F71F100012E
:10E97000F5D397F910305E218D4A03EB43038DF8F0
:10E98000071052F83340BB689A0740F1E480012336
:10E990000DF1070200212046F5F7C4FB4FF4A473E4
:10E9A000844A20460021F5F7BDFBBB689B0740F178
:10E9B000E6800A2605F0E2FD04460D4605F0DEFD80
:10E9C000001B61EB0501B0F57A7F71F10001F5D311
:10E9D000013EEFD1012259213846FFF733FF05F000
:10E9E000CDFD04460D4605F0C9FD001B61EB050198
:10E9F000B0F57A7F71F10001F5D38C2240213846C1
:10EA0000FFF720FF05F0BAFD04460D4605F0B6FD00
:10EA1000001B61EB0501B0F57A7F71F10001F5D3C0
:10EA2000032241213846FFF70DFF05F0A7FD0446FC
:10EA30000D4605F0A3FD001B61EB0501B0F57A7FE3
:10EA400071F10001F5D35C4C0323D8F8382098F815
:10EA50003500B4FBF2F291B2584AFEF7E5FD438867
:10EA60004221B4FBF3F4C8F840400279384642F042
:10EA7000C002FFF7E7FE05F081FD04460D4605F0F4
:10EA80007DFD001B61EB0501B0F57A7F71F100019E
:10EA9000F5D3082243213846FFF7D4FE05F06EFD7A
:10EAA00004460D4605F06AFD001B61EB0501B0F55B
:10EAB0007A7F71F10001F5D3042258213846FFF71F
:10EAC000C1FE05F05BFD04460D4605F057FD001B39
:10EAD00061EB0501B0F57A7F71F10001F5D30A22EF
:10EAE00053213846FFF7AEFE05F048FD04460D46BB
:10EAF00005F044FD001B61EB0501B0F57A7F71F173
:10EB00000001F5D300227C213846FFF79BFE05F07B
:10EB100035FD04460D4605F031FD001B61EB050196
:10EB2000B0F57A7F71F10001F5D306227D213846D8
:10EB3000FFF788FE05F022FD04460D4605F01EFD98
:10EB4000001B61EB0501B0F57A7F71F10001F5D38F
:10EB500002B0BDE8F0817B691BB11A689B881B0479
:10EB60009361174B17491A68174BD2004868A3FBEB
:10EB7000023292094B681B1A9A42FBD207E7104AED
:10EB80004FF4FA70104B12680E4900FB02F248680D
:10EB9000A3FB023292094B681B1A9A42FBD27B6993
:10EBA000002B3FF406AF1A689B88936101E700BF12
:10EBB000A8020024B0770C0840420F00F8780C0837
:10EBC00080360024001000E0D34D62102DE9F041A2
:10EBD000816B0623654D044607686426644A90F8F5
:10EBE0003500B5FBF1F189B2FEF71EFD4388002127
:10EBF00080463846B5FBF3F52564FFF77BFD8022A0
:10EC00006B213846FFF71EFE05F0B8FC04460D46A2
:10EC100005F0B4FC001B61EB0501B0F57A7F71F1E2
:10EC20000001F5D3013EEFD1642607226821384662
:10EC3000FFF708FE05F0A2FC04460D4605F09EFC19
:10EC4000001B61EB0501B0F57A7F71F10001F5D38E
:10EC5000013EEFD1324664266B213846FFF7F2FDC4
:10EC600005F08CFC04460D4605F088FC001B61EBAA
:10EC70000501B0F57A7F71F10001F5D3013EEFD1C6
:10EC80000F2601226B213846FFF7DCFD05F076FCEC
:10EC900004460D4605F072FC001B61EB0501B0F562
:10ECA0007A7F71F10001F5D3013EEFD10F261822D2
:10ECB0001B213846FFF7C6FD05F060FC04460D46F3
:10ECC00005F05CFC001B61EB0501B0F57A7F71F18A
:10ECD0000001F5D3013EEFD10F2618221C21384642
:10ECE000FFF7B0FD05F04AFC04460D4605F046FC72
:10ECF000001B61EB0501B0F57A7F71F10001F5D3DE
:10ED0000013EEFD10F2698F804201A213846FFF76C
:10ED100099FD05F033FC04460D4605F02FFC001B61
:10ED200061EB0501B0F57A7F71F10001F5D3013E89
:10ED3000EFD1642698F8052019213846FFF782FDA7
:10ED400005F01CFC04460D4605F018FC001B61EBA9
:10ED50000501B0F57A7F71F10001F5D3013EEFD1E5
:10ED600038460321BDE8F041C4E400BF40420F0033
:10ED70000C790C082AE700BF00680379012B09D041
:10ED8000022B01D0002070478368F022DB0717D5E3
:10ED9000FF21F9E4826890F910C002F00102417C81
:10EDA00060464FF0F00C10B584B00DF10F040192E5
:10EDB000FF228DF80FC00094F4F7A2FC04B010BD40
:10EDC0007F21E1E40068CA43037941EA0211012B83
:10EDD000CAB208D0022B01D0002070478368DB073D
:10EDE00015D5D221D0E410B584B0846890F910C054
:10EDF0008DF80F200DF10F0204F00104417C009208
:10EE0000D22260460194F4F77BFC04B010BD52217D
:10EE1000BAE400BF00680379012B09D0022B01D0AE
:10EE2000002070478368B422DB0717D5FF21ABE4CD
:10EE3000826890F910C002F00102417C60464FF0F8
:10EE4000B40C10B584B00DF10F040192FF228DF8BF
:10EE50000FC00094F4F754FC04B010BD7F2193E47C
:10EE600000680379012B09D0022B01D000207047E4
:10EE700083680A46DB0715D5A52185E410B584B063
:10EE8000846890F910C00DF10F0204F001048DF8B0
:10EE90000F10417C60460092A5220194F4F730FCEB
:10EEA00004B010BD25216FE400680379012B09D05F
:10EEB000022B01D00020704783689622DB0717D50C
:10EEC000FF2161E4826890F910C002F00102417CE8
:10EED00060464FF0960C10B584B00DF10F0401920E
:10EEE000FF228DF80FC00094F4F70AFC04B010BDA7
:10EEF0007F2149E400680379012B09D0022B01D05E
:10EF00000020704783680A46DB0715D587213BE45C
:10EF100010B584B0846890F910C00DF10F0204F0B0
:10EF200001048DF80F10417C604600928722019405
:10EF3000F4F7E6FB04B010BD072125E40068C90121
:10EF40000379CAB2012B05D0022B01D000207047F3
:10EF5000782119E410B584B0846890F910C08DF858
:10EF60000F200DF10F0204F00104417C0092782281
:10EF700060460194F4F7C4FB04B010BD0068037947
:10EF8000012B0AD0022B01D0002070478368552244
:10EF9000DB0718D5A521FFF7F7BB826890F910C0F1
:10EFA00002F00102417C60464FF0550C10B584B070
:10EFB0000DF10F040192A5228DF80FC00094F4F713
:10EFC0009FFB04B010BD2521FFF7DEBB006803796D
:10EFD000012B0AD0022B01D00020704783682E221B
:10EFE000DB0718D5F421FFF7CFBB826890F910C07A
:10EFF00002F00102417C60464FF02E0C10B584B047
:10F000000DF10F040192F4228DF80FC00094F4F773
:10F0100077FB04B010BD7421FFF7B6BB154B006839
:10F020001A8F03799201012B02F13402D2B209D076
:10F03000022B01D0002070478368DB0716D5F4212E
:10F04000FFF7A2BB10B584B0846890F910C08DF8AA
:10F050000F200DF10F0204F00104417C0092F42214
:10F0600060460194F4F74CFB04B010BD7421FFF727
:10F070008BBB00BF40640024006810B5037984B0E6
:10F08000012B0FD0022B02D0012004B010BD8368E9
:10F090003122DB074CBFF4217421FFF775FB0120FF
:10F0A00004B010BD82680DF10F0490F910C002F099
:10F0B0000102417C60464FF0310C0192F422009431
:10F0C0008DF80FC0F4F71CFB012004B010BD00BF89
:10F0D00000680379012B07D0022B01D00020704774
:10F0E00001225821FFF750BB8268417C02F00102E7
:10F0F00010B590F9104084B020460DF10F04019234
:10F10000582200948DF80F30F4F7FAFA04B010BDCD
:10F1100000680379012B07D0022B01D00020704733
:10F1200001224821FFF730BB8268417C02F00102D6
:10F1300010B590F9104084B020460DF10F040192F3
:10F14000482200948DF80F30F4F7DAFA04B010BDBD
:10F1500000680379012B07D0022B01D000207047F3
:10F160001A460821FFF710BB826890F910C002F020
:10F170000102417C60464FF0020C10B584B00DF1E5
:10F180000F04019208228DF80FC00094F4F7B8FA2A
:10F1900004B010BD00680379012B07D0022B01D009
:10F1A0000020704701220821FFF7EEBA8268417CF7
:10F1B00002F0010210B590F9104084B020460DF124
:10F1C0000F040192082200948DF80F30F4F798FA9A
:10F1D00004B010BD2DE9F04105461F4628481646EB
:10F1E00095F9103082B003EB430350F83380AB68DD
:10F1F0009A0716D501230DF106028DF80610404638
:10F200000DF10701F4F78EFF3B46324600214046E0
:10F21000F4F788FFAB689B0718D5012002B0BDE862
:10F22000F0816B691BB19A88186812048261154BD2
:10F230001868154BC000A3FB0030144B80095A68B6
:10F240005C68A4EB020C6045FAD2D3E70D4A4FF498
:10F25000FA700D4B12680D4900FB02F24868A3FBDF
:10F26000023292094B681B1A9A42FBD26B69002B3F
:10F27000D3D01A6801209B88936102B0BDE8F08169
:10F28000A802002480360024D34D6210001000E054
:10F2900030B5057983B084468E46012D0DD0022D00
:10F2A00002D0002003B030BD8468E40758BF41F0AD
:10F2B000800103B0BDE830408CE7806814460A4600
:10F2C000009400F001049CF811109CF910000194C6
:10F2D000F4F716FA03B030BD2DE9F04105461F469C
:10F2E0002848164695F9103082B003EB430350F8D6
:10F2F0003380AB689A0716D501230DF106028DF80D
:10F30000061040460DF10701F4F70CFF3B460022C2
:10F3100031464046F4F706FFAB689B0718D501203D
:10F3200002B0BDE8F0816B691BB19A8818681204BD
:10F330008261154B1868154BC000A3FB0030144BBD
:10F3400080095A685C68A4EB020C6045FAD2D3E7E6
:10F350000D4A4FF4FA700D4B12680D4900FB02F292
:10F360004868A3FB023292094B681B1A9A42FBD2EF
:10F370006B69002BD3D01A6801209B88936102B07F
:10F38000BDE8F081A802002480360024D34D62102D
:10F39000001000E030B5057983B084468E46012D1B
:10F3A0000DD0022D02D0002003B030BD8468E407E8
:10F3B00058BF41F0800103B0BDE830408CE7806861
:10F3C00014460A46009400F001049CF811109CF9C0
:10F3D00010000194F4F7B0FB03B030BD2DE9F04309
:10F3E000816B85B0804C0623076880467F4A96264D
:10F3F00090F83500B4FBF1F189B2FEF715F94388B6
:10F40000002181463846B4FBF3F4C8F84040FFF7CA
:10F4100071F980226B213846FFF714FA05F0AEF837
:10F4200004460D4605F0AAF8001B61EB0501B0F596
:10F430007A7F71F10001F5D3013EEFD196260322C8
:10F4400068213846FFF7FEF905F098F804460D46A6
:10F4500005F094F8001B61EB0501B0F57A7F71F1BE
:10F460000001F5D3013EEFD103226B213846FFF7AF
:10F47000E9F905F083F804460D4605F07FF8001B16
:10F4800061EB05010F2871F10001F6D310226A210A
:10F490003846FFF7D7F905F071F804460D4605F038
:10F4A0006DF8001B61EB05010F2871F10001F6D327
:10F4B00000226C213846FFF7C5F905F05FF80446D5
:10F4C0000D4605F05BF8001B61EB05010F2871F19B
:10F4D0000001F6D399F8052019213846FFF7B2F953
:10F4E00005F04CF804460D4605F048F8001B61EBAA
:10F4F00005010F2871F10001F6D318221B213846AF
:10F50000FFF7A0F905F03AF804460D4605F036F885
:10F51000001B61EB05010F2871F10001F6D31822E1
:10F520001C213846FFF78EF905F028F804460D46F1
:10F5300005F024F8001B61EB05010F2871F10001B3
:10F54000F6D399F804201A213846FFF77BF905F025
:10F5500015F805460C4605F011F88C4208BF8542A7
:10F56000F9D003213846FFF7C5F8062302AA432144
:10F57000D8F80000FFF70EFF28B3BDF80810BDF85B
:10F580000A30BDF80C20C9BADBBA07EE901AD2BA1D
:10F59000F8EEE76A07EE102A07EE903AB8EEC77A5F
:10F5A000F8EEE77AC8ED076A88ED097AC8ED087ABF
:10F5B000FDEEE77ACDED017A9DF90430013305D0F7
:10F5C00005B0BDE8F083D8ED087AF1E7D8ED077A09
:10F5D000FDEEE77ACDED017A9DF904300133EFD1EC
:10F5E000062005F0A9FC00BF40420F000C790C0872
:10F5F00070B5066882B00546F469002C3ED03379B8
:10F60000221D012B2DD0022B26D1B368304613F0DA
:10F61000010F4FF00C030CBF8C211946FFF75CFE65
:10F62000A070D8B1B4F9043007EE903AF8EEE77A5A
:10F63000C5ED077AB4F9063007EE903AF8EEE77AAE
:10F64000C5ED087AB4F9083007EE903AF8EEE77A9B
:10F65000C5ED097A02B070BD0023A370002002B08E
:10F6600070BDB368717C03F0010396F9100000923D
:10F6700001930C231A46F4F75FFAD1E7092114200D
:10F68000FDF7FCFEF06104462E68B8E770B5066829
:10F6900082B00546F469002C3ED03379E21C012B80
:10F6A0002DD0022B26D1B368304613F0010F4FF056
:10F6B0000D0314BF0C218C21FFF70EFEA070D8B1F2
:10F6C000B4F90A3007EE903AF8EEE77AC5ED077A1A
:10F6D000B4F90C3007EE903AF8EEE77AC5ED087A07
:10F6E000B4F90E3007EE903AF8EEE77AC5ED097AF4
:10F6F00002B070BD0023A370002002B070BDB368DB
:10F70000717C03F0010396F9100000920C22019322
:10F710000D23F4F711FAD1E709211420FDF7AEFE0D
:10F72000F06104462E68B8E7006810B5037984B02C
:10F730000C46012B1AD0022B02D0002004B010BDC1
:10F74000836803AA13F0010F4FF0030314BF2221B3
:10F75000A221FFF7C1FD0028EFD0BDF90D3003EB6A
:10F7600083031B12E633238004B010BD836803AA11
:10F77000417C03F0010390F91000009222220193D2
:10F780000323F4F7D9F9E6E770B5066882B00546B9
:10F79000F469002C3ED03379221D012B2DD0022B91
:10F7A00026D1B368304613F0010F4FF00E0314BF9B
:10F7B0003B21BB21FFF790FDA070D8B1A389DBBA34
:10F7C00007EE903AF8EEE77AC5ED077AE389DBBAFF
:10F7D00007EE903AF8EEE77AC5ED087A238ADBBAAD
:10F7E00007EE903AF8EEE77AC5ED097A02B070BDFF
:10F7F0000023A370002002B070BDB368717C03F0D9
:10F80000010396F9100000923B2201930E23F4F7B6
:10F8100093F9D1E709211420FDF730FE0446F06189
:10F82000B9E700BF006810B5037984B0012B10D090
:10F83000022B01D000200AE003AAF621FFF74CFDBD
:10F840000028F7D0BDF80C30094A5BBA138304B026
:10F8500010BD826803AC417C022302F0010290F9E2
:10F860001000CDE90042F622F4F766F9E8E700BFA0
:10F8700040640024006810B5037984B0012B1DD0CA
:10F88000022B01D0002017E0032303AAF621FFF783
:10F8900023FD0028F6D09DF80D309DF80CC01B020A
:10F8A0000D499DF80E2043EA0C431343B1F938206B
:10F8B000C2F10802D340CB6304B010BD826803AC30
:10F8C000417C032302F0010290F91000CDE90042CF
:10F8D000F622F4F731F9DCE740640024006810B543
:10F8E000037984B0012B31D0022B09D01E490020AE
:10F8F000D1F8E439D1F8E8290B660A6404B010BDE8
:10F90000062302AAF721FFF7E7FC0028EED09DF8B6
:10F9100009309DF80C209DF808C01B019DF80BE0F4
:10F9200012019DF80A1043EA0C3342EA0E329DF8A8
:10F930000DC043EA11130C4942EA1C12C1F8E43924
:10F94000C1F8E8290A640B6604B010BD826802ACF5
:10F95000417C062302F0010290F91000CDE900423B
:10F96000F722F4F7E9F8D0E740640024006810B506
:10F97000037984B0012B1DD0022B0FD09DF80D30E0
:10F9800001209DF80CC01B029DF80E10104A43EA9E
:10F990000C430B43C2F8883004B010BD836803AA3F
:10F9A00013F0010F4FF0030314BF00218021FFF774
:10F9B00093FCE3E7826803AC417C032302F001027D
:10F9C00090F91000CDE900420022F4F7B5F8D5E730
:10F9D00040640024006810B5037984B0012B1DD069
:10F9E000022B0FD09DF80D3001209DF80CC01B029A
:10F9F0009DF80E10104A43EA0C430B43C2F89C30AA
:10FA000004B010BD836803AA13F0010F4FF0030385
:10FA100014BF00218021FFF75FFCE3E7826803AC9D
:10FA2000417C032302F0010290F91000CDE900426D
:10FA30000022F4F781F8D5E740640024006810B58F
:10FA4000037984B0012B28D0022B01D0002022E0C2
:10FA5000836803AA13F0010F4FF003030CBF832147
:10FA60001946FFF739FC0028F0D09DF80C309DF9BD
:10FA70000C109DF80D201B0400299DF80EC043EAD0
:10FA800002230D4AACBF00214FF07F4143EA0C0333
:10FA90000B43C2F8103104B010BD826803AC0323DD
:10FAA000417C02F0010290F91000CDE900421A46B3
:10FAB000F4F742F8D7E700BF40640024006810B5AF
:10FAC000037984B0012B28D0022B01D0002022E042
:10FAD000836803AA13F0010F4FF0030314BF002142
:10FAE0008021FFF7F9FB0028F0D09DF80C309DF93C
:10FAF0000C109DF80D201B0400299DF80EC043EA50
:10FB000002230D4AACBF00214FF07F4143EA0C03B2
:10FB10000B43C2F80C3104B010BD826803AC417CC9
:10FB2000032302F0010290F91000CDE90042002207
:10FB3000F4F702F8D7E700BF4064002490F91030D2
:10FB4000F0B503EB4303264E154683B056F83360F9
:10FB5000044683689A0715D501230DF106028DF836
:10FB6000061030460DF10701F4F7DCFA01230022FC
:10FB700029463046F4F7D6FAA3689B0716D501202C
:10FB800003B0F0BD43691BB19A8818681204826102
:10FB9000144B154A1868154BC0005768A3FB00307A
:10FBA00080095368DB1B9842FBD2D5E70D4A4FF41E
:10FBB000FA700E4B12680C4900FB02F24868A3FB76
:10FBC000023292094B681B1A9A42FBD26369002BDE
:10FBD000D5D01A6801209B88936103B0F0BD00BFA7
:10FBE000A802002480360024001000E0D34D6210EB
:10FBF00010B5037982B08E46012B0DD0022B02D0B6
:10FC0000002002B010BD8368DB0758BF41F08001BF
:10FC100002B0BDE8104091E7816814467246009436
:10FC200001F00104417C90F910000194F3F784FF86
:10FC300002B010BD70B5056884B004460E462B793D
:10FC4000012B15D0022B02D0002004B070BDAB6890
:10FC5000E122DB071CD528461146FEF795FD00285A
:10FC6000F2D03246FF21206804B0BDE87040BFE703
:10FC7000AA68697C02F0010295F910000DF10F05E8
:10FC80000192E12200958DF80F20F3F739FDE6E7A8
:10FC900061212846FEF778FDE1E700BF70B50568F1
:10FCA00084B004460E462B79012B16D0022B02D0CD
:10FCB000002004B070BDAB68C3222846DB074CBFF0
:10FCC000E1216121FEF760FD0028F1D03246FF21DD
:10FCD000206804B0BDE870408AE7AA6895F9100072
:10FCE00002F00102697C01920DF10F020092C32221
:10FCF0008DF80F20E122F3F703FDE5E770B5056805
:10FD000084B004460E462B79012B1BD0022B02D067
:10FD1000002004B070BDAB68F0222846DB074CBF62
:10FD2000E1216121FEF730FD0028F1D02246FF21BC
:10FD300052F8040BFFF75CFF0028E9D023793370F9
:10FD400004B070BDAA6895F9100002F00102697C48
:10FD500001920DF10F020092F0228DF80F20E122A6
:10FD6000F3F7CEFCE0E700BFF0B5046883B00021F4
:10FD7000074664262046FEF7BDFC15227E2120465C
:10FD8000FEF760FD04F0FAFB04460D4604F0F6FBB6
:10FD9000001B61EB0501B0F57A7F71F10001F5D32D
:10FDA000013EEFD1052611227E213868FEF74AFD7B
:10FDB00004F0E4FB04460D4604F0E0FB001B61EB9D
:10FDC0000501B0F57A7F71F10001F5D3013EEFD165
:10FDD0000DF1070203213868FFF70AFF9DF807308D
:10FDE00003F03C03142B40F09B800C224021386828
:10FDF000FEF728FD04F0C2FB04460D4604F0BEFBEE
:10FE0000001B61EB0501B0F57A7F71F10001F5D3BC
:10FE1000454C0923B96B454A97F83500B4FBF1F11D
:10FE200089B2FDF701FC0346422138685A88B4FBC9
:10FE3000F2F43C641A79FEF705FD04F09FFB0446DA
:10FE40000D4604F09BFB001B61EB0501B0F57A7FCA
:10FE500071F10001F5D3082241213868FEF7F2FC68
:10FE600004F08CFB04460D4604F088FB001B61EB9C
:10FE70000501B0F57A7F71F10001F5D3002243212D
:10FE80003868FEF7DFFC04F079FB04460D4604F009
:10FE900075FB001B61EB0501B0F57A7F71F1000184
:10FEA000F5D3102251213868FEF7CCFC04F066FB34
:10FEB00004460D4604F062FB001B61EB0501B0F542
:10FEC0007A7F71F10001F5D30A2253213868FEF7D9
:10FED000B9FC04F053FB04460D4604F04FFB001B35
:10FEE00061EB0501B0F57A7F71F10001F5D3802255
:10FEF00056213868FEF7A6FC04F040FB04460D4688
:10FF000004F03CFB001B61EB0501B0F57A7F71F159
:10FF10000001F5D303213868FEF7ECFB03B0F0BD18
:10FF2000062005F009F800BF40420F00747D0C0860
:10FF3000F0B583B015461C4606460DF107020F4684
:10FF4000FFF756FE9DF8072005EA0203A34201D100
:10FF500003B0F0BD22EA050239463046224303B021
:10FF6000BDE8F040FEF76EBC10B582B00821044633
:10FF700000686A46FFF73CFE9DF80030DB0602D4BD
:10FF8000002002B010BD06236A4600212068FFF75A
:10FF900001FA0028F4D09DF801209DF8001012020B
:10FFA0009DF80230DFED4A6A02EB01429DF8041031
:10FFB00014024FEA01219DF8034013449DF80520E7
:10FFC00001EB044148BF03F17F430A44090207EEF5
:10FFD000903A404B48BF02F17F42F8EEE77A93ED4A
:10FFE0001B6A07EE102AB3F97020F8EEC65AB3F96F
:10FFF0007610B8EEC77A04EE901AB3F97A10C7EE0D
:020000040805ED
:10000000263A87EEA67A06EE902A334AD3ED1A7A7C
:1000100092F8FC43B3F97220F8EEE66A112C06EE72
:10002000102AB3F97420F8EEE77A05EE102AB3F936
:100030007820B8EEC66A04EE102AB8EEC55AF8EE7B
:10004000E44AB3F97C20B8EEC44A66EEA36A27EE10
:10005000232A23D0A7EE045AA7EE246AE5EE075A16
:10006000E5EE877A77EEA67AE6EE027AB3F96620B5
:10007000F6EE006AC3ED207A07EE902AB3F9641019
:10008000F8EEE77A07EE101AB8EEC77A67EEA37AB1
:10009000E7EE267AC3ED217A02B010BD03EE102AF6
:1000A000F8EEC32A03EE101AB8EEC33AA7EE224ABE
:1000B000E7EE034AA4EE075AA4EE876AE5EE075A74
:1000C000E5EE877A77EEA67AE6EE027ACEE700BF13
:1000D000000078484064002418B90024F0B50446B4
:1000E00083B00D461746061D20680379012B19D0F1
:1000F000022B02D0002003B0F0BD83683246FF21FE
:10010000DB075CBF3246FF21FFF718FD0028F1D066
:1001100015B12379DB07E7D4002FECD023793B70AE
:1001200003B0F0BD8268417C02F0010C90F9100030
:10013000FF22CDE9006CF3F7FFFCE7E770B504465A
:10014000051D82B020680379012B16D0022B02D046
:10015000002002B070BD83682A46FF21DE075CBF25
:100160002A46FF21FFF7EAFC0028F1D02379DB07BC
:10017000EFD520680379012BE8D18668FF22417C06
:1001800006F0010690F91000CDE90056F3F7D4FC13
:10019000EAE700BF024630B5044652F8040B83B0CC
:1001A0000379012B0ED0022B01D0002008E0FF21A3
:1001B000FFF7C4FC0028F8D02079C04300F001000C
:1001C00003B030BD8568417C05F0010590F9100051
:1001D0000092FF220195F3F7AFFCEBE770B5B42274
:1001E00082B00446FF210068FEF72CFB10B9002006
:1001F00002B070BD2068251D0379012B13D0022B9E
:10020000F5D183682A46FF21DE075CBF2A46FF211D
:10021000FFF794FC0028EAD02379DB07E8D52068B3
:100220000379012BEBD18668FF22417C06F00106A1
:1002300090F91000CDE90056F3F77EFCEAE700BF25
:1002400070B50A4682B00446A5210068FEF7FAFAA6
:1002500010B9002002B070BD2068251D0379012B64
:1002600013D0022BF5D183682A46FF21DE075CBF3D
:100270002A46FF21FFF762FC0028EAD02379DB073A
:10028000E8D520680379012BEBD18668FF22417CF9
:1002900006F0010690F91000CDE90056F3F74CFC8A
:1002A000EAE700BF70B582B00446CDE90023FFF74E
:1002B00095FF10B9002002B070BD5522A52120681D
:1002C000FEF7C0FA0028F5D0251D2A46FF21206838
:1002D000FFF78EFC0028EDD02379DB07F5D40DF174
:1002E000FF350DF1070615F8011F2046FFF7A8FF9F
:1002F0000028DFD0B542F6D1DDE700BF002A34D0B8
:10030000F0B5044683B00E46051D8F1816F8012B74
:10031000A5212068FEF796FA90B9002003B0F0BD41
:100320008268417C02F0010C90F91000FF22CDE9B7
:10033000005CF3F701FC0028EFD02379DB070FD531
:1003400020680379012BEBD0022BE6D183682A4683
:10035000FF21DB075CBF2A46FF21FFF7EFFBEAE73F
:10036000B742D3D1012003B0F0BD0120704700BFD8
:10037000F0B5962283B00E460446FF210068FEF7D2
:1003800061FA10B9002003B0F0BD251D2068037983
:10039000012B1DD0022BF5D183682A46FF21DF07F0
:1003A0005CBF2A46FF21FFF7C9FB0028EAD023796A
:1003B000DB07EBD4E12220681146FEF743FA002860
:1003C000E0D03246FF21206803B0BDE8F0400FE4E2
:1003D0008768FF22417C07F0010790F91000CDE902
:1003E0000057F3F7A9FBE0E7002A42D0F0B5044636
:1003F00083B00E46051D8F189622FF212068FEF758
:1004000021FA90B9002003B0F0BD8268417C02F06F
:10041000010C90F91000FF22CDE9005CF3F78CFB92
:100420000028EFD02379DB070FD520680379012B53
:10043000EBD0022BE6D183682A46FF21DB075CBFA5
:100440002A46FF21FFF77AFBEAE7E12220681146FE
:10045000FEF7F8F90028D5D03246FF212068FFF7D3
:10046000C7FB0028CED00136B742C5D1012003B06A
:10047000F0BD0120704700BFF0B50B46054616469B
:10048000044683B087211A4655F8040BFEF7DAF9C3
:1004900020680379012B19D0022B02D0002003B071
:1004A000F0BD83682A46FF21DF075CBF2A46FF2193
:1004B000FFF744FB0028F1D02379DA07E8D4002EB7
:1004C000EDD0C3F34013337003B0F0BD8768FF2253
:1004D000417C07F0010790F91000CDE90057F3F7D0
:1004E0002BFBE7E7F0B5782183B0164604460022DF
:1004F0000068FEF7A7F910B9002003B0F0BD251D74
:1005000020680379012B13D0022BF5D183682A468A
:10051000FF21DF075CBF2A46FF21FFF70FFB002802
:10052000EAD02379DA07EBD45B09337003B0F0BD6E
:100530008768FF22417C07F0010790F91000CDE9A0
:100540000057F3F7F9FAEAE770B5CC2282B0044617
:10055000A5210068FEF776F910B9002002B070BD41
:100560002068251D0379012B13D0022BF5D1836858
:100570002A46FF21DE075CBF2A46FF21FFF7DEFA8D
:100580000028EAD02379DB07E8D520680379012B1E
:10059000EBD18668FF22417C06F0010690F910003D
:1005A000CDE90056F3F7C8FAEAE700BF70B5B42208
:1005B00082B00446FF210068FEF744F910B900201C
:1005C00002B070BD251D20680379012B21D0022BBC
:1005D000F5D183682A46FF21DE075CBF2A46FF214A
:1005E000FFF7ACFA0028EAD02379DA07EBD4CC2164
:1005F0002046FFF725FE0028E1D002E02379DB0743
:10060000DED52A46FF212068FFF7F2FA0028F5D14F
:10061000D5E78668FF22417C06F0010690F91000BC
:10062000CDE90056F3F788FADCE700BF2DE9F04F7B
:1006300082468DB0002090460AF10407089106908A
:100640000A930790069B5046DC0008EBC303059312
:10065000FFF7C4FD28B941E09AF8043013F0010215
:1006600008D03A46FF21DAF80000FFF7C1FA002867
:10067000F2D133E003929A070B9040F1CC80F02145
:100680005046FFF7DDFD48B3083CDDF80C9008EB61
:100690000403012409932546089B003B18BF01234E
:1006A0000493049B082D8CBF002303F001039B4699
:1006B000002B5DD06E1E089B43FA06F606F001067D
:1006C000F2017821DAF80000FEF7BCF830B1DAF870
:1006D00000000379012B3FD0022B07D000220A9B98
:1006E0001046069919700DB0BDE8F08F83683A4640
:1006F000FF21DB075CBF3A46FF21FFF71FFA002806
:10070000ECD09AF8043013F00102E0D199094FEAD5
:10071000531E4FEAD31C01EA5313DB074BD4664543
:1007200002D0BBF1000F73D1BCF1000F2DD00599A1
:1007300011F80930234301F809306400013514F041
:10074000FF04EDB2ADD109F101095FFA89F9B9F100
:10075000080F30D00124A4E78268417C02F0010C2C
:1007600090F91000FF22CDE9007CF3F7E5F9C6E728
:10077000069BD3B1079BAB4217D9099B13F80930ED
:100780001C4214BF012600269AE74EEA0101039B92
:1007900011F0010F059908BF2B46039311F809309A
:1007A00023EA040301F80930C7E7079B5E1BB6FA8A
:1007B00086F6760984E7402D07D80A9B069A1B78AF
:1007C00093423FF63FAF024689E7059BDD795C1E09
:1007D0009E1D14F801CF082182EA0C0301394FEA6B
:1007E0005C0C43F3000311F0FF0123F0730383EA71
:1007F0005202D2B2F0D1A642EBD19542DDD1069B96
:100800000133DBB20693039B002BDCD00793D4E7C4
:100810000B9E324663E70646324660E710B5044653
:10082000006882B003796A46022B4FF006030CBFC2
:1008300043210321FEF7AEFD68B1BDF80010BDF8FD
:100840000220BDF8043049BA52BA5BBAE186628729
:10085000238702B010BDC4F83600608702B010BD17
:1008600030B5002385B004460221C0F836300DF1C2
:10087000070243870068FFF7BBF918B19DF80730FE
:10088000DB0703D40025284605B030BD062302AAA5
:1008900003212068FEF77EFD0DF107020921206883
:1008A000FFF7A6F905460028ECD09DF8073013F0B5
:1008B0000C0FE7D1BDF80820BDF80C30BDF80A10C8
:1008C000C2EB8232C3EB8333206889009B00920025
:1008D000218763870A21E2860122FDF7B3FF2846BC
:1008E00005B030BD10B50446002221210068FDF797
:1008F000A9FFFC2220212068FDF7A4FF402224212B
:100900002068FDF79FFF0C2223212068FDF79AFF46
:10091000002222212068FDF795FF012010BD00BFB5
:1009200010B5044694220B210068FDF78BFF71225D
:1009300001212068FDF786FF002204212068FDF7D1
:1009400081FFC82205212068FDF77CFF00220621D7
:100950002068FDF777FFC82207212068FDF772FFA6
:10096000002208212068FDF76DFFC82209212068B8
:10097000FDF768FF012010BD01207047044B0022E5
:10098000002101201A605A609A60D960704700BF48
:10099000E0DA0024104B11491A680346C868121A9D
:1009A000FA2A16D8D1ED006A012091ED017AFDEE08
:1009B000E66AD1ED027ABDEEC77AFDEEE77A16EE71
:1009C000902ADA8617EE102A1A8717EE902A5A878D
:1009D00070470020704700BFF0300024E0DA0024A8
:1009E0000E4B70B51B7C82B00191ABB90C4B1D68EE
:1009F00095B12B681A687AB19B686BB1044628469A
:100A0000984748B1019922462E6828460B4631681E
:100A100002B0BDE87040084702B070BDE0DA0024C3
:100A200040AC00240B4B70B51E688EB133681A6859
:100A300072B19B6863B1054630460C46984738B1A1
:100A400031682A46234630460968BDE870400847A9
:100A500070BD00BF58AC0024014B5B695B68184750
:100A6000E0DA0024024B08305B699B68184700BF3E
:100A7000E0DA002401207047012070470120704710
:100A8000012070470120704731B10B4BD3ED067A3E
:100A9000F8EEE77AC1ED007A6AB10749074BC969F8
:100AA000DFED076A0B4407EE903AF8EEE77A87EE3F
:100AB000A67A82ED007A7047E0DA00244D95FFFFB8
:100AC0000000C84201207047012070477A4A014661
:100AD00000239446104610B490F904400C30012CC9
:100AE0004DD00133082BF7D1734C002394F9040047
:100AF0000C34022858D00133082BF7D16E4C002358
:100B000094F904000C3403286BD00133082BF7D17F
:100B1000694C002394F904000C34052877D0013384
:100B2000082BF7D1644C002394F904000C340628F8
:100B300000F083800133082BF6D1002392F90400E2
:100B40000C32072800F093800133082BF6D15B4B61
:100B50001B68DC0340F1A180594B086803F58C74D5
:100B600003E01433A34200F098801A689042F8D151
:100B7000DA68D201F5D501205DF8044B704703EB2C
:100B800043035CF8233023B34E480B7990F8D140EF
:100B900090F8D000984218BF9C420CBF0120002062
:100BA000A2D15DF8044B704703EB43035CF823309C
:100BB0008BB145480B7990F8D04090F8D10098421D
:100BC00018BF9C420CBF0120002097D15DF8044B58
:100BD0007047394C8AE7384C94F904000C340328E8
:100BE00093D103EB43035CF82330002B3BD0374811
:100BF0000B7990F8D04090F8D100984218BF9C42F1
:100C00000CBF0120002083D15DF8044B704703EB3B
:100C100043035CF8233043B32D480B7990F8D04060
:100C200090F8D100984218BF9C420CBF01200020D0
:100C30007FF478AF5DF8044B704703EB43035CF837
:100C40002330002B3FF47AAF22480B7990F8D04044
:100C500090F8D100984218BF9C420CBF01200020A0
:100C60008AD003466AE7144C54E7134C5CE703EB65
:100C700043035CF82330002B3FF469AF164A0B792D
:100C800092F8D10092F8D0209A4218BF98420CBF37
:100C9000012000207FF45BAF6EE70B79312B04D885
:100CA0002F2B94BF0020012066E7343B012B8CBF23
:100CB0000020012060E700BF3C8C0024D86E002497
:100CC0000803002448070024200A0024F80C00240C
:100CD000D00F0024A8120024801500240B4B84465A
:100CE000002010B503F58C7E02E014339E450BD036
:100CF0001A686245F9D1DA68441C8A42F5D0D96095
:100D00001433E0B29E45F3D110BD00BF08030024A8
:100D1000704700BF40F2FF72034B914203EBC003E8
:100D2000A8BF114699847047E0DA0024112807D83B
:100D3000044B03EB8003D3F880300BB19B68196040
:100D40002AF066BCE0DA0024112807D8044B03EB34
:100D50008003D3F880300BB19B681960704700BFE7
:100D6000E0DA0024F0B5484D83B095F8C8303BB1C7
:100D700095F8C9600446012E38D0022E54D00EB129
:100D800003B0F0BD012280210068FDF75BFD012268
:100D9000FF212068FDF756FD324631462068FDF7F9
:100DA00051FD95F8CA2091212068FDF74BFD314691
:100DB00001222068FDF746FD3246FF212068FDF73D
:100DC00041FD324680212068FDF73CFD314601227D
:100DD0002068FDF737FD2D4B2D4901221B68087057
:100DE00085F8C920C5F8CC3003B0F0BD01AA0021B8
:100DF0000068FEF7FDFE9DF80430254FDA073870D5
:100E000039D5D5F8D030002BBAD0204AD5F8CC103F
:100E1000126892B2521A9342B2D24FF0FF320023BC
:100E20007A6085F8C930ABE701AA13210068FEF7A4
:100E3000DFFE9DF80430164F5B073870E1D0334673
:100E400001AA1E212068FEF7A5FABDF8043020682B
:100E500001225CBA0B21FDF7F5FC0E4BA4B2012276
:100E60003870A3FB0434002385F8D420E40885F807
:100E7000C9307C6084E7054B02221B6885F8C920D5
:100E8000C5F8CC307CE700BFE0DA0024F030002465
:100E9000FC1D0024CDCCCCCC0C4A13787BB10C4B80
:100EA00093F8C81059B193F8D41059B15068002282
:100EB000FA2883F8D420A8BF4FF0FF3070476FF0B6
:100EC000010070476FF00200704700BFFC1D002456
:100ED000E0DA00242DE9F041104C002517460223EA
:100EE00004F1D80884F8D910FF210646424684F858
:100EF000D850FEF7CDF968B1424630460223FF21B3
:100F0000FEF748FA30B1B4F8D83028465BBA3B80D7
:100F1000BDE8F0816FF00C00FAE700BFE0DA0024D2
:100F20000B4B93F8D82182B193F8D92152B10949DA
:100F30000022886883F8D921B0F5967FA8BF4FF0CA
:100F4000FF3070476FF0020070476FF0010070478C
:100F5000E0DA0024FC1D0024024BD3F8DC315B688E
:100F6000184700BFE0DA0024024BD3F8DC319B685D
:100F7000184700BFE0DA0024024BD3F8DC31DB680D
:100F8000184700BFE0DA0024014BD868704700BF63
:100F9000FC1D0024044B93F8E03113B1034B186996
:100FA00070476FF001007047E0DA0024FC1D002458
:100FB00070B52F4C05460323002104F5F27200683A
:100FC000FEF7E8F958B96FF00103C4F8E831294A8F
:100FD000D4F8EC31116832338B423FD370BDB4F892
:100FE000E421F2EE046A94F8E6C1082152BA94F8BA
:100FF000E43192B207EE902AF8EEE77A87EEA67A0D
:10100000BDEEC77A84ED7A7A58B25B0042000028C0
:10101000DBB282F00702B8BFD3B20139F4D194F841
:10102000E5210821534058B25B0042000028DBB2A2
:1010300082F00702B8BFD3B20139F4D19C45C6D1C2
:10104000D4F8E8312BB1D4F8E8214FF6FF739A4277
:10105000BDD14FF0FF33C4F8E831B8E7C4F8EC1164
:10106000012328683121044ABDE87040FEF710B919
:10107000E0DA0024F0300024D0DC0024014BD3F867
:10108000E8017047E0DA0024437A5A1C0344D2B2E4
:1010900042729972037A934200D802B9704703688A
:1010A00000F10A0110B504464068984700236372B6
:1010B00010BD00BF026830B5137985B00446012B1E
:1010C00061D0022B03D00025284605B030BD9168C1
:1010D00002AD1046C9072A464CBF19468221FEF7C9
:1010E0002DFD0028EFD09DF80830DA07EBD52A4611
:1010F000072303212068FEF74DF905460028E2D0BA
:1011000011220A212068FDF79DFB9DF80E301B0778
:10111000D9D42A49BDF80830B1F8F02113FB02F305
:10112000274A93423EDBB3F5000F39DA002BB8BFF4
:10113000FF331B125B421BB2BDF80A20E386B1F8F5
:10114000F23112FB03F31E4A93422FDBB3F5000F7B
:1011500030DA002BB8BFFF3343F30F22BDF80C3059
:10116000B1F8F411228713FB01F3154A93421BDBFC
:10117000B3F5000F1CDA002BB8BFFF331B125B4224
:101180001BB26387A0E7517C02AD92F91000926810
:10119000009502F0010201920222F2F7CDFCA0E7D5
:1011A000084BC9E7084BC7E7074BEAE7064AD5E70C
:1011B000044BE6E747F6FF72D0E700BFE0DA002411
:1011C00001FF7FFF0180FFFF0080FFFF10B50023BC
:1011D00086B0044600688DF80F300379012B31D0BA
:1011E000022B02D0002006B010BD83680DF10F0263
:1011F000D9074CBF2721A721FEF7A0FC0028F1D07A
:101200009DF80F301B07EDD5062304AA282120687E
:10121000FEF7C0F828B3BDF91030002BB8BF033378
:101220009A10BDF91230002BE286B8BF03339A1032
:10123000BDF91430002B2287B8BF03339B1063879E
:1012400006B010BD8268417C02F0010290F910C026
:1012500001920DF10F02604600922722F2F76CFC1A
:10126000CCE7C4F8360060870020BCE730B54FF00B
:10127000000C0446006887B0C4F836C0A4F83AC031
:101280000379012B2AD0022B02D0002007B030BDF9
:1012900083680DF10F02D9074CBF61468021FEF72C
:1012A0004DFC0028F1D09DF80F301B07EDD506232B
:1012B00004AA01212068FEF76DF80028E5D0BDF8EA
:1012C0001430BDF81010BDF812205BBA49BA52BAFA
:1012D0005B42E1862287638707B030BD856862463E
:1012E000417C05F0010590F9100001950DF10F0505
:1012F0000095F2F721FCD4E710B5002304460068FE
:1013000086B0C4F8363063870379012B23D0022BD3
:1013100002D0002006B010BD83680DF10F02D9077E
:101320004CBF06218621FEF709FC0028F1D09DF86C
:101330000F305B07EDD5062304AA00212068FEF7D5
:1013400029F80028E5D0049ABDF81430C4F83620F6
:10135000638706B010BD8268417C02F0010290F9FB
:1013600010C001920DF10F02604600920622F2F7C2
:10137000E3FBDAE710B500230446006886B0C4F842
:10138000363063870379012B29D0022B02D000204D
:1013900006B010BD83680DF10F02D9074CBF0921BB
:1013A0008921FEF7CBFB0028F1D09DF80F30DB0739
:1013B000EDD5062304AA01212068FDF7EBFF0028E4
:1013C000E5D0BDF81210BDF81020BDF81430494228
:1013D00052425B42E1862287638706B010BD826875
:1013E000417C02F0010290F910C001920DF10F0250
:1013F000604600920922F2F79FFBD4E710B5002364
:101400000446006886B0C4F8363063870379012B40
:1014100012D0022B0DD183680DF10B02DB074CBFFC
:101420003421B421FEF78AFB18B19DF90B30002B53
:1014300011DB002006B010BD8268417C02F0010281
:1014400090F910C001920DF10B0260460092342217
:10145000F2F772FBE8E7092303AA24212068FDF7CD
:1014600099FF0028E5D09DF810209DF80F109DF8F9
:10147000133012041B0442EA01629DF8121043EA81
:1014800001639DF80C10C2F30F42C3F30F43228790
:1014900063879DF80D301B0443EA0163C3F30F43D8
:1014A000E38606B010BD00BF0A4600212DE9F041D9
:1014B000DFF8B08084B042F001020446274EFDF709
:1014C000C1F9D8F80070264DC6F8CC7018E0022B90
:1014D0004FF000000BD1A3680DF10F02132120463D
:1014E000DB0702D40DF10F029321FEF727FB9DF8D5
:1014F0000F30287013F0070318D1D6F8D0202ABB7C
:101500002379012BE3D1A2680DF10F0102F0010252
:10151000009101921322617C94F91000F2F70CFB08
:101520009DF80F30287013F00703E6D001220B213D
:101530002046FDF787F9002220461146FDF782F983
:1015400001232870184604B0BDE8F081D8F80010D7
:1015500089B2C91B8A42D3D2F4E700BFE0DA002483
:10156000FC1D0024F030002410B50446006884B04F
:101570000379012B43D0022B07D0002213461046DB
:10158000C4F83620638704B010BD836802AA13F044
:10159000010F4FF0060314BF11219121FDF79CFEAE
:1015A0000028EAD0BDF90C20B7EE086ABDF90A3070
:1015B00007EE902ABDF908205B4206EE902AF8EE6D
:1015C000E77A07EE103AF8EEE66AB8EEC77A67EE09
:1015D000867A66EE866A27EE067AFDEEE77AFDEEFB
:1015E000E66ABDEEC77A17EE903A16EE902A1BB265
:1015F000E28617EE102A6387228704B010BD836845
:1016000002AA417C03F0010390F91000009211221C
:1016100001930623F2F790FAC2E700BF10B500234A
:101620000446006884B0C4F8363063870379012B20
:1016300022D0022B01D000201CE0836802AA13F004
:10164000010F4FF0060314BF03218321FDF744FE71
:101650000028F0D0BDF90A30BDF80810BDF80C2004
:101660005B4201EB410102EB420203EB4303E186E3
:101670006287238704B010BD836802AA417C03F00F
:10168000010390F910000092032201930623F2F760
:1016900053FADDE710B54FF0000C0446006884B043
:1016A000C4F836C0A4F83AC00379012B18D0022B35
:1016B00001D0002012E0836802AA13F0010F4FF05E
:1016C000060314BF61468021FDF706FE0028F0D016
:1016D000029ABDF80C30C4F83620638704B010BD00
:1016E00083686246417C03F0010390F910E00193A6
:1016F00002AB704600930623F2F71EFAE6E700BF3E
:1017000010B5002384B0044600680293CDF80B3076
:101710000279012A1ED0022A19D1836802AA13F085
:10172000010F4FF0070314BF4E21CE21FDF7D4FD6A
:10173000BDF80910BDF80B20BDF80D30C9BAD2BAFA
:10174000DBBA0120E1862287638704B010BD1A4608
:101750001946F6E7826802AB90F910C002F0010268
:10176000417C00936046019207234E22F2F7E4F990
:10177000DEE700BF006810B5037984B0012B0BD001
